:020000040000FA
:0408000090EF07F07E
:020808003BD0E3
:0808180087D0E26BE36BE46B97
:10082000E56BF86A080EF76E000EF66A0900F550DF
:10083000E527E86AE423E323E223FF0EF762F6D715
:10084000FA0EF662F3D7E51FE41FE31FE21FE52B64
:0A085000E86AE423E323E223FFD764
:10088000026ED8CF03F0D9CF05F0DACF04F0E1CF74
:1008900007F0E2CF06F0E9CF09F0EACF08F09EBA00
:1008A0000BD0F2B201D030D0F292A081A0A32CD014
:1008B00091C092F0916B28D0AECFC9F03D8E0A0E58
:1008C000C95D22E00D0EC9630BD06B511DE022EE15
:1008D00000F0D926C9C0DFFF6B6BA6EC59F014D02D
:1008E00022EE00F06B51D926C9C0DFFF6B2B3E0E04
:1008F000C96302D03F8008D03FA006D0200EC96354
:1009000003D03F823F906B6B05C0D9FF04C0DAFF74
:1009100007C0E1FF06C0E2FF09C0E9FF08C0EAFF27
:10092000025003C0D8FF1000006ED8CF01F0E9CF0D
:100930000AF0EACF0BF0A4AA18D0A49A1AEE00F09D
:100940006ECFF7F00A0EF75DD8B4AED2F851E126BB
:10095000F7C0E7FF0D0EF76306D0E12AE76AF86BF0
:100960005EEC63F0A1D2F82B9FD2F0A203D0F092FC
:1009700035809AD2F2A498D2F294AA2F1ED00A0EF1
:10098000AA6FA0B3912B39B002D0809816D083AE55
:10099000808883BE809883AE678983BE67996739F4
:1009A0006719010BE8A009D067A904D067816785A2
:1009B000679303D0679167956783AB67AB07B167B0
:1009C000B107AD5305E0AE0703E1640EAE6FAD07AE
:1009D000AF5305E0B00703E1640EB06FAF07B25349
:1009E00005E0B40703E10A0EB46FB207B35305E0A4
:1009F000B50703E1640EB56FB307B65305E0B7075B
:100A000003E10A0EB76FB607B85305E0B90703E173
:100A1000640EB96FB80760EC07F036B462D036B236
:100A200024D036B00DD035A06FD03590C26BC36BDB
:100A3000366A376A36800A0EB46F050EB26F64D01C
:100A4000B26702D0366A60D035A05ED0359036905D
:100A50003682C26BC46BC36B0A0EB46F140EB26FD6
:100A6000640EB56F2D0EB36F4FD0C22B35B017D0BB
:100A7000B2674AD036923684369636A80CD0358284
:100A8000358635843698640EB56F2D0EB36FC46B02
:100A9000C26BC36B39D035923594359635D03590CD
:100AA0000A0EB46F140EB26F36B605D0C2C0C3F0D2
:100AB000C26B367629D03676C251C327430EC36146
:100AC0000BD00F0EC36508D0C36BC26BC42B050ED1
:100AD000C4651AD0368818D03696C46BC26BC36B07
:100AE00013D0B36704D0366AC00E35160DD035A0CA
:100AF0000BD03590C46BC26BC36B3682369436967E
:100B00000A0EB46F1E0EB26F3AA6E3EF05F03AB0CC
:100B1000BDEF05F03AB2A1EF05F06C2FE3EF05F061
:100B2000140E6C6F80746D2FE3EF05F01D50D8B478
:100B30003A841BC06DF03A828086809480828090D7
:100B400042D06C2FE3EF05F0140E6C6F6D2FE3EFC6
:100B500005F01C5008E06D6F3A923A8080868094D0
:100B60008092808030D01AC06DF03A923A90C52BB6
:100B7000808680948092808026D03AB2D2EF05F0B1
:100B80006C2FE3EF05F0140E6C6F80746D2FE3EFA4
:100B900005F01DC06DF03A823A8480868094808290
:100BA000809011D06C2FE3EF05F0140E6C6F6D2F59
:100BB000E3EF05F01AC06DF03A923A90C52B8086AB
:100BC000809480928080BFAF6FD1010EC06308D047
:100BD000000EC16304D0B5EC5DF0C12B65D164D1CA
:100BE000020EC06345D0000EC1630BD0C12BE0C91B
:100BF000E8FFFF0BD8B458D15CEC07F0C0EC5DF017
:100C000053D1010EC1630DD0B6674ED1C12BE1C9DE
:100C1000E8FFFF0BD8B448D15CEC07F0F5EC5DF0D1
:100C200043D1020EC1630DD0B6673ED1C12BE2C9DC
:100C3000E8FFFF0BD8B438D15CEC07F0C0EC5DF0F6
:100C400033D1030EC1630DD0B6672ED1C12BE3C9DA
:100C5000E8FFFF0BD8B428D15CEC07F0F5EC5DF0B1
:100C600023D1040EC16320D1B6671ED1C16B1CD144
:100C7000030EC06345D0000EC1630BD0C12BE4C985
:100C8000E8FFFF0BD8B410D15CEC07F0CBEC5DF0C3
:100C90000BD1010EC1630DD0B66706D1C12BE5C9DA
:100CA000E8FFFF0BD8B400D15CEC07F0F5EC5DF089
:100CB000FBD0020EC1630DD0B667F6D0C12BE6C9DA
:100CC000E8FFFF0BD8B4F0D05CEC07F0CBEC5DF0A4
:100CD000EBD0030EC1630DD0B667E6D0C12BE7C9D8
:100CE000E8FFFF0BD8B4E0D05CEC07F0F5EC5DF06A
:100CF000DBD0040EC163D8D0B667D6D0C16BD4D0D8
:100D0000040EC06345D0000EC1630BD0C12BE8C9EF
:100D1000E8FFFF0BD8B4C8D05CEC07F0D6EC5DF070
:100D2000C3D0010EC1630DD0B667BED0C12BE9C9D7
:100D3000E8FFFF0BD8B4B8D05CEC07F0F5EC5DF041
:100D4000B3D0020EC1630DD0B667AED0C12BEAC9D5
:100D5000E8FFFF0BD8B4A8D05CEC07F0D6EC5DF050
:100D6000A3D0030EC1630DD0B6679ED0C12BEBC9D3
:100D7000E8FFFF0BD8B498D05CEC07F0F5EC5DF021
:100D800093D0040EC16390D0B6678ED0C16B8CD067
:100D9000050EC06363D0000EC16307D0C12B0A0EDD
:100DA0005CEC07F0B5EC5DF07FD0010EC16309D0BB
:100DB000B6677AD0F5EC5DF0C12B0A0E5CEC07F05B
:100DC00073D0020EC16309D0B6676ED0B5EC5DF08A
:100DD000C12B0A0E5CEC07F067D0030EC16309D08B
:100DE000B66762D0F5EC5DF0C12B0A0E5CEC07F043
:100DF0005BD0040EC16309D0B66756D0C12BB5ECE9
:100E00005DF00A0E5CEC07F04FD0050EC16309D00F
:100E1000B6674AD0F5EC5DF0C12B0A0E5CEC07F02A
:100E200043D0060EC16309D0B6673ED0B5EC5DF085
:100E3000C12BFA0E5CEC07F037D0070EC16307D068
:100E4000B66732D0C12BF00E5CEC07F02DD0080E47
:100E5000C1632AD0B66728D0C16B26D0060EC06306
:100E600023D0000EC16307D0E1EC5DF0C12B0A0E68
:100E70005CEC07F019D0010EC16309D0B66714D03D
:100E8000F5EC5DF0C12B0A0E5CEC07F00DD0020E04
:100E9000C1630AD0B66708D0E1EC5DF0010EC16F06
:100EA0000A0E5CEC07F000D00AC0E9FF0BC0EAFFB5
:100EB000005001C0D8FF1000B66F0A0EB76F1200C5
:100EC0000001D42BFA0ED46324D0D46BD32B040EA0
:100ED000D3631FD0D36BD52BBA67BA07010EBB5FA4
:100EE000E86ABC5BBB6707D0BC6705D026C0BBF017
:100EF00027C0BCF06481010EBD5FE86ABE5BBD67C0
:100F000007D0BE6705D065C0BDF066C0BEF0648581
:100F100034801200D880EF50E75ED8A0E76C120052
:100F2000C26A0F0EC16E070EB46E806A816A826A51
:100F3000836A846A856A866A000E926E070E936ED3
:100F4000B80E946EA10E956E090E966E000E976EF9
:100F5000140E986E82928290838684888492848410
:100F6000808A8186D66AD76A530ED56ED58E336A4B
:100F7000326A0001D36BD46BD56BF86BA16B996BA4
:100F8000A66BA76B346A646BBF6B356A366A376AC7
:100F9000386A396A3A6A3B6A576A586A596A5A6AB9
:100FA000676B3D6A3F6AA06B6B6B426A8A6B140E7B
:100FB000976F00EE43F0EE6A972FFDD7400E976FC4
:100FC00004EEC0F0EE6A972FFDD7976B0DEE00F0A0
:100FD0001EEE00F0EE68E668972FFCD7120E976FB2
:100FE00001EE8CF011EE9EF0200EEE6EE66E972F65
:100FF000FBD77BEC60F08EEC5FF08E6F9DEC5FF0CA
:101000008F6FABEC5FF08388690EAF6E260EAC6E0F
:10101000920EAB6E080E6F6E260E6C6E920E6B6E9D
:10102000D08EF28AF194F294F288F292F16AF06A28
:10103000F0889F8A9D8A9F989D98A59AA38AA598D3
:10104000A398F28CF28EF28C34EC62F095EC62F0A4
:10105000A66BA76B53EC5FF08086809480828090B3
:101060008690DB0EF76E660EF66E20EED6F0F5EC8F
:1010700061F0F50EF76E340EF66E20EEE6F0F5EC4C
:1010800061F013EC62F0640EAE6F0A0EAD6FAD67E7
:1010900047EF08F029EC5EF0CBEC35F030A2DAEC4B
:1010A00035F030B213D039AE09D0EF0EF76E360EF0
:1010B000F66E20EEE6F0F5EC61F008D0EF0EF76E7C
:1010C000460EF66E20EEE6F0F5EC61F039AC09D094
:1010D000EF0EF76E160EF66E20EED6F0F5EC61F020
:1010E00008D0EF0EF76E260EF66E20EED6F0F5EC79
:1010F00061F013EC62F0640EAE6F140EAD6FAD676D
:10110000FED721EC5EF0A5EC5EF0A66BA76B53EC6E
:101110005FF0A68753EC5FF0A78953EC5FF0300EC9
:101120002414E86664873994EF0EF76E560EF66E57
:1011300020EED6F0F5EC61F0DB0EF76ED60EF66E13
:1011400020EEE6F0F5EC61F013EC62F08280576A75
:10115000640EAE6F050EAD6FAD67FED78290640E64
:10116000AE6F140EAD6FAD67FED7050E976F3D9055
:101170003D92D70EF76EB40EF66E23EE00F0EEEC55
:1011800061F0DE6ADFEC61F0640EAE6F140EAD6FDD
:101190003DB0E2EF08F0AD67FBD7972FE8D7DC0E44
:1011A000F76E160EF66E20EED6F0F5EC61F0DC0E62
:1011B000F76E260EF66E20EEE6F0F5EC61F013EC1D
:1011C00062F0FFD73D903D92D80EF76E120EF66E8C
:1011D00023EE00F0EEEC61F0DE6ADFEC61F0640E0D
:1011E000AE6F320EAD6F3DB0FCEF08F03DB2CFEF09
:1011F00008F0AD67F8D7D3D7640EAE6F0A0EAD6FA7
:10120000AD67FED73D903D92D80EF76E2E0EF66E6E
:1012100023EE00F0EEEC61F0DE6ADFEC61F0640ECC
:10122000AE6F320EAD6F3DB01CEF09F03DB2CFEFA7
:1012300008F0AD67F8D7B3D7640EAE6F140EAD6F7C
:10124000AD67FED73D903D92D80EF76E460EF66E16
:1012500023EE00F0EEEC61F0DE6ADFEC61F0640E8C
:10126000AE6F320EAD6F3DB03CEF09F03DB2CFEF47
:1012700008F0AD67F8D793D73D903D92D80EF76E42
:10128000FA0EF66E23EE00F0EEEC61F0DE6ADFECB3
:1012900061F0640EAE6F640EAD6F3DB056EF09F0B5
:1012A0003DB2CFEF08F0AD67F8D779D7640EAE6FD7
:1012B0000A0EAD6FAD67FED73D903D92D80EF76E2A
:1012C0009A0EF66E23EE00F0EEEC61F0DE6ADFECD3
:1012D00061F0640EAE6F640EAD6F57B678EF09F033
:1012E00057B078EF09F03DB03D90AD67F6D757D7CE
:1012F0005796DC0EF76EC60EF66E20EEE6F0F5ECB5
:1013000061F013EC62F03D903D92D80EF76EBE0E88
:10131000F66E23EE00F0EEEC61F0DE6ADFEC61F0D9
:10132000640EAE6F320EAD6F3DB09FEF09F03DB26F
:101330009CEF09F0AD67F8D73D92CFEF08F03D90F4
:101340003D92D70EF76ECA0EF66E23EE00F0EEEC6D
:1013500061F0DE6ADFEC61F0640EAE6F320EAD6FED
:101360003DB0BBEF09F03DB2B8EF09F0AD67F8D77B
:101370003D92CFEF08F0388C3D903D92D80EF76E3D
:10138000600EF66E23EE00F0EEEC61F0DE6ADFEC4C
:1013900061F0640EAE6F320EAD6F3DB0D7EF09F065
:1013A0003DB2D5EF09F0AD67F8D73D92F8D63D9044
:1013B000389C100E976F08EE52F018EE22F0EECF28
:1013C000E6FF972FFCD7DE0EF76E060EF66E20EEC8
:1013D000D6F0F5EC61F020C084F059EC5DF0200E01
:1013E000E16FE46F300E806380C0E1F081C0E2F015
:1013F00021C084F059EC5DF0300E806380C0E4F0D1
:1014000081C0E5F01FC0F4F147EC59F013EC62F035
:10141000640EAE6F320EAD6FAD67FED703EE00F017
:10142000410EEE6E540EEE6E2B0EEE6E570EEE6EFD
:101430004D0EEE6E420EEE6E530EEE6E3D0EEE6EE5
:101440001FC084F059EC5DF07FC0EEFF80C0EEFF5E
:1014500081C0EEFFEE6A3D6ADFEC61F0640EAE6FB4
:10146000320EAD6F3DB054EF0AF03DB23AEF0AF0E4
:10147000AD67F8D73D92EA0EF76E860EF66E20EE57
:10148000D6F0F5EC61F0EA0EF76E960EF66E20EEF1
:10149000E6F0F5EC61F013EC62F0640EAE6F320E24
:1014A000AD6FAD67FED701D03D90DB0EF76EE60E57
:1014B000F66E20EED6F0F5EC61F0DB0EF76EF60E70
:1014C000F66E20EEE6F0F5EC61F0310EE96F13EC0C
:1014D00062F0060EC06FC16BBF8F399639823886B5
:1014E0003498E2EC31F0E86658EF0FF038823D9A1C
:1014F0003D903D92D90EF76E260EF66E23EE00F06B
:10150000EEEC61F0DE6ADFEC61F0640EAE6F320E7D
:10151000AD6F3DB0A8EF0AF03DB293EF0AF0AD67B2
:10152000F8D7CFEF08F03D92DC0EF76E360EF66E70
:1015300020EED6F0F5EC61F0DC0EF76E460EF66E9E
:1015400020EEE6F0F5EC61F013EC62F08FEF14F0B2
:101550003D90640EAE6F040EAD6FAD67FED73D904B
:101560003D92D90EF76E340EF66E23EE00F0EEECDF
:1015700061F0DE6ADFEC61F0640EAE6F320EAD6FCB
:101580003DBACCEF0AF03DB0D0EF0AF03DB2CEEF5D
:101590000AF0AD67F5D703D63D9AF2D73D92FFD555
:1015A0003D90DD0EF76E560EF66E20EED6F0F5ECA1
:1015B00061F0DD0EF76E660EF66E20EEE6F0F5ECED
:1015C00061F001EE7CF010EEDEF0080E976FEECFCA
:1015D000E6FF972FFCD7310E39B4320EE96F13ECCA
:1015E00062F0976B640EAE6F640EAD6F57B005EF8F
:1015F0000BF057B828EF0BF034B020EF0BF03DB0F4
:101600001EEF0BF0AD67F2D724D05990DC0EF76EC9
:10161000B60EF66E20EED6F0F5EC61F0DC0EF76E4D
:10162000A60EF66E20EEE6F0F5EC61F0310E39B460
:10163000320EF06F13EC62F055EF0AF03D90D6D702
:101640003490070E9715F56F972B13EC62F0CED7F9
:1016500057983D903D92D70EF76ED60EF66E23EE5C
:1016600000F0EEEC61F0DE6ADFEC61F0640EAE6F6C
:10167000320EAD6F3DB045EF0BF03DB242EF0BF0D7
:10168000AD67F8D73D92CFEF08F03D9003EE00F044
:10169000410EEE6E540EEE6E2B0EEE6E570EEE6E8B
:1016A000560EEE6E520EEE6E3D0EEE6E20C084F0C3
:1016B00059EC5DF07FC0EEFF80C0EEFF81C0EEFF11
:1016C0002C0EEE6E21C084F059EC5DF07FC0EEFF71
:1016D00080C0EEFF81C0EEFFEE6A3D6ADFEC61F094
:1016E000640EAE6F320EAD6F3DB07EEF0BF03DB2CB
:1016F0007CEF0BF0AD67F8D73D92C2D33D903D90A3
:101700003D92D80EF76E3A0EF66E23EE00F0EEEC38
:1017100061F0DE6ADFEC61F0640EAE6F320EAD6F29
:101720003DB09AEF0BF03DB298EF0BF0AD67F8D7F4
:101730003D92A6D33BEC3CF0640EAE6F320EAD6F23
:101740003DB0AAEF0BF03DB2A8EF0BF0AD67F8D7B4
:101750003D9296D31CEC3CF0640EAE6F320EAD6F32
:101760003DB0BAEF0BF03DB2B8EF0BF0AD67F8D774
:101770003D9286D33D9018EE22F0E6CF7FF0E6CF83
:1017800080F0E6CF81F0330E7F6307D0340E8063A4
:1017900004D0330E816301D028D0330E7F6307D08D
:1017A000340E806304D0340E816301D01ED0340E19
:1017B0007F6307D0340E806304D0330E816301D081
:1017C00014D0360E7F6307D0350E806304D0370EF9
:1017D000816301D00AD0350E7F6307D0340E806359
:1017E00004D0310E816301D00BD13D903D92DA0ED1
:1017F000F76E6C0EF66E23EE00F0EEEC61F0DE6A32
:10180000DFEC61F0640EAE6F320EAD6F3DB010EFE5
:101810000CF03DB20EEF0CF0AD67F8D73D9230D32F
:101820003D903D92DA0EF76E5E0EF66E23EE00F0FE
:10183000EEEC61F0DE6ADFEC61F0640EAE6F320E4A
:10184000AD6F3DB02BEF0CF03DB229EF0CF0AD6762
:10185000F8D73D9215D33D903D92DA0EF76E520EB9
:10186000F66E23EE00F0EEEC61F0DE6ADFEC61F084
:10187000640EAE6F320EAD6F3DB046EF0CF03DB270
:1018800044EF0CF0AD67F8D73D92FAD23D903D9011
:101890003D92DA0EF76E120EF66E23EE00F0EEECCD
:1018A00061F0DE6ADFEC61F0640EAE6F320EAD6F98
:1018B0003DB086EF0DF03DB260EF0CF0AD67F8D7AC
:1018C0003D92F40EF76E840EF66E20EED6F0F5EC37
:1018D00061F0F40EF76E940EF66E20EEE6F0F5EC85
:1018E00061F013EC62F0640EAE6F280EAD6FAD6761
:1018F000FED719D43D903D92D90EF76EE20EF66EEA
:1019000023EE00F0EEEC61F0DE6ADFEC61F0640ED5
:10191000AE6F320EAD6F3DB095EF0CF03DB293EF70
:101920000CF0AD67F8D73D92ABD23D903D92D90E09
:10193000F76ED40EF66E23EE00F0EEEC61F0DE6A88
:10194000DFEC61F0640EAE6F320EAD6F3DB0B0EF04
:101950000CF03DB2AEEF0CF0AD67F8D73D9290D2EF
:101960003D903D92D90EF76EC60EF66E23EE00F056
:10197000EEEC61F0DE6ADFEC61F0640EAE6F320E09
:10198000AD6F3DB0CBEF0CF03DB2C9EF0CF0AD67E1
:10199000F8D73D9275D23D903D903D92D90EF76EAD
:1019A000AC0EF66E23EE00F0EEEC61F0DE6ADFECDA
:1019B00061F0640EAE6F320EAD6F3DB086EF0DF08C
:1019C0003DB2E5EF0CF0AD67F8D73D92F40EF76E3F
:1019D000840EF66E20EED6F0F5EC61F0F40EF76EA4
:1019E000940EF66E20EEE6F0F5EC61F013EC62F08A
:1019F000640EAE6F280EAD6FAD67FED793EF08F0A3
:101A00003D903D92DA0EF76EB00EF66E23EE00F0CA
:101A1000EEEC61F0DE6ADFEC61F0640EAE6F320E68
:101A2000AD6F3DB01BEF0DF03DB219EF0DF0AD679E
:101A3000F8D73D9225D23D903D92DA0EF76EA20E78
:101A4000F66E23EE00F0EEEC61F0DE6ADFEC61F0A2
:101A5000640EAE6F320EAD6F3DB036EF0DF03DB29D
:101A600034EF0DF0AD67F8D73D920AD23D903D922C
:101A7000DA0EF76E940EF66E23EE00F0EEEC61F0E7
:101A8000DE6ADFEC61F0640EAE6F320EAD6F3DB01A
:101A900051EF0DF03DB24FEF0DF0AD67F8D73D922D
:101AA000EFD13D903D903D92DA0EF76E7A0EF66ED4
:101AB00023EE00F0EEEC61F0DE6ADFEC61F0640E24
:101AC000AE6F320EAD6F3DB086EF0DF03DB26BEFF5
:101AD0000DF0AD67F8D73D92F40EF76E840EF66EFA
:101AE00020EED6F0F5EC61F0F40EF76E940EF66E83
:101AF00020EEE6F0F5EC61F013EC62F0640EAE6FF0
:101B0000280EAD6FAD67FED793EF08F03D903D9284
:101B1000D90EF76EA00EF66E23EE00F0EEEC61F03B
:101B2000DE6ADFEC61F0640EAE6F320EAD6F3DB079
:101B3000A1EF0DF03DB29FEF0DF0AD67F8D73D92EC
:101B40009FD13D903D92D80EF76EA60EF66E23EE15
:101B500000F0EEEC61F0DE6ADFEC61F0640EAE6F77
:101B6000320EAD6F3DB0BCEF0DF03DB2BAEF0DF0EF
:101B7000AD67F8D73D9284D13D903D92D80EF76E77
:101B8000E40EF66E23EE00F0EEEC61F0DE6ADFECC0
:101B900061F0640EAE6F320EAD6F3DB0D7EF0DF059
:101BA0003DB2D5EF0DF0AD67F8D73D9269D13D90CC
:101BB0003D92D80EF76EEE0EF66E23EE00F0EEECD0
:101BC00061F0DE6ADFEC61F0640EAE6F320EAD6F75
:101BD0003DB0F2EF0DF03DB2F0EF0DF0AD67F8D78C
:101BE0003D924ED13D903D92D90EF76E720EF66E3B
:101BF00023EE00F0EEEC61F0DE6ADFEC61F0640EE3
:101C0000AE6F320EAD6F3DB024EF0EF03DB20BEF74
:101C10000EF0AD67F8D73D92F40EF76EC40EF66E77
:101C200020EED6F0F5EC61F0F40EF76ED40EF66E01
:101C300020EEE6F0F5EC61F013EC62F0640EAE6FAE
:101C4000280EAD6FAD67FED73D90F00EF76E260EF5
:101C5000F66E20EED6F0F5EC61F0F00EF76E360E73
:101C6000F66E20EEE6F0F5EC61F013EC62F03D90DC
:101C70003D92DA0EF76EBE0EF66E23EE00F0EEEC3D
:101C800061F0DE6ADFEC61F0640EAE6F640EAD6F82
:101C90003DB052EF0EF03DB250EF0EF0AD67F8D709
:101CA0003D925FD03D903D92DA0EF76ECA0EF66E11
:101CB00023EE00F0EEEC61F0DE6ADFEC61F0640E22
:101CC000AE6F640EAD6F3DB06DEF0EF03DB26BEFD9
:101CD0000EF0AD67F8D73D9244D03D903D92DA0EBC
:101CE000F76ED60EF66E23EE00F0EEEC61F0DE6AD3
:101CF000DFEC61F0640EAE6F640EAD6F3DB088EF47
:101D00000EF03DB286EF0EF0AD67F8D73D9229D0C8
:101D10003D903D92DA0EF76EF40EF66E23EE00F073
:101D2000EEEC61F0DE6ADFEC61F0640EAE6FFA0E8D
:101D3000AD6F3DB0AFEF0EF03DB2ADEF0EF0AD6761
:101D4000F8D7640EAE6FFA0EAD6F3DB0AFEF0EF088
:101D50003DB2ADEF0EF0AD67F8D73D9202D03D90A9
:101D600018D0F40EF76EE40EF66E20EED6F0F5EC19
:101D700061F0F40EF76EF40EF66E20EEE6F0F5EC80
:101D800061F013EC62F0640EAE6F280EAD6FAD67BC
:101D9000FED73EEC59F03D903D92D80EF76E800E86
:101DA000F66E23EE00F0EEEC61F0DE6ADFEC61F03F
:101DB000640EAE6F640EAD6F3DB0E6EF0EF03DB257
:101DC000E4EF0EF0AD67F8D73D925AD009EE00F07F
:101DD000EECF5BF0EECF5CF0EECF5DF0EECF5EF0DD
:101DE000EECF00F0EECF00F0EECF00F0EECF00F03F
:101DF000EECF5FF0EECF60F0EECF61F0EECF62F0AD
:101E0000636B640EAE6F050EAD6FAD67FED73D9090
:101E10003D92D70EF76EB80EF66E23EE00F0EEECA4
:101E200061F0DE6ADFEC61F0640EAE6F320EAD6F12
:101E30003DB023EF0FF03DB220EF0FF0AD67F8D7C4
:101E40003D92CFEF08F03D903D92D80EF76EFA0E1E
:101E5000F66E23EE00F0EEEC61F0DE6ADFEC61F08E
:101E6000640EAE6F640EAD6F3DB03EEF0FF03DB24D
:101E70003CEF0FF0AD67F8D73D9202D03D9018D0FF
:101E8000DE0EF76E460EF66E20EED6F0F5EC61F043
:101E9000DE0EF76E560EF66E20EEE6F0F5EC61F013
:101EA00013EC62F0640EAE6F320EAD6FAD67FED70D
:101EB000040E9A6F9AC0E5F0576A586A596AAFECF7
:101EC0005DF0809A358C320EAB6FAB67FED782AA7D
:101ED0007CEF0FF0ED0EF76E660EF66E20EED6F08C
:101EE000F5EC61F0ED0EF76E760EF66E20EEE6F094
:101EF000F5EC61F0358E11D0ED0EF76E460EF66EF4
:101F000020EED6F0F5EC61F0ED0EF76E560EF66EA3
:101F100020EEE6F0F5EC61F0359E808A359C13ECFE
:101F200062F0640EAE6F140EAD6FAD67FED7FFECBE
:101F300061F009EC62F0808680948082809000D00D
:101F400067936795349A30B0348A34B893EF08F0C9
:101F500026C0BBF027C0BCF0A66BA76B53EC5FF0AC
:101F6000A68753EC5FF0809A358C320EAB6FAB676F
:101F7000FED7359E82BA358E808A359C3BEC3CF08C
:101F8000640EAE6F320EAD6F3DB0CDEF0FF03DB2CF
:101F9000CCEF0FF0AD67F8D73D923D90389E389E5C
:101FA000576A586A3D6A3E6AF66B120E976F01EEE9
:101FB0008CF011EE9EF0200EEE6EE66E972FFBD7A2
:101FC00039A41DD039963982060EC06FC16BBF8F00
:101FD000DF0EF76E660EF66E20EED6F0F5EC61F0D1
:101FE000DF0EF76E760EF66E20EEE6F0F5EC61F0A1
:101FF00013EC62F03886E2EC31F0E8665BD0A66B59
:10200000A76B53EC5FF0AFEC5DF038B6BBD264A7C2
:1020100015D0649724C09AF09A3B030E9A17000ECD
:102020009A5DD8B4F6D2010E9A5DD8B400D3020EF0
:102030009A5DD8B4A5D3CF0E2416EBD2F50EF76E69
:10204000240EF66E20EED6F0F5EC61F0EC0EF76E95
:10205000E60EF66E20EEE6F0F5EC61F035BE13D03C
:1020600000EEEEF0200E4E0EEE6E6F0EEE6E200EB7
:10207000EE6E4C0EEE6E690EEE6E6E0EEE6E650E30
:10208000EE6E200EEE6E38B2348238B2388038B23E
:102090000FD0389000EEE6F04E0EEE6E6F0EEE6E44
:1020A000200EEE6E470EEE6E530EEE6E4D0EEE6E81
:1020B00013EC62F034BAA7EF10F067B5C0EF12F07E
:1020C00067B3BEEF12F081A29CEF14F05AB06AEF32
:1020D00012F05AB26DEF12F05AB46DEF12F05AB618
:1020E0006DEF12F05AB86AEF12F05ABA6DEF12F0B3
:1020F00035B27EEF18F038B457EF1FF03BB6ADEFB6
:1021000027F038BA7CEF2AF057B081EF12F057B2BF
:1021100097EF12F059B0B6EF12F059B2BBEF12F0D0
:1021200034B071EF14F06BA203D06B9800006B8891
:1021300024C081F0300E8117100E815D54E024C060
:1021400081F0030E8117010E8163B4D7FBD0349A5E
:102150003D903D92D80EF76E200EF66E23EE00F005
:10216000EEEC61F0DE6ADFEC61F0640EAE6F320E11
:10217000AD6F3DB0DCEF10F03DB2C1EF10F0AD67D8
:10218000F8D73D92F40EF76E440EF66E20EED6F0C0
:10219000F5EC61F0F40EF76E540EF66E20EEE6F0FC
:1021A000F5EC61F013EC62F0640EAE6F280EAD6FCB
:1021B000AD67FED73090C4D63D90F40EF76E640E36
:1021C000F66E20EED6F0F5EC61F0F40EF76E740EBC
:1021D000F66E20EEE6F0F5EC61F013EC62F081A211
:1021E0009CEF14F0FCD764A565D76495040E976F37
:1021F0008A2B040E8A618A6B19EEA2F0080E8A03FC
:10220000F350E126F450E222E6CF7CF0E6CF7DF0F9
:10221000E6CF7EF0E6CF7FF0E6CF80F0E6CF81F02C
:10222000E6CF7AF0E6CF7BF0200E7D5D04E07A67A2
:102230001FD07B671DD08A2B972FDED7DD0EF76E60
:10224000E60EF66E20EED6F0F5EC61F0DD0EF76EE0
:10225000F60EF66E20EEE6F0F5EC61F013EC62F0AF
:10226000640EAE6F320EAD6FAD67FED755EF0AF05C
:1022700003EE00F0410EEE6E540EEE6E2B0EEE6E7F
:10228000430EEE6E4F0EEE6E500EEE6E530EEE6E71
:102290003D0EEE6E310EEE6E2C0EEE6E320EEE6ECA
:1022A0002C0EEE6E7CC0EEFF7DC0EEFF7EC0EEFF1A
:1022B0007FC0EEFF80C0EEFF81C0EEFF000EEE6E2D
:1022C0003D6A576A586ADFEC61F0640EAE6FC80E63
:1022D000AD6F3DB098EF11F03DB271EF11F0AD6709
:1022E000F8D73D92DD0EF76E960EF66E20EED6F024
:1022F000F5EC61F0DD0EF76EB60EF66E20EEE6F050
:10230000F5EC61F07CC0E0F07DC0E1F07EC0E2F071
:102310007FC0E3F080C0E4F081C0E5F013EC62F030
:10232000640EAE6F320EAD6FAD67FED755EF0AF09B
:1023300064957AC065F07BC066F065C0BDF066C08C
:10234000BEF07CD664A1B6D664913EEC59F03D90C7
:102350003D92D80EF76E800EF66E23EE00F0EEEC96
:1023600061F0DE6ADFEC61F0640EAE6F640EAD6F9B
:102370003DB0C2EF11F03DB2C0EF11F0AD67F8D73C
:102380003D9298D6060E976F632B060E6361636BC2
:1023900009EE16F0160E6303F350E926F450EA2610
:1023A000EECF7AF0EECF7BF0EECF7CF0EECF7DF08B
:1023B000EECF7EF0EECF7FF0300E286412D07A514F
:1023C000286285D07B51296282D07C512A627FD0DD
:1023D0007D512B627CD07E512C6279D07F512D6251
:1023E00076D0EECF7AF0EECF7BF0EECF7CF0EECF72
:1023F0007DF0200E7A5D6BE07A515B620AD07B51F2
:102400005C6207D07C515D6204D07D515E6201D078
:102410005ED07AC0C2F97BC0C3F97CC0C4F97DC06C
:10242000C5F909EE24F0160E6303F350E926F450C3
:10243000EA26EECFC6F9EECFC7F9EECFC8F9EECF58
:10244000C9F9EECF7EF0EECF7FF0EECF80F0EECF89
:1024500081F0200E7F5D300ED8B47F6F200E805D3E
:10246000300ED8B4806F0FEC5DF0845125602FD012
:10247000C2C95BF0C3C95CF0C4C95DF0C5C95EF0F8
:1024800003EE00F0410EEE6E540EEE6E2B0EEE6E6D
:10249000430EEE6EEE6E450EEE6E4C0EEE6EEE6E72
:1024A0003D0EEE6EC6C9EEFFC7C9EEFFC8C9EEFF0E
:1024B000C9C9EEFFEE6A5A6ADFEC61F0C6C95FF087
:1024C000C7C960F0C8C961F0C9C962F0F3D5972FD8
:1024D0005BD7F0D55A905A98EDD55A6AE60EF76E4A
:1024E000160EF66E20EED6F0F5EC61F0E60EF76E05
:1024F000260EF66E20EEE6F0F5EC61F013EC62F0DD
:10250000D9D5579038903492DC0EF76E560EF66E91
:1025100020EED6F0F5EC61F0DC0EF76E760EF66E7E
:1025200020EEE6F0F5EC61F013EC62F0C3D55792C3
:1025300038903492DC0EF76E560EF66E20EED6F022
:10254000F5EC61F0DC0EF76E860EF66E20EEE6F02E
:10255000F5EC61F013EC62F039963982640EAE6FDF
:10256000140EAD6FAD67FED755EF0AF05990389055
:10257000349255EF0AF0599255EF0AF06793C2D79B
:102580006795D6D738961EC09AF09A3B030E9A17D5
:10259000000E9A630ED03D903D92D70EF76EEE0E70
:1025A000F66E23EE00F0EEEC61F0DE6ADFEC61F037
:1025B0001ED0010E9A630ED03D903D92D70EF76E5D
:1025C000FA0EF66E23EE00F0EEEC61F0DE6ADFEC60
:1025D00061F00DD03D903D92D80EF76E060EF66E6E
:1025E00023EE00F0EEEC61F0DE6ADFEC61F0640EE9
:1025F000AE6F320EAD6F3DB007EF13F03DB204EF9A
:1026000013F0AD67F8D703D53D9207EF10F03D907A
:10261000FED43D903D92D90EF76E000EF66E23EE7D
:1026200000F0EEEC61F0DE6ADFEC61F007D5040E3D
:10263000976F8A6B19EEA2F0080E8A03F350E12619
:10264000F450E222E6CF7CF0E6CF7DF0E6CF7EF0DC
:10265000E6CF7FF0E6CF80F0E6CF81F0E6CF7AF0EC
:10266000E6CF7BF0200E7D5D04E07A671FD07B67AC
:102670001DD08A2B972FDED7DD0EF76EE60EF66E95
:1026800020EED6F0F5EC61F0DD0EF76EF60EF66E8C
:1026900020EEE6F0F5EC61F013EC62F0640EAE6F44
:1026A000280EAD6FAD67FED755EF0AF003EE00F0D0
:1026B000410EEE6E540EEE6E2B0EEE6E430EEE6E6F
:1026C0004F0EEE6E500EEE6E530EEE6E3D0EEE6E33
:1026D000310EEE6E2C0EEE6E320EEE6E2C0EEE6E97
:1026E0007CC0EEFF7DC0EEFF7EC0EEFF7FC0EEFF40
:1026F00080C0EEFF81C0EEFF000EEE6E3D6A576AAD
:10270000586ADFEC61F0640EAE6FC80EAD6F3DB07D
:10271000B6EF13F03DB28FEF13F0AD67F8D73D92EF
:10272000DD0EF76E960EF66E20EED6F0F5EC61F04B
:10273000DD0EF76EB60EF66E20EEE6F0F5EC61F00B
:102740007CC0E0F07DC0E1F07EC0E2F07FC0E3F04D
:1027500080C0E4F081C0E5F013EC62F0640EAE6F6F
:10276000320EAD6FAD67FED755EF0AF064957AC0B3
:1027700065F07BC066F065C0BDF066C0BEF05ED49B
:10278000DD0EF76E760EF66E20EED6F0F5EC61F00B
:10279000DD0EF76E860EF66E20EEE6F0F5EC61F0DB
:1027A000200E9BC99AF09A631AD0DD0EF76EC60E02
:1027B000F66E20EED6F0F5EC61F0DD0EF76ED60E7B
:1027C000F66E20EEE6F0F5EC61F013EC62F0640ECC
:1027D000AE6F280EAD6FAD67FED755EF0AF003EE72
:1027E00000F0410EEE6E540EEE6E2B0EEE6E430EAA
:1027F000EE6E4F0EEE6E500EEE6E530EEE6E3D0E02
:10280000EE6E310EEE6E2C0EEE6E320EEE6E2C0E65
:10281000EE6E19EE9AF0060E976F200EE75C05E05B
:10282000E6CFEEFF972F0DEF14F0000EEE6E3D6A2F
:10283000576A586ADFEC61F0640EAE6FC80EAD6F78
:102840003DB04DEF14F03DB228EF14F0AD67F8D76E
:102850003D92DD0EF76E960EF66E20EED6F0F5EC9C
:1028600061F0DD0EF76EB60EF66E20EEE6F0F5ECDA
:1028700061F0060E976F19EE9AF000EEE0F0E6CFE9
:10288000EEFF972FFCD713EC62F0640EAE6F320EA2
:10289000AD6FAD67FED755EF0AF0DD0EF76E960E01
:1028A000F66E20EED6F0F5EC61F0DD0EF76EA60EBA
:1028B000F66E20EEE6F0F5EC61F0060E976F19EE7D
:1028C0009AF000EEE0F0E6CFEEFF972FFCD713EC86
:1028D00062F0640EAE6F320EAD6FAD67FED71EEFC5
:1028E00010F0CAEC58F05AEF10F0A66BA76B53EC3F
:1028F0005FF0A68753EC5FF0BFC081F0030E811735
:10290000816705D0020EC06FC16BBF8F0CD0010E66
:10291000816305D0030EC06FC16BBF8F04D0060E5C
:10292000C06FC16BBF8F81A293EF14F0FC0EBF0B81
:10293000AFEC5DF0A0EF0FF021EC5EF0A5EC5EF0E7
:10294000A66BA76B53EC5FF0A68753EC5FF0A789EB
:1029500053EC5FF0320EAB6FAB67FED7FFEC61F06C
:1029600009EC62F0DE0EF76E660EF66E20EED6F023
:10297000F5EC61F009EC62F013EC62F0010EC06F4F
:10298000C16BBF8F2EEC59F03494640EAB6FAB6704
:10299000FED7640EAE6FFA0EAD6F81B2D7EF14F0B2
:1029A000A0B10AD0AD67F9D7010EBF139ED7AFEC27
:1029B0005DF03482A0EF0FF0AFEC5DF001EED2F0ED
:1029C00010EEE6F09E6B34943496FCEC5DF09DC006
:1029D000EEFF9DC0E6FF13EC62F09E2B230E9D5D83
:1029E000D8B434842A0E9D5DD8B43486640EAE6F9C
:1029F00017C0ADF081B255EF15F0A0B104D0AD67AE
:102A0000F9D7A1EF15F0FCEC5DF09E2B230E9D6332
:102A100006D034B41FEF36F034B649D008D02A0EB1
:102A20009D6317EF15F034B67DD034B4B6D0020EE6
:102A30009E6307D034A405D02B0EE8CFD2F1E8CFA7
:102A4000E6F034943496110E9E612FEF15F09DC080
:102A5000EEFF9DC0E6FF13EC62F0F6EF14F0E7C066
:102A6000E6F0E8C0E7F0E9C0E8F0EAC0E9F0EBC062
:102A7000EAF0ECC0EBF0EDC0ECF0EEC0EDF0EFC032
:102A8000EEF0F0C0EFF0F1C0F0F0F2C0F1F0F3C002
:102A9000F2F0F4C0F3F0F5C0F4F09DC0EEFF9DC07D
:102AA000F5F013EC62F0F6EF14F0A0EF0FF0F50E76
:102AB000F76E040EF66E20EED6F0F5EC61F009EC40
:102AC00062F0100E976F08EE22F010EEE6F0EECFF7
:102AD000E6FF972FFCD713EC62F081B2A0EF0FF066
:102AE000A0B174EF15F0F9D7FCEC5DF0F50EF76EC0
:102AF000140EF66E20EED6F0F5EC61F0F50EF76EE2
:102B0000340EF66E20EEE6F0F5EC61F013EC62F0B8
:102B100081B2A0EF0FF0A0B18FEF15F0F9D7FCEC68
:102B20005DF0C5D7DF0EF76E560EF66E20EEE6F0BE
:102B3000F5EC61F013EC62F081A29CEF15F0A0EFD0
:102B40000FF06FEC31F0E866F7EF15F00CA804D049
:102B5000040EC06FC16BBF8F39B60AD0DF0EF76E9F
:102B6000760EF66E20EED6F0F5EC61F039940AD0D0
:102B7000DF0EF76E860EF66E20EED6F0F5EC61F005
:102B80003984398213EC62F03886E2EC31F0E86681
:102B900002D0F5EF1CF0A0EF0FF0DE0EF76ED60EB0
:102BA000F66E20EED6F0F5EC61F0DE0EF76EE60E76
:102BB000F66E20EEE6F0F5EC61F013EC62F0809A30
:102BC000358CA66BA76B53EC5FF0A68953EC5FF0D6
:102BD000A68353EC5FF081B2EFEF15F0FCD7A66B44
:102BE000A76B53EC5FF0808A359CA0EF0FF0DF0EEF
:102BF000F76E160EF66E20EED6F0F5EC61F009ECED
:102C000062F013EC62F0809A358CA66BA76B53ECE4
:102C10005FF0A68F53EC5FF0A68953EC5FF0A683BC
:102C200053EC5FF0320EAB6FAB67FED782AA67EF53
:102C300016F0358E640EAE6F080EAD6FAD67FED721
:102C40009E6B01EED2F011EE78F0200EE76430D0EA
:102C5000040E976FEF50E7622BD0EE50E650200E37
:102C6000E76201D002D0972FF5D797C09AF010EE07
:102C7000E6F0040E976F01EE78F00CAE04EC2FF046
:102C80000CBE45EC2FF0E86639D00F5009E0976F85
:102C9000640EAE6F0A0EAD6FAD67FED7972FF8D7F3
:102CA00001EED2F09A510508E926E86AEA2204D03A
:102CB00001EED2F010EEE6F0200E976F0CAE04ECB1
:102CC0002FF00CBE45EC2FF0E86618D02DD0808A8E
:102CD000359C359EEF0EF76E760EF66E20EED6F032
:102CE000F5EC61F0EF0EF76E860EF66E20EEE6F074
:102CF000F5EC61F013EC62F08FEF14F0808A359CF4
:102D0000F00EF76E060EF66E20EED6F0F5EC61F0E2
:102D1000F00EF76E160EF66E20EEE6F0F5EC61F0B2
:102D200013EC62F087EF14F0A66BA76B53EC5FF027
:102D3000A68953EC5FF0A68353EC5FF0A78953ECB0
:102D40005FF0A68753EC5FF0DF0EF76E260EF66E8F
:102D500020EED6F0F5EC61F013EC62F0A5EC5EF03D
:102D6000FCEC5DF0A06B579C349481B2C9EF16F077
:102D700038B4E2EF16F03DB6EEEF16F057BCD1EFE7
:102D800016F0A0A1F2D7FCEC5DF0230E9D63EDD709
:102D90004FD0FA0EAB6FAB67FED781B246EF18F09B
:102DA000E4D7579C010E7063E0D738943D96DF0E50
:102DB000F76E260EF66E20EED6F0F5EC61F013EC11
:102DC00062F0D3D73894ED0EF76E360EF66E20EE25
:102DD000D6F0F5EC61F013EC62F0C7D73D9625EC28
:102DE00018F0030E1E140208D8A4BFD72FEC35F03C
:102DF0003BA0BBD73D903D92640EAE6F140EAD6FFD
:102E00003D903D92D70EF76EBE0EF66E23EE00F0AB
:102E1000EEEC61F0DE6ADFEC61F03DB014EF17F02C
:102E20003DB216EF17F0F9D73D909FD73D929DD751
:102E30003484DF0EF76E360EF66E20EED6F0F5EC2B
:102E400061F009EC62F013EC62F02EEC59F001EE47
:102E5000D2F010EEE6F09E6B640EAE6F17C0ADF0D0
:102E600081B246EF18F038B4EFEF17F03DB6FBEF44
:102E700017F057BCDEEF17F0A0B142EF17F0AD67C7
:102E8000EFD742D0FCEC5DF0230E9D6309D034A453
:102E90003BD001EE50F0200EEF6253D0349442D07C
:102EA00034942A0E9D5D35E09E2B110E9E6107D055
:102EB0009DC0EEFF9DC0E6FF13EC62F0CDD7E7C0EA
:102EC000E6F0E8C0E7F0E9C0E8F0EAC0E9F0EBC0FE
:102ED000EAF0ECC0EBF0EDC0ECF0EEC0EDF0EFC0CE
:102EE000EEF0F0C0EFF0F1C0F0F0F2C0F1F0F3C09E
:102EF000F2F0F4C0F3F0F5C0F4F09DC0EEFF9DC019
:102F0000F5F013EC62F0A8D701EED2F0200EEF62DC
:102F100033D02EEC59F009EC62F0E9EC35F0FCEC22
:102F20005DF012D7DF0EF76E960EF66E20EED6F03D
:102F3000F5EC61F013EC62F004EC36F0FCEC5DF0C3
:102F400003D72EEC59F0100E8B6F9E6B11EED2F062
:102F500001EE50F0200EEF5C05E0EECFE6FF9E2B79
:102F60008B2FF8D7100E8B6F01EED2F010EEE6F03B
:102F7000EECFE6FF8B2FFCD7A66BA76B53EC5FF071
:102F8000A68F53EC5FF0A78B53EC5FF0040EC06F7D
:102F9000C16BBF8F24AC06D0A68D53EC5FF0A78326
:102FA00053EC5FF0DF0EF76E460EF66E20EED6F0B5
:102FB000F5EC61F013EC62F066EF1BF0579C010E2C
:102FC00070634AD738943D96DF0EF76E260EF66E84
:102FD00020EED6F0F5EC61F013EC62F03DD73894BA
:102FE000ED0EF76E360EF66E20EED6F0F5EC61F0D3
:102FF00013EC62F031D73D9625EC18F0030E1E1449
:103000000208D8A429D72FEC35F03BA025D73D9056
:103010003D92640EAE6F140EAD6F3D903D92D70E93
:10302000F76EBE0EF66E23EE00F0EEEC61F0DE6A97
:10303000DFEC61F03DB021EF18F03DB223EF18F066
:10304000ECD63D9009D73D9207D700EEDBF00B0E92
:10305000976F200EEE6E972F29EF18F001EE8CF08F
:1030600010EEDBF00A0E976FEECFE6FF972F34EFEE
:1030700018F013EC62F0100E976F01EE8CF011EE69
:103080009EF0EECFE6FF972FFCD7120021EC5EF00A
:10309000A06BA5EC5EF0808A359CA66BA76B53EC09
:1030A0005FF0ED0EF76EC60EF66E20EED6F0F5EC84
:1030B00061F0ED0EF76EA60EF66E20EEE6F0F5EC82
:1030C00061F0B4EC34F013EC62F0640EAE6F140EE9
:1030D000AD6FAD67FED7C00E3516A0EF0FF0808A3A
:1030E000359C3C0EAB6FAB67FED7809A358C280EB3
:1030F000AB6FAB67FED79F2FF2D71200640EAE6F97
:10310000140EAD6F35B403D0AD67FCD70FD0A66BEE
:10311000A76B53EC5FF0A78B53EC5FF0819688ECC4
:1031200030F08186A66BA76B53EC5FF0ED0EF76E67
:10313000260EF66E20EED6F0F5EC61F0ED0EF76E91
:10314000260EF66E20EEE6F0F5EC61F013EC62F080
:103150004CEC31F0640EAE6F1E0EAD6F36B202D085
:10316000AD67FCD70CC081F0030E81178167A3D037
:1031700037B006D001EE8CF0200EEE6EEE6E0AD067
:1031800010EEE6F001EE8CF0100E976FE6CFEEFF3A
:10319000972FFCD750EC30F0A66BA76B53EC5FF089
:1031A000A78953EC5FF0A68753EC5FF0140E6C6FA9
:1031B0001AC06DF03A903A923A863A94C56B80867E
:1031C00080948092808016A44ED016C081F0030EA9
:1031D0008117816718D0140E6C6F1AC06DF03A9089
:1031E0003A923A863A94C56B808680948092808029
:1031F0003AA4FED7640EAE6F060EAD6FAD67FED774
:10320000D6EC2FF030D0010E816312D0AFEC34F049
:1032100085EC2FF0140E6C6F1AC06DF03A903A9254
:103220003A863A94C56B80868094809280801BD0C9
:10323000020E8163D0D7140E6C6F1AC06DF03A90F5
:103240003A923A863A94C56B8086809480928080C8
:103250003AA4FED7640EAE6F060EAD6FAD67FED713
:10326000D6EC2FF000D081A245EF19F035A63AEF49
:1032700019F0F9D73A6A8086809480828090FA0E9D
:10328000AB6FAB67FED7A0EF0FF0AFEC5DF03A6A23
:103290008086809480828090A8EC34F0809A358C6F
:1032A0003596FA0EAB6FAB67FED709EC62F013EC04
:1032B00062F094EF16F0010E8163E8D0A66BA76B65
:1032C00053EC5FF0A68F53EC5FF0A78B53EC5FF0ED
:1032D000A68D53EC5FF0A78353EC5FF021EC5EF01A
:1032E000A5EC5EF0809A358C3596DF0EF76E160EE3
:1032F000F66E20EED6F0F5EC61F02EEC59F009EC0C
:1033000062F013EC62F0640EAE6F050EAD6FAD6748
:10331000FED7050EC06FC16BBF8F01EED2F010EE6D
:10332000E6F09E6B640EAE6F640EAD6FA0B103D07D
:10333000AD67FCD7A3D0AFEC5DF0FCEC5DF0230EE5
:103340009D6301D0DAD79DC0EEFF9DC0E6FF13EC70
:1033500062F09E2B11509E6149D0640EAE6F12C078
:10336000ADF0640EB06F1350AF6FA0B109D0105024
:103370009E6103D0AF67F9D781D0AD67F6D736D05D
:10338000FCEC5DF0230E9D6301D0B7D79E2B110E90
:103390009E6107D09DC0EEFF9DC0E6FF13EC62F07A
:1033A000D9D7E7C0E6F0E8C0E7F0E9C0E8F0EAC046
:1033B000E9F0EBC0EAF0ECC0EBF0EDC0ECF0EEC0F1
:1033C000EDF0EFC0EEF0F0C0EFF0F1C0F0F0F2C0C1
:1033D000F1F0F3C0F2F0F4C0F3F0F5C0F4F09DC0EA
:1033E000EEFF9DC0F5F013EC62F0B4D7A66BA76BAF
:1033F00053EC5FF0A68F53EC5FF0A78B53EC5FF0BC
:10340000040EC06FC16BBF8F24AC0DEF1AF0A68DF8
:1034100053EC5FF0A78353EC5FF00CA657D110502C
:103420009E6554D1100E976F01EED2F011EE8CF024
:10343000EECFE6FF972FFCD7E3EC34F03CB846D153
:10344000808A359CF40EF76E040EF66E20EED6F0F0
:10345000F5EC61F0F40EF76E140EF66E20EEE6F069
:10346000F5EC61F013EC62F0640EAE6F140EAD6F0C
:10347000AD67FED7C00E3516A0EF0FF0A66BA76B99
:1034800053EC5FF0808A359CA0EF0FF0020E816351
:103490006FD601EE50F0200EEF6213D0ED0EF76EF6
:1034A000860EF66E20EED6F0F5EC61F0ED0EF76EBE
:1034B000960EF66E20EEE6F0F5EC61F013EC62F09D
:1034C00057D60E503BE1A66BA76B53EC5FF0A68F6F
:1034D00053EC5FF0A78B53EC5FF024AC0CD0809AD8
:1034E000358CA68D53EC5FF0A78353EC5FF0040E90
:1034F000C06FC16BBF8FDF0EF76E460EF66E20EE0B
:10350000D6F0F5EC61F009EC62F02EEC59F0100EFB
:103510008B6F11EED2F001EE50F0EECFE6FF8B2F65
:10352000FCD7100E8B6F01EED2F010EEE6F0EECF6E
:10353000E6FF8B2FFCD713EC62F0C8D001EE50F001
:1035400037B006D001EE8CF0200EEE6EEE6E0AD093
:1035500010EEE6F001EE8CF0100E976FE6CFEEFF66
:10356000972FFCD750EC30F0A66BA76B53EC5FF0B5
:10357000A78953EC5FF0A68753EC5FF0140E6C6FD5
:103580001AC06DF03A903A923A863A94C56B8086AA
:1035900080948092808016A44DD016C081F0030ED6
:1035A0008117816718D0140E6C6F1AC06DF03A90B5
:1035B0003A923A863A94C56B808680948092808055
:1035C0003AA4FED7640EAE6F060EAD6FAD67FED7A0
:1035D000D6EC2FF02FD0010E816312D0AFEC34F077
:1035E00085EC2FF0140E6C6F1AC06DF03A903A9281
:1035F0003A863A94C56B80868094809280801AD0F7
:10360000020E8163E8D5140E6C6F1AC06DF03A900B
:103610003A923A863A94C56B8086809480928080F4
:103620003AA4FED7640EAE6F060EAD6FAD67FED73F
:1036300013EC30F0A66BA76B53EC5FF0A68F53EC46
:103640005FF0A78B53EC5FF024AC0CD0809A358CE4
:10365000A68D53EC5FF0A78353EC5FF0040EC06FB0
:10366000C16BBF8F81A245EF19F024BC03D035A6F2
:103670005BEF1BF00E50C563F5D73A6A80868094E5
:10368000808280902EEC59F0100E8B6F11EED2F0EC
:1036900001EE50F0EECFE6FF8B2FFCD7100E8B6FB4
:1036A00001EED2F010EEE6F0EECFE6FF8B2FFCD766
:1036B00013EC62F00BD03A6A80868094808280900E
:1036C000FA0EAB6FAB67FED7A0EF0FF00CA406D0DD
:1036D0006FEC31F0E8661FD039B60BD0DF0EF76E15
:1036E000760EF66E20EED6F0F5EC61F03996399450
:1036F0000AD0DF0EF76E860EF66E20EED6F0F5ECF1
:1037000061F03984398213EC62F03886E2EC31F0F2
:10371000E86601D02AD0F40EF76E240EF66E20EE85
:10372000D6F0F5EC61F0F40EF76E340EF66E20EE86
:10373000E6F0F5EC61F013EC62F0809A358CA68F20
:1037400053EC5FF0A78B53EC5FF0030EC06FC16BBF
:10375000BF8F640EAE6F140EAD6FAD67FED7808A5B
:10376000359CC00E3516A0EF0FF048EC2AF0DE0EA7
:10377000F76EA60EF66E20EED6F0F5EC61F0310E87
:1037800039B4320EE56F13EC62F0B2EC5EF021EC6E
:103790005EF00CEC58F01E0EBA6FA0B118EC58F0A9
:1037A000A0B5E5D0A0AB03D0AF51D8B4E0D057B0AE
:1037B000FDEF1BF057B4FFEF1BF057BA01EF1CF001
:1037C00057BC03EF1CF058B008EF1CF058B20AEFDA
:1037D0001CF03DB20FEF1CF03DB02DEF1CF03EB0E1
:1037E00011EF1CF03EB21FEF1CF035BC03D035A624
:1037F000B7EF1CF0BA67D1D7A7D05790A5D0579490
:10380000CCD7579ACAD7579C010E7063C6D79CD0A5
:1038100058909AD0589224BCAFEC5DF0BED73D9240
:1038200093D03E90F30EF76E160EF66E20EED6F0A5
:10383000F5EC61F0E8EC1CF013EC62F0AAD03E92DB
:10384000F30EF76E260EF66E20EED6F0F5EC61F074
:10385000E8EC1CF013EC62F09CD03D90AFEC5DF016
:10386000809A358CA66BA76B53EC5FF0A78B53EC5B
:103870005FF0A68D53EC5FF0A78353EC5FF0DE0E94
:10388000F76EB60EF66E20EED6F0F5EC61F0310E66
:1038900039B4320EE56F13EC62F021EC5EF0A0B1AA
:1038A00018EC58F0A0B563D0A0AB03D0AF51D8B49A
:1038B0005ED057B072EF1CF057BC74EF1CF058B0DC
:1038C00079EF1CF03DB07BEF1CF03DB27DEF1CF0BA
:1038D0003EB07FEF1CF03EB28DEF1CF03DB49BEF8D
:1038E0001CF0DDD7579030D0579C010E7063D7D7AE
:1038F0002BD0589029D03D90D2D73D9225D03E90E4
:10390000F30EF76E160EF66E20EED6F0F5EC61F0C3
:10391000E8EC1CF013EC62F03CD03E92F30EF76E34
:10392000260EF66E20EED6F0F5EC61F0E8EC1CF019
:1039300013EC62F02ED03D94030E1E140208D8A49E
:10394000AED72FEC35F0ABD7ED0EF76EC60EF66E98
:1039500020EED6F0F5EC61F0ED0EF76ED60EF66EB9
:1039600020EEE6F0F5EC61F013EC62F012D0ED0E13
:10397000F76EC60EF66E20EED6F0F5EC61F0ED0EA9
:10398000F76EB60EF66E20EEE6F0F5EC61F013EC95
:1039900062F0AFEC5DF0A66BA76B53EC5FF0808A32
:1039A000359C3D903D92D70EF76EBE0EF66E23EE1F
:1039B00000F0EEEC61F0DE6ADFEC61F0640EAE6FF9
:1039C000140EAD6FAD67FED7C00E3516A0EF0FF029
:1039D00009EC62F0100E976F11EED2F000EEE6F0F7
:1039E000E6CFEEFF972FFCD71200A66BA76B53EC28
:1039F0005FF0A78153EC5FF0A68753EC5FF024AC37
:103A000003D0A68553EC5FF003EE00F0410EEE6E9E
:103A1000540EEE6E440EEE6E9EC097F011EED2F094
:103A2000E6CFEEFF972F10EF1DF03B0EEE6E000E6F
:103A3000EE6E3D6A3E6A576A586ADFEC61F0DE0E50
:103A4000F76EA60EF66E20EED6F0F5EC61F0310EB4
:103A500039B4320EE8CFE5F013EC62F03C0EBA6FE9
:103A600057B050EF1DF057BC56EF1DF058B05FEF48
:103A70001DF058B26FEF1DF03DB274EF1DF03DB078
:103A80009AEF1DF03EB07AEF1DF03EB28AEF1DF0C6
:103A900081B2D2EF1EF0BA67E3D7AFEC5DF06FD121
:103AA0005790AFEC5DF0020EBF1369D1579C010E29
:103AB0007063D6D7AFEC5DF0010EBF1360D15890A4
:103AC000AFEC5DF0020EBF13DC0EF76EB60EF66EB5
:103AD00020EEE6F0F5EC61F013EC62F075D158924F
:103AE00024BCAFEC5DF0BCD73D92AFEC5DF0020EB4
:103AF000BF1345D13E90AFEC5DF0F30EF76E360E7E
:103B0000F66E20EED6F0F5EC61F013EC62F0000EEC
:103B1000BF1335D13E92AFEC5DF0F30EF76E460E5B
:103B2000F66E20EED6F0F5EC61F013EC62F0000ECC
:103B3000BF1325D13D90AFEC5DF0A66BA76B53ECA6
:103B40005FF0A78153EC5FF0A68553EC5FF0A68F82
:103B500053EC5FF0A78953EC5FF0A8EC34F021EC54
:103B60005EF0A5EC5EF09A6B640EAB6FAB67FED7B0
:103B7000DE0EF76EB60EF66E20EED6F0F5EC61F0C6
:103B8000310E39B4320EE8CFE5F013EC62F081B2B9
:103B9000D2EF1EF035B6B2D057B0EAEF1DF057BCE9
:103BA000EEEF1DF058B047EF1EF03DB255EF1EF09E
:103BB0003EB059EF1EF03EB267EF1EF03DB475EF18
:103BC0001EF03DB0E8EF1DF0A0B10EEC1FF0DFD706
:103BD0003D90DDD75790020EBF13D1D0579C010EF8
:103BE000706329D03D903D92DB0EF76E420EF66E6B
:103BF00023EE00F0EEEC61F0DE6ADFEC61F09A6B30
:103C00002EEC1FF0C80EAB6F3DB00DEF1EF03DB2B5
:103C100055EF1EF0AB67F8D7BAD73D903D92DB0E5B
:103C2000F76E360EF66E23EE00F0EEEC61F0DE6A13
:103C3000DFEC61F0ACD7020E7063A9D73D903D92E6
:103C4000DB0EF76E4E0EF66E23EE00F0EEEC61F03A
:103C5000DE6ADFEC61F09A6B23EC1FF0C80EAB6FED
:103C60003DB039EF1EF03DB255EF1EF0AB67F8D70F
:103C70008ED73D903D92DB0EF76E360EF66E23EE3C
:103C800000F0EEEC61F0DE6ADFEC61F080D7589076
:103C9000020EBF13DC0EF76EB60EF66E20EEE6F0E7
:103CA000F5EC61F013EC62F08FD03D92020EBF1381
:103CB00066D03E90F30EF76E360EF66E20EED6F01E
:103CC000F5EC61F013EC62F0000EBF1358D03E9299
:103CD000F30EF76E460EF66E20EED6F0F5EC61F0C0
:103CE00013EC62F0000EBF134AD03D94030E1E1475
:103CF0000208D8A44CD72FEC35F049D7809A358CE0
:103D0000ED0EF76E060EF66E20EED6F0F5EC61F0D5
:103D1000ED0EF76E160EF66E20EEE6F0F5EC61F0A5
:103D200013EC62F0640EAE6F280EAD6F020EC06F22
:103D3000C16BBF8FAD67FED7AFEC5DF0808A359C5D
:103D4000C00E3516DE0EF76EB60EF66E20EED6F00D
:103D5000F5EC61F0310E39B4320EE8CFE5F09EC0DB
:103D600097F009EC62F011EED2F000EEE6F0E6CF4B
:103D7000EEFF972FB7EF1EF013EC62F008D7ED0EB1
:103D8000F76EC60EF66E20EED6F0F5EC61F0ED0E95
:103D9000F76ED60EF66E20EEE6F0F5EC61F013EC61
:103DA00062F012D0ED0EF76EC60EF66E20EED6F073
:103DB000F5EC61F0ED0EF76EA60EF66E20EEE6F075
:103DC000F5EC61F013EC62F0B4EC34F03D903D9210
:103DD000D70EF76EBE0EF66E23EE00F0EEEC61F03D
:103DE000DE6ADFEC61F0640EAE6F140EAD6FAD678E
:103DF000FED73D903D923E6A579A579C8B6B75EF6C
:103E000014F009EC62F0100E976F11EE9EF000EEC8
:103E1000E6F0E6CFEEFF972FFCD71200FCEC5DF04A
:103E20002A0E9D6326D03D903D92DB0EF76E360E36
:103E3000F66E23EE00F0EEEC61F0DE6ADFEC61F08E
:103E40009A2B9AB10BD0310EDB6F4C0EDC6F2D0E1E
:103E5000DD6FE8EC1CF013EC62F028D0320EDB6F63
:103E60004C0EDC6F2D0EDD6F01EC1FF013EC62F0D9
:103E70001DD0230E9D631AD03D903D92DB0EF76E50
:103E80002A0EF66E23EE00F0EEEC61F0DE6ADFEC57
:103E900061F0200EDB6FDC6FDD6F9AB1E8EC1CF097
:103EA0009AA101EC1FF013EC62F09A6B1200DE0E87
:103EB000F76E760EF66E20EED6F0F5EC61F0DE0EC3
:103EC000F76EF60EF66E20EEE6F0F5EC61F013EC10
:103ED00062F0C56B3B923D963E6A5790579C589056
:103EE000640EAE6FFA0EAD6F57B08CEF1FF057BC7B
:103EF0008EEF1FF058B093EF1FF03EB095EF1FF01C
:103F00003EB295EF1FF03DB6B4EF1FF038B4CBEFE3
:103F10001FF0AD67E9D70AD0579008D0579C010E23
:103F20007063E2D703D0589001D03E6A3D903D9235
:103F30003D903D92D70EF76EBE0EF66E23EE00F06A
:103F4000EEEC61F0DE6ADFEC61F0640EAE6F140E31
:103F5000AD6F3DB0B1EF1FF03DB2B1EF1FF0AD67F7
:103F6000F8D73894A0EF0FF03D963BB2BDD73B8217
:103F700009EC62F001EE8CF0200EEF5CB5E010EE83
:103F8000E6F0100E976FEECFE6FF972FC3EF1FF00E
:103F900013EC62F0A9D73894C52B010EC565A4D7E0
:103FA0001EC081F0030E81178167E1EF21F034D04C
:103FB000EE0EF76E460EF66E20EED6F0F5EC61F0E2
:103FC000EE0EF76E560EF66E20EEE6F0F5EC61F0B2
:103FD00013EC62F03B903B923D903D92D70EF76E12
:103FE000BE0EF66E23EE00F0EEEC61F0DE6ADFEC62
:103FF00061F0640EAE6F140EAD6F3DB005EF20F0B2
:104000003DB205EF20F0AD67F8D7AD67FED73D9024
:104010003D923D96FFEF0FF01EA40CD0E3EC34F080
:104020003CB208D0500EEA6303D01EBE03D0C0D706
:1040300016A6BED73D903D923E6A5790579C589029
:1040400050EC30F0A66BA76B53EC5FF0A78953ECF4
:104050005FF0A68753EC5FF016B40ED0140E6C6FB1
:104060001AC06DF03A903A923A863A94C56B8086BF
:1040700080948092808034D016C081F0030E811726
:10408000816718D0140E6C6F1AC06DF03A903A9296
:104090003A863A94C56B80868094809280803AA458
:1040A000FED7640EAE6F060EAD6FAD67FED7D6ECD1
:1040B0002FF016D0010E816312D0AFEC34F085ECF6
:1040C0002FF0140E6C6F1AC06DF03A903A923A8647
:1040D0003A94C56B808680948092808001D0D2D73C
:1040E00081B27AEF20F0640EAB6FAB67FED781A28E
:1040F00094EF20F057B084EF20F057BC88EF20F009
:1041000058B086EF20F0ECD7579006D0589004D0E6
:10411000579C010E7063E4D738943A6A8086809485
:1041200080828090A0EF0FF03A6A8086809480822F
:104130008090A8EC34F0FA0EAB6FAB67FED7DE0EC2
:10414000F76EB60EF66E20EED6F0F5EC61F013ECDD
:1041500062F0A66BA76B53EC5FF0A78153EC5FF0A6
:10416000A68553EC5FF0A68F53EC5FF0A78953EC64
:104170005FF021EC5EF0A5EC5EF09A6B38BE0DD0DE
:104180003D903D92D70EF76EC40EF66E23EE00F012
:10419000EEEC61F0DE6ADFEC61F081B2EDEF20F071
:1041A0003DB03D9057BC36EF21F035B6F5EF20F02D
:1041B0003DB4E4EF20F03DB2E2EF20F0A0B10EEC10
:1041C0001FF0EBD73D92ABD03D94030E1E140208B6
:1041D000D8A4E3D72FEC35F0E0D7FA0EAB6FAB677E
:1041E000FED781B2A5EF21F0D8D7809A358CED0E9D
:1041F000F76E060EF66E20EED6F0F5EC61F0ED0EE1
:10420000F76E160EF66E20EEE6F0F5EC61F013ECAC
:1042100062F0640EAE6F280EAD6F020EC06FC16B00
:10422000BF8FAD67FED7AFEC5DF0808A359CC00EC6
:104230003516DE0EF76EB60EF66E20EED6F0F5EC05
:1042400061F0310E39B4320EE8CFE5F009EC62F0DE
:1042500001EE8CF010EEE6F0100E976FEECFE6FF59
:10426000972F2EEF21F013EC62F097D7579C010E99
:10427000706329D03D903D92DB0EF76E420EF66ED4
:1042800023EE00F0EEEC61F0DE6ADFEC61F09A6B99
:104290002EEC1FF0C80EAB6F3DB055EF21F03DB2D4
:1042A000E2EF20F0AB67F8D778D73D903D92DB0E78
:1042B000F76E360EF66E23EE00F0EEEC61F0DE6A7D
:1042C000DFEC61F06AD7020E706367D73D903D92D4
:1042D000DB0EF76E4E0EF66E23EE00F0EEEC61F0A4
:1042E000DE6ADFEC61F09A6B23EC1FF0C80EAB6F57
:1042F0003DB081EF21F03DB2E2EF20F0AB67F8D79F
:104300004CD73D903D92DB0EF76E360EF66E23EEE7
:1043100000F0EEEC61F0DE6ADFEC61F03ED738943D
:10432000ED0EF76EC60EF66E20EED6F0F5EC61F0EF
:10433000ED0EF76ED60EF66E20EEE6F0F5EC61F0BF
:1043400013EC62F0010EBF1312D0ED0EF76EC60E25
:10435000F66E20EED6F0F5EC61F0ED0EF76EA60EDF
:10436000F66E20EEE6F0F5EC61F013EC62F0B4ECE2
:1043700034F0320EAB6FAB67FED73D903D923D906F
:104380003D92D70EF76EBE0EF66E23EE00F0EEEC09
:1043900061F0DE6ADFEC61F0640EAE6F140EAD6F9B
:1043A0003DB0D8EF21F03DB2D8EF21F0AD67F8D79E
:1043B000640EAE6F140EAD6FAD67FED7389475EF17
:1043C00014F0010E8163DAD11EA417D0E3EC34F0AF
:1043D0003BA003D03CB00BD0EBD5500EEA6303D02A
:1043E0001EBE05D0E5D516A6E3D51AEF20F001EEE6
:1043F00060F0200EEF6201D0BCD0100E976F01EE7E
:1044000060F011EED2F0EECFE6FF972FFCD7A66B4F
:10441000A76B53EC5FF0A68F53EC5FF0A78B53ECC8
:104420005FF0809A358C320EAB6FAB67FED782AAF5
:1044300003EF23F0358E640EAE6F0A0EAD6FAD67DD
:10444000FED721EC5EF038BE0ED03D903D92D70EE7
:10445000F76EC40EF66E23EE00F0EEEC61F0DE6A4D
:10446000DFEC61F0388EED0EF76EF60EF66E20EE94
:10447000D6F0F5EC61F013EC62F009EC62F0640E3A
:10448000AE6F050EAD6F3DB03D90AD67FCD7389473
:1044900001EED2F010EEE6F0100E976F0CAE04ECC9
:1044A0002FF00CBE45EC2FF0E8664AD03DB03D90B1
:1044B00057B075EF22F057BC77EF22F058B07CEF81
:1044C00022F03DB27EEF22F0A66BA76B53EC5FF0BB
:1044D000A68753EC5FF0A78D53EC5FF0A68D53ECED
:1044E0005FF0A78353EC5FF0B8D0579009D0579C8A
:1044F000010E7063B2D004D0589002D03D9200D02B
:10450000ED0EF76EC60EF66E20EED6F0F5EC61F00D
:10451000ED0EF76ED60EF66E20EEE6F0F5EC61F0DD
:1045200013EC62F0A66BA76B53EC5FF0808A359CAE
:10453000640EAE6F140EAD6FAD67FED7A0EF0FF037
:10454000F00EF76E060EF66E20EED6F0F5EC61F08A
:10455000F00EF76E160EF66E20EEE6F0F5EC61F05A
:1045600013EC62F0808A359CA66BA76B53EC5FF06E
:104570005FD0A66BA76B53EC5FF0A68753EC5FF0A0
:10458000A78D53EC5FF0A68D53EC5FF0A78353EC3F
:104590005FF0809A358C640EAB6FAB67FED782AA52
:1045A00003EF23F0358E3D903D92D90EF76EFA0E53
:1045B000F66E23EE00F0EEEC61F0DE6ADFEC61F007
:1045C000640EAE6F0A0EAD6F3DB03D90AD67FCD787
:1045D0003C9E349438BE41D0388E3D903D92D70EEB
:1045E000F76EC40EF66E23EE00F0EEEC61F0DE6ABC
:1045F000DFEC61F0640EAE6F0A0EAD6F3DB03D9022
:10460000AD67FCD72AD0808A359C359EED0EF76EBB
:10461000460EF66E20EED6F0F5EC61F0ED0EF76E7C
:10462000560EF66E20EEE6F0F5EC61F013EC62F05B
:104630003D903D92D70EF76EBE0EF66E23EE00F063
:10464000EEEC61F0DE6ADFEC61F0640EAE6F140E2A
:10465000AD6FAD67FED7A0EF0FF021EC5EF0A5ECDB
:104660005EF0A06B020EC06FC16BBF8FDE0EF76EE7
:10467000B60EF66E20EED6F0F5EC61F009EC62F0C5
:1046800001EE8CF0200EEF5C09E010EEE6F0100E6B
:10469000976FEECFE6FF972F49EF23F013EC62F010
:1046A000A0B10CD03DB03D9057B06AEF23F057BC9D
:1046B0006EEF23F058B06CEF23F0F2D73CAE3BEC3A
:1046C0003CF03C8EFCEC5DF0230E9D63E9D71EAC04
:1046D000E7D735D0579006D0589004D0579C010E9C
:1046E0007063DED7ED0EF76EC60EF66E20EED6F0D6
:1046F000F5EC61F0ED0EF76ED60EF66E20EEE6F0FC
:10470000F5EC61F013EC62F0A66BA76B53EC5FF075
:10471000808A359C3D903D92D70EF76EBE0EF66EA8
:1047200023EE00F0EEEC61F0DE6ADFEC61F0640E87
:10473000AE6F140EAD6FAD67FED7A0EF0FF0EE0EAB
:10474000F76E060EF66E20EED6F0F5EC61F0EE0E8A
:10475000F76E160EF66E20EEE6F0F5EC61F013EC57
:1047600062F0A66BA76B53EC5FF0808A359C640EF9
:10477000AE6F140EAD6FAD67FED739D6020E8163F2
:1047800026EF24F0100E976F11EE8CF001EE9EF0E4
:10479000E6CFEEFF972FFCD72FEC35F03BA048D4A7
:1047A0003CA420D03B903B923D903D92D70EF76EBB
:1047B000BE0EF66E23EE00F0EEEC61F0DE6ADFEC8A
:1047C00061F03DB0E8EF23F03DB2E8EF23F0F9D718
:1047D0003D903D923D963B86640EB96F320EB86FA8
:1047E000FFEF0FF0EE0EF76E460EF66E20EED6F0EF
:1047F000F5EC61F0EE0EF76E560EF66E20EEE6F07A
:10480000F5EC61F013EC62F03B903B923D903D92F1
:10481000D70EF76EBE0EF66E23EE00F0EEEC61F0F2
:10482000DE6ADFEC61F0640EAE6F140EAD6F3DB06A
:104830001FEF24F03DB21FEF24F0AD67F8D7AD674E
:10484000FED73D903D923D96FFEF0FF01EC081F0E8
:10485000030E8117030E8163A0EF0FF0100E976F08
:1048600011EE8CF001EE9EF0E6CFEEFF972FFCD715
:104870007DEC35F03CA6B6D73B903B923D903D9207
:10488000D70EF76EBE0EF66E23EE00F0EEEC61F082
:10489000DE6ADFEC61F03DB052EF24F03DB252EF42
:1048A00024F0F9D73D903D923D963B86640EB96F5A
:1048B000320EB86FFFEF0FF06FEC31F0E86602D008
:1048C00039B60AD0DF0EF76E760EF66E20EED6F011
:1048D000F5EC61F039960AD0DF0EF76E860EF66EB3
:1048E00020EED6F0F5EC61F039823984DE0EF76EF9
:1048F000860EF66E20EED6F0F5EC61F013EC62F069
:104900003886E2EC31F0E866A0EF0FF048EC2AF0D0
:10491000DE0EF76EA60EF66E20EED6F0F5EC61F028
:10492000310E39B4320EE56F13EC62F0640EAE6FE7
:10493000FA0EAD6F3DB0D0EF24F057B0AFEF24F0DA
:1049400057BCB1EF24F058B0B6EF24F03EB0B8EF4A
:1049500024F03EB2C4EF24F0AD67ECD7B2D257904A
:10496000B0D2579C010E7063E5D7ABD25890A9D254
:104970003E90F30EF76EC40EF66E20EED6F0F5EC18
:1049800061F013EC62F09DD23E92F30EF76EB40E1E
:10499000F66E20EED6F0F5EC61F013EC62F091D2F9
:1049A00021EC5EF0A5EC5EF0A06BA66BA76B53EC60
:1049B0005FF0A78753EC5FF0A78D53EC5FF0DE0E3E
:1049C000F76EC60EF66E20EED6F0F5EC61F009EC4F
:1049D00062F02EEC59F013EC62F0050EC06FC16B63
:1049E000BF8F9E6BA0B11CD03DB03D9057B007EF7C
:1049F00025F057BC09EF25F058B00EEF25F03DB477
:104A000003EF25F0EFD73D947DEC35F0EBD75790D1
:104A100058D2579C010E7063E5D753D2A0EF0FF028
:104A2000AFEC5DF0FCEC5DF0230E9D5DD0E000EEA0
:104A3000E6F011EED2F09DC0EEFF9DC0E6FF13EC54
:104A400062F09E2B640EAE6F17C0ADF0A0B111D016
:104A50003DB03D9057B073EF25F057BC75EF25F092
:104A600058B07AEF25F03DB46FEF25F0AD67EED783
:104A700043D0FCEC5DF0230E9D6301D0A8D79E2BA4
:104A8000110E9E6107D09DC0EEFF9DC0E6FF13ECA6
:104A900062F0D8D7E7C0E6F0E8C0E7F0E9C0E8F098
:104AA000EAC0E9F0EBC0EAF0ECC0EBF0EDC0ECF0EE
:104AB000EEC0EDF0EFC0EEF0F0C0EFF0F1C0F0F0BE
:104AC000F2C0F1F0F3C0F2F0F4C0F3F0F5C0F4F08E
:104AD0009DC0EEFF9DC0F5F013EC62F0B3D73D949E
:104AE0007DEC35F0B3D75790ECD1579C010E706335
:104AF000ADD7E7D1A0EF0FF06FEC31F0E86601D051
:104B0000CBD0809A358C640EAB6FAB67FED782AA90
:104B100003EF23F0358EA66BA76B53EC5FF0A68FE7
:104B200053EC5FF0A78D53EC5FF0A68D53EC5FF074
:104B3000A78353EC5FF0640EAE6F080EAD6FAD67E8
:104B4000FED79E6B01EED2F011EE78F0200EE764F6
:104B500030D0040E976FEF50E7622BD0EE50E65046
:104B6000200EE76201D002D0972FF5D797C09AF0B8
:104B700010EEE6F0040E976F01EE78F00CAE04EC48
:104B80002FF00CBE45EC2FF0E8665DD00F5009E029
:104B9000976F640EAE6F0A0EAD6FAD67FED7972F9D
:104BA000F8D701EED2F09A510508E926E86AEA2220
:104BB00004D001EED2F010EEE6F0200E976F0CAEAE
:104BC00004EC2FF00CBE45EC2FF0E8663CD0A66B51
:104BD000A76B53EC5FF0A68753EC5FF0A78D53EC07
:104BE0005FF0A68D53EC5FF0A78353EC5FF02DEFE1
:104BF00023F0808A359C359EEF0EF76E760EF66EAA
:104C000020EED6F0F5EC61F0EF0EF76E860EF66E44
:104C100020EEE6F0F5EC61F013EC62F03D903D9291
:104C2000D70EF76EBE0EF66E23EE00F0EEEC61F0DE
:104C3000DE6ADFEC61F0640EAE6F140EAD6FAD672F
:104C4000FED7A0EF0FF0808A359CF00EF76E060EAF
:104C5000F66E20EED6F0F5EC61F0F00EF76E160E63
:104C6000F66E20EEE6F0F5EC61F013EC62F03D90AC
:104C70003D92D70EF76EBE0EF66E23EE00F0EEEC10
:104C800061F0DE6ADFEC61F0640EAE6F140EAD6FA2
:104C9000AD67FED7A0EF0FF0F30EF76E740EF66E51
:104CA00020EED6F0F5EC61F009EC62F09EC097F0D2
:104CB00001EED2F010EEE6F0EECFE6FF972FFCD734
:104CC00013EC62F03D903D92DB0EF76E360EF66E01
:104CD00023EE00F0EEEC61F0DE6ADFEC61F0640ED2
:104CE000AE6F320EAD6F3DB083EF26F03DB286EF72
:104CF00027F057BC7FEF26F0AD67F5D7E2D0579C81
:104D0000010E7063F0D703EE00F0410EEE6E540E0C
:104D1000EE6E440EEE6E9EC097F011EED2F0E6CF2E
:104D2000EEFF972F8FEF26F03B0EEE6E000EEE6E2D
:104D30003D6A3E6A576A586ADFEC61F0F30EF76E1F
:104D4000A40EF66E20EED6F0F5EC61F013EC62F0F6
:104D50003C0EBA6F57B0C8EF26F057BCCAEF26F02A
:104D600058B0CFEF26F058B2D1EF26F03DB2D3EFD6
:104D700026F03DB0F5EF26F03EB0D5EF26F03EB27E
:104D8000E1EF26F03DB4EDEF26F0BA67E3D799D016
:104D9000579097D0579C010E7063DCD792D05890F3
:104DA00090D05892D7D73D928CD03E90F30EF76EAC
:104DB000C40EF66E20EED6F0F5EC61F013EC62F066
:104DC00080D03E92F30EF76EB40EF66E20EED6F063
:104DD000F5EC61F013EC62F074D03D94030E1E14F8
:104DE0000208D8B47DEC35F0B5D73D903D903D92AA
:104DF000DB0EF76E5A0EF66E23EE00F0EEEC61F06D
:104E0000DE6ADFEC61F0F30EF76ED40EF66E20EE84
:104E1000D6F0F5EC61F0A5EC5EF0FCEC5DF0A06B7B
:104E200013EC62F0A0B113D057B02DEF27F057BCB0
:104E300039EF27F058B02FEF27F03DB031EF27F0D2
:104E40003DB233EF27F03DB435EF27F0EBD7FCEC64
:104E50005DF0230E9D63E6D715D0579032D0589061
:104E600030D03D90DFD73D9251D03D947DEC35F070
:104E7000D9D7579C010E706301D023D0579C020EE6
:104E80007063D0D71EAC1DD03D903D92DB0EF76E07
:104E90004E0EF66E23EE00F0EEEC61F0DE6ADFEC13
:104EA00061F0640EAE6F320EAD6F3DB05EEF27F075
:104EB0003DB286EF27F0AD67F8D703D0388ED0EF3C
:104EC00024F0F30EF76E840EF66E20EED6F0F5ECBD
:104ED00061F0F30EF76E940EF66E20EEE6F0F5EC50
:104EE00061F03D903D92D70EF76EBE0EF66E23EE4A
:104EF00000F0EEEC61F0DE6ADFEC61F0640EAE6FA4
:104F0000140EAD6FAD67FED7A0EF0FF0F30EF76E86
:104F1000E40EF66E20EED6F0F5EC61F0F30EF76ECF
:104F2000F40EF66E20EEE6F0F5EC61F013EC62F0B4
:104F30003D903D92D70EF76EBE0EF66E23EE00F05A
:104F4000EEEC61F0DE6ADFEC61F0640EAE6F140E21
:104F5000AD6FAD67FED7A0EF0FF0B8675AEF10F056
:104F6000400E976F14EEC0F0E76606D0E650972F1C
:104F7000FBD73B965AEF10F03B94E7B23B84E76ACD
:104F800097514008A26F9E6B15EE08F00A0EA2031F
:104F9000F350E126F450E222E7CF3CF02EEC59F03A
:104FA00001EED2F015EE00F00A0EA203F350E12656
:104FB000F450E222080ECB6F200E806FE7380F0B03
:104FC000300F816F3F0E816180C081F0080ECB638E
:104FD00005D03B0E816302D02B0E816F81C0EEFFA6
:104FE000200E815D12E09E2BE6500F0B9A6F300F62
:104FF000816F3F0E816180C081F081C0EEFF200E85
:10500000815F03E09E2BCB2FD9D71EC081F0030E0A
:105010008117020E81635CEF24F03BB402D01EB610
:10502000BAD06FEC31F0E86602D039B60AD0DF0EA4
:10503000F76E760EF66E20EED6F0F5EC61F039964E
:105040000AD0DF0EF76E860EF66E20EED6F0F5EC87
:1050500061F039823984DE0EF76E860EF66E20EE30
:10506000D6F0F5EC61F013EC62F03886E2EC31F04A
:10507000E866A0EF0FF048EC2AF0DE0EF76EA60E01
:10508000F66E20EED6F0F5EC61F0310E39B4320E4A
:10509000E56F13EC62F0640EAE6FFA0EAD6F3DB0CB
:1050A00088EF28F057B064EF28F057BC66EF28F07F
:1050B00058B06BEF28F03EB06DEF28F03EB27AEFBB
:1050C00028F0AD67ECD722D0579020D0579C010E26
:1050D0007063E5D71BD0589019D03E90F30EF76E51
:1050E000560EF66E20EED6F0F5EC61F013EC62F0A1
:1050F00086EF28F03E92F30EF76E660EF66E20EE07
:10510000D6F0F5EC61F013EC62F000D072EF23F012
:10511000388E3BA4F7EF21F01DEE00F0080EA2033D
:10512000F350E126F450E2222EEC59F09E6B01EE92
:10513000D2F0080ECB6F200E806FE7380F0B300FC8
:10514000816F3F0E816180C081F081C0EEFF200E33
:10515000816512D09E2BE6500F0B9A6F300F816F36
:105160003F0E816180C081F081C0EEFF200E81651D
:1051700003D09E2BCB2FE1D71DEE00F0080EA2032B
:10518000F350E126F450E222080E976FE668972F5D
:10519000FDD707EF22F0DF0EF76E160EF66E20EE4B
:1051A000D6F0F5EC61F009EC62F013EC62F0809A55
:1051B000358CA66BA76B53EC5FF0A68F53EC5FF0BA
:1051C000A68953EC5FF0A68353EC5FF0320EAB6F11
:1051D000AB67FED782AA2BEF2AF0358E640EAE6F36
:1051E000080EAD6FAD67FED79E6B01EED2F02B0EB1
:1051F000EF6202D001EED3F011EE70F0200EE76402
:1052000035D0080E976FEF50E76230D0EE50E65081
:10521000200EE76201D002D0972FF5D797C09AF001
:1052200010EEE6F0040E976F01EE78F00CAE04EC91
:105230002FF00CBE45EC2FF0E866F1D00F5009E0DE
:10524000976F640EAE6F0A0EAD6FAD67FED7972FE6
:10525000F8D701EED2F02B0EEF6202D001EED3F0C0
:105260009A510908E926E86AEA224AD001EED2F00A
:105270002B0EEF6202D001EED3F011EE78F0200E8B
:10528000E76435D0040E976FEF50E76230D0EE50F0
:10529000E650200EE76201D002D0972FF5D797C0D5
:1052A0009AF010EEE6F0040E976F01EE78F00CAE77
:1052B00004EC2FF00CBE45EC2FF0E866B0D00F5098
:1052C00009E0976F640EAE6F0A0EAD6FAD67FED743
:1052D000972FF8D701EED2F02B0EEF6202D001EE3D
:1052E000D3F09A510508E926E86AEA2209D001EECE
:1052F000D2F02B0EEF6202D001EED3F010EEE6F00A
:10530000200E976F0CAE04EC2FF00CBE45EC2FF086
:10531000E86685D0A66BA76B53EC5FF0A78953ECCA
:105320005FF0A68753EC5FF050EC30F016B40ED06F
:10533000140E6C6F1AC06DF03A903A923A863A9415
:10534000C56B80868094809280802BD016A012D06E
:10535000AFEC34F085EC2FF0140E6C6F1AC06DF0CA
:105360003A903A923A863A94C56B808680948092BD
:10537000808017D0140E6C6F1AC06DF03A903A927C
:105380003A863A94C56B80868094809280803AA455
:10539000FED7640EAE6F060EAD6FAD67FED7D6ECCE
:1053A0002FF0640EB06FFA0EAF6F81B2DFEF29F00D
:1053B000640EAB6FAB67FED781A206EF2AF0AF6732
:1053C000F4D7808A359CA66BA76B53EC5FF0EE0E8A
:1053D000F76E260EF66E20EED6F0F5EC61F0EE0ECE
:1053E000F76E360EF66E20EEE6F0F5EC61F013EC9B
:1053F00062F03A6A8086809480828090640EAE6FFC
:10540000140EAD6FAB67FED7A0EF0FF03A6A80863F
:10541000809480828090A8EC34F094EF16F0808A1B
:10542000359CF00EF76E060EF66E20EED6F0F5EC1B
:1054300061F0F00EF76E160EF66E20EEE6F0F5EC6B
:1054400061F013EC62F0640EAE6F140EAD6FAD67D9
:10545000FED7A0EF0FF0808A359C359EEF0EF76ED9
:10546000760EF66E20EED6F0F5EC61F0EF0EF76EEC
:10547000860EF66E20EEE6F0F5EC61F013EC62F0CD
:10548000640EAE6F140EAD6FAD67FED7A0EF0FF0D8
:1054900009EC62F09E6B11EED2F003EE00F0410ECB
:1054A000EE6E540EEE6E440EEE6E200E976FE750C9
:1054B000200804E0E6CFEEFF972FF9D73B0EEE6E03
:1054C000000EEE6E00EEE6F011EED2F0100E976FC9
:1054D000E750200804E0E6CFEEFF972FF9D713EC52
:1054E00062F03D903D923E6A57905794579A579C70
:1054F0005890DFEC61F01200140E976F00EE43F04D
:10550000426AEF6607D0422AEE50972FFAD7389AB0
:10551000A0EF0FF0EF6A200E976F08EE32F0200E2A
:10552000EE6E972FFCD73F9E42C084F059EC5DF0A1
:105530003D903D9203EE00F0410EEE6E540EEE6E85
:105540002B0EEE6E430EEE6E4D0EEE6E470EEE6EB1
:10555000520EEE6E3D0EEE6E300E7F637FC0EEFF9C
:10556000806380C0EEFF81C0EEFF000EEE6EDFECC8
:1055700061F0640EAE6FFA0EAD6F3DB0D8EF2AF059
:105580003DB2C5EF2AF0AD67F8D73D92F00EF76E49
:10559000460EF66E20EEE6F0F5EC61F013EC62F0EC
:1055A000640EAE6F1E0EAD6FAD67FED7A0EF0FF0AD
:1055B0003D902EA0EED018EE52F0430EE6626CD075
:1055C000620EE662A5D2120E976F01EEB0F0200EC9
:1055D000EE6E972FFCD7000EE7620BD0120E976F7E
:1055E00018EE32F001EEB0F0E6CFEEFF972FFCD7C9
:1055F0000BD0100E976F01EEB0F0000EE75C04E0E8
:10560000E6CFEEFF972FF9D7B5EC2EF03BA09BD25B
:105610003CA414D01E50030B020828E13B8614EE74
:10562000C0F0A251E126E86AE222E768640EB96F91
:10563000140EB86F7AEC2EF0A0EF0FF0F00EF76EAC
:10564000A60EF66E20EEE6F0F5EC61F000EED6F078
:1056500011EEB0F0100E976FE6CFEEFF972FFCD74C
:1056600013EC62F07AEC2EF0A0EF0FF0F40EF76E70
:10567000A40EF66E20EED6F0F5EC61F0F40EF76EA7
:10568000B40EF66E20EEE6F0F5EC61F013EC62F08D
:105690007AEC2EF0A0EF0FF02EA27BD0120E976FB7
:1056A00008EE00F011EEB0F0200EEE6EE66E972FD1
:1056B000FBD718EE52F0530EE6626BD0630EE66233
:1056C00027D2000EE75CD8B423D2100E976F08EEF5
:1056D00000F02E0EE75C07E0000EE75C04E0E6CF8A
:1056E000EEFF972FF6D7000EE7620BD0120E976FE2
:1056F00018EE32F001EEB0F0E6CFEEFF972FFCD7B8
:1057000011D02E0EE66204D2000EE75CEFE0100E20
:10571000976F01EEB0F0000EE75C04E0E6CFEEFF1D
:10572000972FF9D73C6AB5EC2EF03BA00CD23CA4E5
:1057300085D71E50030B020899E13B8614EEC0F09A
:10574000A251E126E86AE222020EE76E1DEE00F0A9
:10575000080EA203F350E126F450E222080ECB6FAC
:1057600008EE00F0200EEF64EF68EE38F00B816F6A
:10577000200EEF64EF680F0EEE148111E66ECB2F52
:10578000F1D7640EB96F140EB86F7AEC2EF0A0EF5B
:105790000FF02EB41CD0F20EF76ED60EF66E20EE81
:1057A000D6F0F5EC61F0F20EF76EE60EF66E20EE36
:1057B000E6F0F5EC61F013EC62F07AEC2EF0640E9A
:1057C000AE6F140EAD6FAD67FED7A0EF0FF001EE18
:1057D0002EF0200EEF5C19E0100E976F01EE2EF008
:1057E00018EE32F02B0EE76202D018EE33F0EE50D6
:1057F000E6620BD0972FFBD7100E976F01EEB0F03B
:10580000200EEE6E972FFCD712D02EA810D0100EBF
:10581000976F01EE1CF018EE32F02B0EE76202D00B
:1058200018EE33F0EE50E66285D1972FFBD7080EC5
:10583000976F01EE0CF018EE52F0200EEF6202D0DE
:10584000EE5005D0EE50E6625AD1972FF6D7100EE3
:10585000976F01EEB0F0200EEE6E972FFCD72E0E54
:10586000E66256D1410EE6629DD0640EE66299D0A2
:10587000640EE66295D02E0EE66291D0100E976F00
:1058800001EEB0F02E0EE75C04E0E6CFEEFF972FBE
:10589000F9D72E0EE6623CD13C6A590EE76202D07F
:1058A0003C8004D04E0EE76233D13C90E6502E0E81
:1058B000E6622ED1590EE76202D03C8204D04E0E31
:1058C000E76226D13C92E6502E0EE66221D1590EB7
:1058D000E76202D03C8404D04E0EE76219D13C94BA
:1058E000E6502E0EE66214D1590EE76202D03C86D5
:1058F00004D04E0EE7620CD13C96E6502E0EE662C6
:1059000007D1590EE76202D03C8804D04E0EE76200
:10591000FFD03C98B5EC2EF03BA00BD015EE08F074
:105920000A0EA203F350E126F450E2223CC0E7FF46
:1059300021D0F0EC2EF03BA0F4D015EE00F00A0ED2
:10594000A203F350E126F450E222080ECB6F01EEE1
:10595000B0F0200EEF64EF68EE38F00B816F200E90
:10596000EF64EF680F0EEE148111E66ECB2FF1D7C6
:105970003CC0E6FF05EE00F00A0EA203F350E92654
:10598000F450EA22010EAA6E200EA96EF350A92649
:10599000F450AA220A0ECB6FC6EC61F0E9D0E10602
:1059A000E106E106E106430EE66243D06C0EE662D4
:1059B0003FD0720EE6623BD02E0EE66237D0100E5C
:1059C000976F01EEB0F0000EE75C07E02E0EE75C8B
:1059D00004E0E6CFEEFF972FF6D7B5EC2EF03BA014
:1059E000B2D015EE00F00A0EA203F350E126F450F7
:1059F000E222080ECB6FFF0EE66ECB2FFCD7E66AD5
:105A0000E66805EE00F00A0EA203F350E926F45012
:105A1000EA22010EAA6E200EA96EF350A926F450B8
:105A2000AA220A0ECB6FC6EC61F0A2D0E106E10615
:105A3000E106E106460EE6626BD06C0EE66268D0C7
:105A40006D0EE66265D02E0EE66262D0100E976F84
:105A500001EEB0F02E0EE75C0AE02F0EE76458D09E
:105A60003A0EE76055D0E6CFEEFF972FF3D72E0E14
:105A7000E6624ED03C6A590EE76202D03C6804D020
:105A80004E0EE76245D03C6AE6502E0EE66240D0EC
:105A90002F0EE7643DD03A0EE7603AD0E6CF9AF099
:105AA0000F0E9A17100E976F11EEB0F001EE50F036
:105AB000E6CFEEFF972FFCD7FC0E0C16020E3C66CD
:105AC0000C129AC00EF0030EAA6E9E0E100ECB6F33
:105AD00005EE00F0C6EC61F0030EAA6E020E00EEB9
:105AE0000EF0010ECB6FC6EC61F0030EAA6E000E35
:105AF00000EE0CF0010ECB6FC6EC61F039D0F00E69
:105B0000F76E560EF66E20EEE6F0F5EC61F023D05F
:105B1000F00EF76E660EF66E20EEE6F0F5EC61F034
:105B20001AD0F00EF76E760EF66E20EEE6F0F5EC7B
:105B300061F011D0F00EF76E860EF66E20EEE6F0F4
:105B4000F5EC61F008D0F00EF76E960EF66E20EED2
:105B5000E6F0F5EC61F03F8E00EED6F011EEB0F01D
:105B6000100E976FE6CFEEFF972FFCD713EC62F085
:105B70007AEC2EF02EA6A0EF0FF03D903D9203EEB2
:105B800000F0410EEE6E540EEE6E2B0EEE6E430ED6
:105B9000EE6E4D0EEE6E470EEE6E530EEE6E3D0E39
:105BA000EE6E220EEE6E200E976F18EE32F0200E83
:105BB000E75C04E0E6CFEEFF972FF9D7220EEE6EFA
:105BC000EE6ADFEC61F0640EAE6F320EAD6F3DB287
:105BD000EFEF2DF03FB2F1EF2DF0AD67F8D73D922A
:105BE0006FD03F9203EE00F0530EEE6E4D0EEE6E50
:105BF000530EEE6E200EEE6E530EEE6E650EEE6ED2
:105C0000740EEE6E750EEE6E700EEE6E200EEE6E73
:105C10002F0EEE6E400E976F18EE52F0000EE75CFE
:105C200004E0E6CFEEFF972FF9D72F0EEE6E200E91
:105C3000EE6E770EEE6E610EEE6E730EEE6E200E51
:105C4000EE6E3FAE0DD0660EEE6E610EEE6E690E1C
:105C5000EE6E6C0EEE6E650EEE6E640EEE6E12D093
:105C6000730EEE6E750EEE6E630EEE6EEE6E650EDC
:105C7000EE6E730EEE6EEE6E660EEE6E750EEE6EE0
:105C80006C0EEE6E1A0EEE6EEE6A3D903D923F94F3
:105C9000DFEC61F0640EAE6F320EAD6F3DB259EFC6
:105CA0002EF03DB05DEF2EF03FB45BEF2EF0AD6710
:105CB000F5D73D9205D03F94F1D73D90A0EF0FF07E
:105CC000F20EF76E360EF66E20EED6F0F5EC61F0C1
:105CD000F20EF76E460EF66E20EEE6F0F5EC61F091
:105CE00013EC62F0640EAE6F140EAD6FAD67FED7AD
:105CF000A0EF0FF0640EB06F140EAF6F42C084F0CF
:105D000059EC5DF03D903D9203EE00F0410EEE6ED9
:105D1000540EEE6E2B0EEE6E430EEE6E4D0EEE6ECC
:105D2000470EEE6E440EEE6E3D0EEE6E300E7F634D
:105D30007FC0EEFF806380C0EEFF81C0EEFF000EEB
:105D4000EE6EDFEC61F0640EAE6FFA0EAD6F3DB03B
:105D5000B1EF2EF03DB2AFEF2EF0AD67F8D73D9228
:105D600001D03D90AF67FED71200A26B3B9015EEBD
:105D700000F00A0EA203F350E126F450E22201EEF5
:105D8000B0F0FF0EE76026D0080ECB6FE7380F0BA0
:105D9000300F806F080ECB6305D03B0E806302D0BE
:105DA0002B0E806FE6500F0B300F816F200E9A6F15
:105DB0003F0E80619AC080F081619AC081F0EE5000
:105DC000806308D0EE50816305D0CB2FDFD73C84B1
:105DD0003B801200A22B400EA263C9D73B90120059
:105DE000A26B15EE00F00A0EA203F350E126F45068
:105DF000E222FF0EE76202D03B801200A22B3F0E90
:105E0000A265EFD73B901200640EAB6FAB67FED775
:105E1000EECF9DF0200E9D5DD8B436D005EC59F044
:105E2000EFEC5DF0640EAB6FAB67FED7AFEC5DF0EF
:105E3000110E9E6103D09DC0E6FF20D0E7C0E6F0C2
:105E4000E8C0E7F0E9C0E8F0EAC0E9F0EBC0EAF04A
:105E5000ECC0EBF0EDC0ECF0EEC0EDF0EFC0EEF01A
:105E6000F0C0EFF0F1C0F0F0F2C0F1F0F3C0F2F0EA
:105E7000F4C0F3F0F5C0F4F09DC0F5F013EC62F05F
:105E8000974F02D09E2BC0D7000C640EAE6F050E4C
:105E9000AD6FAD67FED7EECF9DF0200E9D5D33E078
:105EA000EFEC58F00B0E9F612FD06FEC18F0110E35
:105EB0009E6103D09DC0E6FF20D0E7C0E6F0E8C0B9
:105EC000E7F0E9C0E8F0EAC0E9F0EBC0EAF0ECC0C6
:105ED000EBF0EDC0ECF0EEC0EDF0EFC0EEF0F0C096
:105EE000EFF0F1C0F0F0F2C0F1F0F3C0F2F0F4C066
:105EF000F3F0F5C0F4F09DC0F5F013EC62F0974FAD
:105F000002D09E2BC2D7000CFF0CC80EAB6FAB6744
:105F1000FED7640EAB6FE8EC5DF0AB67FED7AFEC7D
:105F20005DF03C0EAB6FAB67FED7110ECE6F000E6F
:105F3000CF6FD0EC5EF0300ECE6F180ECF6FD5EC79
:105F40005EF0960EAB6FAB67FED7300ECE6F160EBF
:105F5000CF6FD5EC5EF03C0EAB6FAB67FED7110E8A
:105F6000CE6F480ECF6FD0EC5EF081B0FED7E9EC7B
:105F70005EF004EE00F0EECFCEF0DFEC5EF081B02C
:105F8000FED7E9EC5EF081B0FED7E9EC5EF0CB2FF6
:105F9000F2D7110ECE6F000ECF6FD0EC5EF0F5ECA5
:105FA0005DF0FA0EAB6FAB67FED71200110ECE6F2D
:105FB000000ECF6FD0EC5EF0300ECE6F180ECF6FAC
:105FC000D5EC5EF0FA0EAB6FAB67FED7300ECE6F3E
:105FD000160ECF6FD5EC5EF0960EAB6FAB67FED7AB
:105FE000110ECE6F480ECF6FD0EC5EF081B0FED7B1
:105FF000E9EC5EF004EE00F0EECFCEF0DFEC5EF008
:1060000081B0FED7E9EC5EF081B0FED7E9EC5EF03E
:10601000CB2FF2D7110ECE6F000ECF6FD0EC5EF00B
:10602000F5EC5DF01200110ECE6F000ECF6FD0ECCC
:106030005EF0500ECE6F180ECF6FD5EC5EF0FA0EFC
:10604000AB6FAB67FED7500ECE6F160ECF6FD5EC91
:106050005EF0960EAB6FAB67FED7110ECE6F480E9B
:10606000CF6FD0EC5EF081B0FED7E9EC5EF004EECD
:1060700000F0EECFCEF0DFEC5EF081B0FED7E9ECC1
:106080005EF081B0FED7E9EC5EF0CB2FF2D7110EB7
:10609000CE6F000ECF6FD0EC5EF0F5EC5DF012002D
:1060A000CB6B04EE00F0800EEE6E000EEE6E020E74
:1060B000EE6E000EEE6E11EE8CF0200EE76205D053
:1060C000500EEE6E010ECB270AD0100E976F200EE9
:1060D000E75C05E0CB2BE6CFEEFF972FF8D7CBC0E0
:1060E00003F4020ECB27CBC001F4020ECB27CBC0AA
:1060F00097F004EE00F0C86BEE50C827972F7CEFA6
:1061000030F0C81F010EC827C8C0EEFFCB2B12000D
:10611000376A100E976F01EEC2F0200EEE6E972FC9
:10612000FCD708EE52F0500E976FEE6A972F95EF5E
:1061300030F0E9EC5EF0E4EC5EF03E0ECE6F160E51
:10614000CF6FDAEC5EF0110ECE6F420ECF6FD0EC57
:106150005EF0640EB06F140EAF6FAF51D8B49AD02A
:1061600081B0FBD7E9EC5EF0CEC09AF0E4EC5EF0D3
:106170009AA3F3D7AF51D8B48DD081B0FBD7E9EC57
:106180005EF0CFC09AF0E4EC5EF09AAFF3D73E0E2B
:10619000CE6F360ECF6FDAEC5EF0110ECE6F410E81
:1061A000CF6FD0EC5EF0C86BCB6B08EE52F0AF5106
:1061B00071E081B0FCD7E9EC5EF0E4EC5EF0CEC0BB
:1061C000EEFFCE51C827CB2BAF5164E081B0FCD796
:1061D000E9EC5EF0E4EC5EF0CEC0EEFFCEC097F0EE
:1061E000CE51C827CB27CB2B97510FE0AF5152E0B0
:1061F00081B0FCD7E9EC5EF0E4EC5EF0CEC0EEFFDF
:10620000CE51C827972FF6EF30F0AF5143E081B061
:10621000FCD7E9EC5EF0E4EC5EF0CEC0EEFFCE51D0
:10622000C827CB2B110ECE6F000ECF6FD0EC5EF0D7
:10623000C8672BD018EE52F0800EE66226D0E6CF6B
:1062400097F0020EE76214D0E650E6CFCBF0500E86
:10625000E7601DD0CB5119E0100ECB6501D0CB6F9C
:1062600001EEC2F0E6CFEEFFCB2FFCD73780120055
:10627000040EE76201D00BD0E650E6CFCBF0E6503B
:10628000974F03D0CB2FFBD7DCD737841200378250
:1062900037801200FAD7120037A016D037B20BD0D1
:1062A000100E976F11EEC2F000EEE6F0E6CFEEFFB3
:1062B000972FFCD711D0DE0EF76EF60EF66E20EE9D
:1062C000E6F0F5EC61F008D0DF0EF76E060EF66E24
:1062D00020EEE6F0F5EC61F013EC62F0120004EE53
:1062E00040F0200E976F8B6BFF0EEF5C58E0EF389D
:1062F0000F0B7A6FEE500F0B7B6FEF380F0B7C6F2D
:10630000EE500F0B7D6FEF380F0B7E6FEE500F0BC3
:106310007F6FEF380F0B806FEE500F0B816F0F0EFA
:10632000815D3DE00A0E7A6303D0FA0E7A6F05D0E4
:106330000B0E7A6302D0FB0E7A6F300E7A277B2722
:106340007C277D277E277F27802711EED2F07A5188
:10635000E66225D03F0E7B5D30E07B51E6621FD0C8
:106360003F0E7C5D2AE07C51E66219D03F0E7D5DD8
:1063700024E07D51E66213D03F0E7E5D1EE07E512B
:10638000E6620DD03F0E7F5D18D07F51E66207D0E8
:106390003F0E805D12D08051E66201D00ED08B2B73
:1063A000040E8B03F35004EE40F0E926E86AEA227B
:1063B000972F74EF31F03996FF0C3996010E8163F7
:1063C0003986000C39B607D039B202D038B2AED215
:1063D0003992399402D0398400D038923992399068
:1063E0005790640EAE6F140EAD6F57B0FAEF31F0E8
:1063F000AD67FBD75790389239B4838C39A4839C0E
:106400003D6A576A586A596A39803D903D92D80E64
:10641000F76E9A0EF66E23EE00F0EEEC61F0DE6A97
:10642000DFEC61F0640EAE6F320EAD6F3DB021EF68
:1064300032F03DB21FEF32F0AD67F8D73AD03D925F
:1064400038D03D90640EB06FFA0EAF6F57B058EF72
:1064500033F057B270EF33F057B6C1EF33F059B0A5
:1064600000EF34F059B203EF34F059B469EF34F06F
:1064700059B66BEF34F059B87FEF34F059BA93EF57
:1064800034F03DB26CEF32F0AF67E0D7DD0EF76E5F
:10649000160EF66E20EED6F0F5EC61F0DD0EF76E1E
:1064A000260EF66E20EEE6F0F5EC61F013EC62F0ED
:1064B00040D2EF0EF76EC60EF66E20EED6F0F5EC7B
:1064C00061F0EF0EF76ED60EF66E20EEE6F0F5EC0C
:1064D00061F013EC62F02DD23D923DB812D00A0E5D
:1064E000405CD8B4A3D00B0E405C58E00C0E405C6E
:1064F00042E00D0E405C2BE0100E405CD8B4B2D0F0
:1065000000D0EE0EF76EF60EF66E20EED6F0F5EC3D
:1065100061F0EF0EF76E060EF66E20EEE6F0F5EC8B
:1065200061F010EEEEF0826B40C083F075EC5DF030
:10653000350E3DB87F6F300E7F637FC0E6FF80630E
:1065400080C0E6FF81C0E6FF13EC62F0F2D1EF0EEF
:10655000F76EA60EF66E20EED6F0F5EC61F0EF0EBB
:10656000F76EB60EF66E20EEE6F0F5EC61F013EC89
:1065700062F00000DED1EE0EF76ED60EF66E20EE63
:10658000D6F0F5EC61F0EE0EF76EE60EF66E20EE4C
:10659000E6F0F5EC61F013EC62F0CBD111EE40F0D7
:1065A00039B411EE48F0200EE75CD8B46ED003EE9B
:1065B00000F0410EEE6E540EEE6E2B0EEE6E430E9C
:1065C000EE6E500EEE6E490EEE6E4E0EEE6E3D0EFF
:1065D000EE6E080E976F200EE75C05E0E6CFEEFF4B
:1065E000972FEBEF32F0000EEE6E3D903D92DFEC18
:1065F00061F0640EAE6F320EAD6F3DB006EF33F05A
:106600003DB208EF33F0AD67F8D7A1D73D901ED764
:106610003D923DB876D70A0E405C08E00C0E405C17
:10662000D8B4A9D7100E405C1DE06BD73D92DC0EAC
:10663000F76EB60EF66E20EED6F0F5EC61F0DC0EDD
:10664000F76EA60EF66E20EEE6F0F5EC61F0310E78
:1066500039B4320EF06F39A4399C39B4399E13EC39
:1066600062F067D1EE0EF76EC60EF66E20EED6F033
:10667000F5EC61F0EF0EF76E960EF66E20EEE6F09A
:10668000F5EC61F013EC62F054D1EE0EF76E760E7D
:10669000F66E20EED6F0F5EC61F0EE0EF76E860E9B
:1066A000F66E20EEE6F0F5EC61F013EC62F041D10D
:1066B0005790DC0EF76E560EF66E20EED6F0F5EC27
:1066C00061F0DC0EF76E760EF66E20EEE6F0F5EC7D
:1066D00061F0310E39B4320EDC6F13EC62F029D167
:1066E00057923D903D923D983D903D92D90EF76E68
:1066F000820EF66E23EE00F0EEEC61F0DE6ADFEC67
:1067000061F0640EAE6F320EAD6F3DB09FEF33F0AF
:106710003DB291EF33F03DBCA1EF33F0AD67F5D75B
:10672000C8D63DA893D63D983D920F0E4062C1D683
:10673000640EAE6F050EAD6FAD67FED7D5D73D9039
:1067400085D63D9C000E6F6301D080D6010E6F632D
:1067500001D024D7020E6F6301D00DD7EF0EF76E74
:10676000E60EF66E20EED6F0F5EC61F0EF0EF76E69
:10677000F60EF66E20EEE6F0F5EC61F013EC62F04A
:10678000D8D057963D903D923D903D92D80EF76EF1
:10679000BE0EF66E23EE00F0EEEC61F0DE6ADFEC8A
:1067A00061F0640EAE6F320EAD6F3DB0E0EF33F0CE
:1067B0003DB2DEEF33F0AD67F8D77BD63D9279D6A8
:1067C0003D903D923D903D92D70EF76ECA0EF66E0B
:1067D00023EE00F0EEEC61F0DE6ADFEC61F0640EB7
:1067E000AE6F320EAD6F3DB0FEEF33F03DB2FCEF59
:1067F00033F0AD67F8D75DD63D925BD63D9026D697
:106800005990389223D65992388238A68FD038962C
:106810001E389A6F030E9A17000E9A630ED03D90A1
:106820003D92D70EF76EEE0EF66E23EE00F0EEEC14
:1068300061F0DE6ADFEC61F01ED0010E9A630ED0CB
:106840003D903D92D70EF76EFA0EF66E23EE00F0F5
:10685000EEEC61F0DE6ADFEC61F00DD03D903D9230
:10686000D80EF76E060EF66E23EE00F0EEEC61F039
:10687000DE6ADFEC61F0640EAE6F320EAD6F3DB0DC
:106880004BEF34F03DB248EF34F0AD67F8D74ED05F
:106890003D923DA84BD03D903D903D92D80EF76E75
:1068A000D60EF66E23EE00F0EEEC61F0DE6ADFEC61
:1068B00061F0640EAE6F320EAD6F3DB067EF34F035
:1068C0003DB265EF34F0AD67F8D73D922FD03D90E3
:1068D0002DD05994BBD55996DC0EF76ED60EF66EB8
:1068E00020EED6F0F5EC61F0DC0EF76E960EF66E4B
:1068F00020EEE6F0F5EC61F013EC62F01AD0599856
:10690000DC0EF76EF60EF66E20EED6F0F5EC61F0CA
:10691000DC0EF76E960EF66E20EEE6F0F5EC61F00A
:1069200013EC62F006D0599A388200D0000C3D92E8
:10693000C0D5060EC06FC16BBF8F640EAE6F320E36
:10694000AD6FAD67FED7AFEC5DF034923490EE0CD6
:10695000000E186201D01200010E1862120080862B
:106960008084808280901200000E186201D0120094
:10697000010E186204D08086809480828090020E7E
:1069800018620FD08086808480828090640EAE6F03
:1069900019C0ADF0AD67FED780868094808280906C
:1069A0001200030E186212008096809480928090EC
:1069B000640EAE6F19C0ADF0AD67FED780868094CF
:1069C000808280901200A26B3B90E00E3C1611EE8C
:1069D0008CF0200EE76201D0120015EE00F00A0ED6
:1069E000A203F350E126F450E22201EE8CF0FF0EF8
:1069F000E7602FD0080ECB6FE7380F0B300F806F9A
:106A0000080ECB6305D03B0E806302D02B0E806F47
:106A1000E6500F0B300F816F200E9A6F3F0E806192
:106A20009AC080F081619AC081F0EE50806311D0ED
:106A3000EE5081630ED0CB2FDFD7E7B03C80E7B2BA
:106A40003C82E7B43C84E7B63C86E7B83C883B80B0
:106A50001200A22B400EA263C0D73B901200A26B83
:106A60003B90F00E3C1611EE9EF0200EE76201D036
:106A7000120015EE00F00A0EA203F350E126F450C6
:106A8000E22201EE9EF0FF0EE76031D0080ECB6FE0
:106A9000E7380F0B300F806F080ECB6305D03B0E2D
:106AA000806302D02B0E806FE6500F0B300F816F8A
:106AB000200E9A6F3F0E80619AC080F081619AC06B
:106AC00081F0EE50806313D0EE50816310D0CB2F55
:106AD000DFD73B80E7A412003C843B8614EEC0F075
:106AE000A251E126E86AE222010EE76E1200A22B13
:106AF000400EA263BED73B901200A26B3B90F00EFB
:106B00003C1611EE9EF0200EE76201D0120015EE49
:106B100000F00A0EA203F350E126F450E22201EE47
:106B20009EF0FF0EE76031D0080ECB6FE7380F0BF9
:106B3000300F806F080ECB6305D03B0E806302D010
:106B40002B0E806FE6500F0B300F816F200E9A6F67
:106B50003F0E80619AC080F081619AC081F0EE5052
:106B6000806313D0EE50816310D0CB2FDFD7E7A620
:106B700012003C863B803B8614EEC0F0A251E12619
:106B8000E86AE222010EE76E1200A22B400EA26319
:106B9000BED73B9012003990020EAB6FAB67FED7A9
:106BA000839C020EAB6FAB67FED783AE398C83BE7E
:106BB000399C12003990020EAB6FAB67FED7838C05
:106BC000020EAB6FAB67FED783AE398E83BE399EA4
:106BD0001200C80EAB6FAB67FED7050EEFEC5DF091
:106BE000640EAB6FAB67FED7AFEC5DF0640EAB6FBE
:106BF000AB67FED7050EEFEC5DF0640EAB6FAB67D5
:106C0000FED7AFEC5DF01200C80EAB6FAB67FED7DE
:106C1000050EEFEC5DF0FA0EAB6FAB67FED7AFEC95
:106C20005DF0640EAB6FAB67FED7050EEFEC5DF069
:106C3000FA0EAB6FAB67FED7AFEC5DF01200389089
:106C40003492DE0EF76E260EF66E20EED6F0F5ECE0
:106C500061F009EC62F013EC62F02EEC59F09E6BDF
:106C6000716BE9EC35F001EED2F010EEE6F081B296
:106C7000A0EF0FF0A0B13EEF36F0F9D7FCEC5DF0DD
:106C8000230E9D5D75E09E2B200E9E659DC0EEFF40
:106C90002A0E9A6F100E9E659AC0E6FF13EC62F002
:106CA00037EF36F001EED2F0300EEE6253D0300EF8
:106CB000EE6250D0310EEE624DD0310EEE624AD00F
:106CC000320EEE6247D0320EEE6244D0330EEE62E8
:106CD00041D0330EEE623ED001EE00F0300EEE6E8B
:106CE000EE6EEE6EEE6E01EE0CF0310EEE6E320ECA
:106CF000EE6E330EEE6E340EEE6E350EEE6E360E1A
:106D0000EE6E370EEE6E380EEE6E01EE14F0310EB2
:106D1000EE6E320EEE6E330EEE6E340EEE6E350EFD
:106D2000EE6E360EEE6E370EEE6E380EEE6E01EE35
:106D300004F0340EEE6E320EEE6E330EEE6E380E42
:106D4000EE6E360EEE6E370EEE6E380EEE6E330EC3
:106D5000EE6E22D0DE0EF76E360EF66E20EED6F018
:106D6000F5EC61F009EC62F013EC62F08FEF14F0D7
:106D7000040E9E630DD001EED2F011EE00F0040E71
:106D8000976FEE50E662E6D7972FC1EF36F010D03E
:106D9000080E9E63DFD786D7E9EC35F0716B640E81
:106DA000AE6F0F0EAD6FAD67FED781B2ECEF57F04F
:106DB000000E716315D0DF0EF76EA60EF66E20EE94
:106DC000D6F0F5EC61F0DF0EF76EB60EF66E20EE43
:106DD000E6F0F5EC61F0310EDD6F13EC62F062D09D
:106DE000010E716315D0DF0EF76EA60EF66E20EE63
:106DF000D6F0F5EC61F0DF0EF76EC60EF66E20EE03
:106E0000E6F0F5EC61F0320EDD6F13EC62F04AD083
:106E1000020E716315D0DF0EF76EA60EF66E20EE31
:106E2000D6F0F5EC61F0DF0EF76ED60EF66E20EEC2
:106E3000E6F0F5EC61F0330EDD6F13EC62F032D06A
:106E4000030E716315D0DF0EF76EA60EF66E20EE00
:106E5000D6F0F5EC61F0DF0EF76EE60EF66E20EE82
:106E6000E6F0F5EC61F0340EDD6F13EC62F01AD051
:106E7000040E716315D0DF0EF76EA60EF66E20EECF
:106E8000D6F0F5EC61F0DF0EF76EF60EF66E20EE42
:106E9000E6F0F5EC61F0350EDD6F13EC62F002D038
:106EA000716B86D781B2ECEF57F0A0B159EF37F094
:106EB000F9D7FCEC5DF0230E9D631BD0000E7163CF
:106EC00002D0EEEF52F0010E716302D050EF4BF0A2
:106ED000020E716302D0A1EF45F0030E716302D080
:106EE000FCEF3AF0040E716302D081EF37F0716B62
:106EF0005FD72A0E9D635CD7712B050E7161716B94
:106F000057D7E9EC35F0640EAE6F0F0EAD6FAD677D
:106F1000FED781B2ECEF57F0F00EF76EB60EF66EBC
:106F200020EED6F0F5EC61F0F00EF76EC60EF66EC0
:106F300020EEE6F0F5EC61F013EC62F081B2CCEFFC
:106F400036F0A0B1A5EF37F0F9D7FCEC5DF0230ED9
:106F50009D632AEF3AF0F00EF76EF60EF66E20EE15
:106F6000D6F0F5EC61F0F10EF76E060EF66E20EE3F
:106F7000E6F0F5EC61F013EC62F02EEC59F09E6B4C
:106F800081B283EF37F0A0B1E5EF37F0F9D70F0EFC
:106F90009A6F100E9E619AC09EF09E5111EED2F033
:106FA0009DC0E3FF00EEEEF0070E9A6F9EC097F0D3
:106FB000080E9E619AC097F02A0E9A6F97519AC058
:106FC000EBFF13EC62F09E2BDBD7FCEC5DF0230EA5
:106FD0009D63DDD7080E9E630AD001EE14F011EE1A
:106FE000D2F0EE50E66203D09E2FFBD71CD0F10EFC
:106FF000F76E160EF66E20EED6F0F5EC61F0F10E9F
:10700000F76E260EF66E20EEE6F0F5EC61F013EC6E
:1070100062F004EC36F0640EAE6F140EAD6FAD6727
:10702000FED7CCEF36F0F10EF76E760EF66E20EE50
:10703000D6F0F5EC61F02EB409D0F10EF76E860EA5
:10704000F66E20EEE6F0F5EC61F008D0F10EF76E8A
:10705000960EF66E20EEE6F0F5EC61F013EC62F0C1
:1070600081B283EF37F0A0B137EF38F0F9D7FCECFD
:107070005DF02A0E9D6302D02E74D5D7230E9D633A
:10708000EFD7F10EF76EB60EF66E20EED6F0F5ECF9
:1070900061F02EB609D0F10EF76EC60EF66E20EE38
:1070A000E6F0F5EC61F008D0F10EF76ED60EF66E54
:1070B00020EEE6F0F5EC61F013EC62F081B283EFC4
:1070C00037F0A0B165EF38F0F9D7FCEC5DF02A0E8F
:1070D0009D6302D02E76D5D7230E9D63EFD7F10E98
:1070E000F76EE60EF66E20EED6F0F5EC61F02EB8F7
:1070F00009D0F10EF76EF60EF66E20EEE6F0F5EC26
:1071000061F008D0F20EF76E060EF66E20EEE6F095
:10711000F5EC61F013EC62F081B283EF37F0A0B1CF
:1071200093EF38F0F9D7FCEC5DF02A0E9D6302D0A6
:107130002E78D5D7230E9D63EFD7F20EF76E560E3D
:10714000F66E20EED6F0F5EC61F0100E976F00EEC3
:10715000E6F011EE1CF0E6CFEEFF972FFCD713EC14
:1071600062F09E6B81B2E4EF38F0A0B1B9EF38F075
:10717000F9D7FCEC5DF02A0E9D6306D009EC62F0B5
:1071800013EC62F09E6BEED7230E9D630BD0100EB6
:10719000976F10EEE6F001EE1CF0E6CFEEFF972FB2
:1071A000FCD71ED09E6704D009EC62F010EEE6F02A
:1071B000100E9E619E690F0E9E179E519DC0E3FFAB
:1071C00013EC62F09E2BCED7100E976F10EEE6F008
:1071D00001EE1CF0E6CFEEFF972FFCD783EF37F0E0
:1071E000F20EF76E660EF66E20EED6F0F5EC61F05C
:1071F00009EC62F0080E976F00EEE6F011EE0CF06D
:10720000E6CFEEFF972FFCD713EC62F09E6B81B2B6
:1072100030EF39F0A0B10EEF39F0F9D7FCEC5DF0AA
:107220002A0E9D6308D009EC62F010EEE6F013EC34
:1072300062F09E6BECD7230E9D5D1DE09E6704D02F
:1072400009EC62F010EEE6F0080E9E619E690F0EEA
:107250009E179E519DC0E3FF9E2B13EC62F0D7D783
:10726000080E976F10EEE6F001EE0CF0E6CFEEFFA1
:10727000972FFCD748D6080E976F10EEE6F001EE78
:107280000CF0E6CFEEFF972FFCD7F20EF76E760EDE
:10729000F66E20EED6F0F5EC61F009EC62F013EC3E
:1072A00062F09E6B81B283EF37F0A0B159EF39F0F5
:1072B000F9D7FCEC5DF02A0E9D6325D6F20EF76E31
:1072C000860EF66E20EED6F0F5EC61F0F20EF76E5B
:1072D000960EF66E20EEE6F0F5EC61F013EC62F03F
:1072E0002EEC59F09E6B81B283EF37F0A0B198EF8E
:1072F00039F0F9D70F0E9A6F100E9E619AC09EF06A
:107300009E5111EED2F09DC0E3FF00EEEEF0070EAD
:107310009A6F9EC097F0080E9E619AC097F02A0E51
:107320009A6F97519AC0EBFF13EC62F09E2BDBD75C
:10733000FCEC5DF0230E9D63DDD7080E9E631BD031
:1073400011EED2F0330EE66216D0380EE66213D09C
:10735000370EE66210D0360EE6620DD0380EE662C9
:107360000AD0330EE66207D0320EE66204D0340E45
:10737000E66201D01CD0F20EF76EA60EF66E20EE7D
:10738000D6F0F5EC61F0F20EF76EB60EF66E20EE6A
:10739000E6F0F5EC61F013EC62F004EC36F0640E0C
:1073A000AE6F140EAD6FAD67FED7CCEF36F09E6BAF
:1073B000F20EF76EC60EF66E20EED6F0F5EC61F02A
:1073C000100E976F00EEE6F011EE2EF0E6CFEEFF16
:1073D000972FFCD713EC62F081B21EEF3AF0A0B108
:1073E000F3EF39F0F9D7FCEC5DF02A0E9D6306D07F
:1073F00009EC62F013EC62F09E6BEED7230E9D63F6
:107400000BD0100E976F10EEE6F001EE2EF0E6CFE7
:10741000EEFF972FFCD777D59E6704D009EC62F07A
:1074200010EEE6F0100E9E619E690F0E9E179E51A3
:107430009DC0E3FF13EC62F09E2BCED7100E976F2A
:1074400010EEE6F001EE2EF0E6CFEEFF972FFCD720
:1074500083EF37F0F00EF76ED60EF66E20EED6F014
:10746000F5EC61F0F00EF76EE60EF66E20EEE6F04B
:10747000F5EC61F013EC62F081B283EF37F0A0B16C
:1074800043EF3AF0F9D7FCEC5DF0230E9D6344D551
:10749000F10EF76E360EF66E20EED6F0F5EC61F0DA
:1074A00009EC62F013EC62F02EEC59F09E6B81B2A5
:1074B00083EF37F0A0B173EF3AF0F9D70F0E9A6F60
:1074C000100E9E619AC09EF02A0E9A6F9E5111EE88
:1074D000D2F000EEE6F09DC0E3FF9AC0EBFF13ECA4
:1074E00062F09E2BE4D7FCEC5DF0230E9D63E6D7A3
:1074F000080E9E637CD5080E976F11EE14F001EE16
:10750000D2F0E650EE6273D5972FFBD7F10EF76EEF
:10751000460EF66E20EED6F0F5EC61F009EC62F066
:107520002EEC59F013EC62F09E6B81B283EF37F0D2
:10753000A0B19CEF3AF0F9D7FCEC5DF0230E9D630F
:107540002BD02F0E11EED2F0E7643BD03A0EE7605D
:1075500038D0080E976F01EE14F0E6CFEEFF972FAC
:10756000FCD7F10EF76E560EF66E20EED6F0F5EC67
:1075700061F0F10EF76E660EF66E20EEE6F0F5ECB9
:1075800061F013EC62F0640EAE6F140EAD6FAD6778
:10759000FED7E9EC35F0B7D4070E9A6F080E9E615E
:1075A0009AC09EF02A0E9A6F9E5111EED2F000EE14
:1075B000E6F09DC0E3FF9AC0EBFF13EC62F09E2B58
:1075C000B4D704EC36F0F20EF76E160EF66E20EE1F
:1075D000D6F0F5EC61F0F20EF76E260EF66E20EEA8
:1075E000E6F0F5EC61F013EC62F0640EAE6F140E91
:1075F000AD6FAD67FED787D4E9EC35F0640EAE6FA2
:107600000F0EAD6FAD67FED781B2ECEF57F0E90E0C
:10761000F76E660EF66E20EED6F0F5EC61F0E90E30
:10762000F76E760EF66E20EEE6F0F5EC61F0310EB8
:10763000DF6F13EC62F081B2CCEF36F0A0B122EF35
:107640003BF0F9D7FCEC5DF0230E9D63D8EF3CF0E6
:10765000E90EF76E860EF66E20EED6F0F5EC61F0D0
:10766000E90EF76E960EF66E20EEE6F0F5EC61F0A0
:1076700099EC3CF080C0F3F081C0F4F05AEC3CF09F
:1076800080C0E3F081C0E4F013EC62F09E6B640E06
:10769000B06F060EAF6F81B2F5EF3BF0A0B16DEFAA
:1076A0003BF0AF67F8D7200EE36FE46F13EC62F0A6
:1076B000640EB06F020EAF6F81B2F5EF3BF0A0B178
:1076C0006DEF3BF0AF67F8D75AEC3CF080C0E3F0C9
:1076D00081C0E4F013EC62F0DAD7FCEC5DF0230E2D
:1076E0009D5D25E02A0E9D6303D0300E226EC6D725
:1076F000310E9D5D10E0320E9D5D0DE0330E9D5DFF
:107700000AE0370E9D5D0DE0380E9D5D0AE0390EF2
:107710009D5D07E0B3D7000E2264B0D7F00E22269D
:10772000ADD7600E2260AAD7100E2226A7D75AEC3A
:107730003CF080C0E3F081C0E4F099EC3CF080C004
:10774000F3F081C0F4F013EC62F0640EB06F060E3B
:10775000AF6F81B2F5EF3BF0A0B1CBEF3BF0AF677D
:10776000F8D7200EF36FF46F13EC62F0640EB06F75
:10777000020EAF6F81B2F5EF3BF0A0B1CBEF3BF063
:10778000AF67F8D799EC3CF080C0F3F081C0F4F01B
:1077900013EC62F0DAD7FCEC5DF0230E9D5D25E082
:1077A0002A0E9D6303D0000E236EC7D7310E9D5D58
:1077B00010E0320E9D5D0DE0330E9D5D0AE0370E48
:1077C0009D5D0DE0380E9D5D0AE0390E9D5D07E080
:1077D000B4D70C0E235CB1E0040E2326AED7F40E12
:1077E000235CABE0FC0E2326A8D799EC3CF080C0CC
:1077F000F3F081C0F4F013EC62F01CEC3CF0640E8A
:10780000AE6F320EAD6F3DB00CEF3CF03DB20BEF02
:107810003CF0AD67F8D73D923BEC3CF0640EAE6FA8
:10782000320EAD6F3DB01BEF3CF03DB21AEF3CF0B5
:10783000AD67F8D73D92E2D603EE00F0410EEE6E52
:10784000540EEE6E2B0EEE6E560EEE6E470EEE6E74
:10785000520EEE6E3D0EEE6E22C084F059EC5DF0DD
:107860007FC0EEFF80C0EEFF81C0EEFFEE6A3D6A92
:10787000DFEC61F0120003EE00F0410EEE6E540EEC
:10788000EE6E2B0EEE6E560EEE6E470EEE6E540E34
:10789000EE6E3D0EEE6E23C084F059EC5DF07FC0BD
:1078A000EEFF80C0EEFF81C0EEFFEE6A3D6ADFECC6
:1078B00061F01200100E226005D02B0E806F360E84
:1078C000816F1200200E226005D02B0E806F340EC7
:1078D000816F1200300E226005D02B0E806F320EA9
:1078E000816F1200400E226005D0200E806F300E96
:1078F000816F1200500E226005D02D0E806F320E67
:10790000816F1200600E226005D02D0E806F340E44
:10791000816F1200700E226005D02D0E806F360E22
:10792000816F1200300E226E200E806F300E816F3C
:1079300012000C0E236205D02B0E806F360E816F65
:107940001200080E236205D02B0E806F340E816F5B
:107950001200040E236205D02B0E806F320E816F51
:107960001200000E236205D0200E806F300E816F52
:107970001200FC0E236205D02D0E806F320E816F37
:107980001200F80E236205D02D0E806F340E816F29
:107990001200F40E236205D02D0E806F360E816F1B
:1079A0001200000E236E200E806F300E816F1200C9
:1079B000E90EF76E660EF66E20EED6F0F5EC61F08D
:1079C000E90EF76EA60EF66E20EEE6F0F5EC61F02D
:1079D000320EDF6F13EC62F081B2FEEF3AF0A0B12D
:1079E000F3EF3CF0F9D7FCEC5DF0230E9D632EEF36
:1079F0003EF0E90EF76EB60EF66E20EED6F0F5EC20
:107A000061F0E90EF76EC60EF66E20EEE6F0F5ECCC
:107A100061F020C084F059EC5DF0200EE36FE46F5C
:107A2000300E806380C0E4F081C0E5F021C084F0B6
:107A300059EC5DF0200EF36FF46F300E806380C060
:107A4000F4F081C0F5F013EC62F0640EB06F060E36
:107A5000AF6F81B261EF3DF0A0B153EF3DF0AF6782
:107A6000F8D7200EE36FE46FE56F13EC62F0640E5D
:107A7000B06F020EAF6F81B261EF3DF0A0B153EF76
:107A80003DF0AF67F8D720C084F059EC5DF0200ED0
:107A9000E36FE46F300E806380C0E4F081C0E5F0F6
:107AA00013EC62F0D2D7FCEC5DF0230E9D6301D0A5
:107AB00018D02A0E9D63ADD7202A0F0E2060206AB1
:107AC000A8D720C084F059EC5DF0200EE36FE46F7E
:107AD000300E806380C0E4F081C0E5F013EC62F00A
:107AE00067D020C084F059EC5DF0200EE36FE46FA6
:107AF000300E806380C0E4F081C0E5F021C084F0E6
:107B000059EC5DF0200EF36FF46F300E806380C08F
:107B1000F4F081C0F5F013EC62F0640EB06F060E65
:107B2000AF6F81B2C9EF3DF0A0B1BBEF3DF0AF67E1
:107B3000F8D7200EF36FF46FF56F13EC62F0640E5C
:107B4000B06F020EAF6F81B2C9EF3DF0A0B1BBEFD5
:107B50003DF0AF67F8D721C084F059EC5DF0200EFE
:107B6000F36FF46F300E806380C0F4F081C0F5F0E5
:107B700013EC62F0D2D7FCEC5DF0230E9D6301D0D4
:107B800008D02A0E9D63BAD7212A0F0E2160216AE0
:107B9000B5D721C084F059EC5DF0200EF36FF46F7F
:107BA000300E806380C0F4F081C0F5F013EC62F019
:107BB00003EE00F0410EEE6E540EEE6E2B0EEE6EE6
:107BC000570EEE6E560EEE6E520EEE6E3D0EEE6ED1
:107BD00020C084F059EC5DF07FC0EEFF80C0EEFF66
:107BE00081C0EEFF2C0EEE6E21C084F059EC5DF0EA
:107BF0007FC0EEFF80C0EEFF81C0EEFFEE6A3D6AFF
:107C0000DFEC61F0640EAE6F320EAD6F3DB02BEF66
:107C10003EF03DB20EEF3EF0AD67F8D73D92E90E73
:107C2000F76ED60EF66E20EED6F0F5EC61F0E90EAA
:107C3000F76EE60EF66E20EEE6F0F5EC61F013EC72
:107C400062F0640EAE6F320EAD6FAD67FED7050EFB
:107C5000206E216ACED63D903488D0D4E90EF76EDE
:107C6000660EF66E20EED6F0F5EC61F0E90EF76EDA
:107C7000F60EF66E20EEE6F0F5EC61F0330EDF6FF7
:107C800013EC62F081B2FEEF3AF0A0B149EF3EF0A2
:107C9000F9D7FCEC5DF0230E9D6331EF3FF0EA0E67
:107CA000F76E060EF66E20EED6F0F5EC61F0DAEC2B
:107CB0003EF013EC62F0640EB06F060EAF6F81B24F
:107CC0008BEF3EF0A0B17EEF3EF0AF67F8D7E20E4B
:107CD000F76E560EF66E20EEE6F0F5EC61F013EC62
:107CE00062F0640EB06F020EAF6F81B28BEF3EF0A8
:107CF000A0B17EEF3EF0AF67F8D7D9D7FCEC5DF0CE
:107D00002A0E9D6305D01F2A070E1F601F6ACFD75A
:107D1000230E9D63D0D7DAEC3EF013EC62F003EE55
:107D200000F0410EEE6E540EEE6E2B0EEE6E570E00
:107D3000EE6E4D0EEE6E420EEE6E530EEE6E3D0E7C
:107D4000EE6E1FC084F059EC5DF07FC0EEFF80C086
:107D5000EEFF81C0EEFFEE6A3D6ADFEC61F0640E7B
:107D6000AE6F320EAD6F3DB0D7EF3EF03DB2BBEF20
:107D70003EF0AD67F8D73D92EA0EF76E860EF66ECE
:107D800020EED6F0F5EC61F0EA0EF76E960EF66E88
:107D900020EEE6F0F5EC61F013EC62F0640EAE6FED
:107DA000320EAD6FAD67FED7050E1F6E78D73D90D2
:107DB000348824D4000E1F6209D0EA0EF76E160E26
:107DC000F66E20EEE6F0F5EC61F01200010E1F6297
:107DD00009D0EA0EF76E260EF66E20EEE6F0F5EC10
:107DE00061F01200020E1F6209D0EA0EF76E360E25
:107DF000F66E20EEE6F0F5EC61F01200030E1F6265
:107E000009D0EA0EF76E460EF66E20EEE6F0F5ECBF
:107E100061F01200040E1F6209D0EA0EF76E560ED2
:107E2000F66E20EEE6F0F5EC61F01200050E1F6232
:107E300009D0EA0EF76E660EF66E20EEE6F0F5EC6F
:107E400061F01200060E1F6209D0EA0EF76E760E80
:107E5000F66E20EEE6F0F5EC61F01200050E1F6EF6
:107E6000A9D7E90EF76E660EF66E20EED6F0F5ECA9
:107E700061F0EA0EF76EA60EF66E20EEE6F0F5EC77
:107E800061F0340EDF6F13EC62F081B2FEEF3AF076
:107E9000A0B14CEF3FF0F9D7FCEC5DF0230E9D63F1
:107EA00091EF3FF0E9EC35F0EA0EF76EB60EF66EA4
:107EB00020EED6F0F5EC61F009EC62F013EC62F024
:107EC00001EED2F010EEE6F09E6B81B2FCEF3AF0DC
:107ED000A0B16CEF3FF0F9D7FCEC5DF0230E9D6391
:107EE00012D0040E9E63AAEF36F001EED2F011EE2E
:107EF00000F0EECFE6FFEECFE6FFEECFE6FFEECFEF
:107F0000E6FFFEEF3AF09E2B200E9E659DC0EEFF31
:107F10002A0E9A6F100E9E659AC0E6FF13EC62F06F
:107F2000D4D7E90EF76E660EF66E20EED6F0F5ECBD
:107F300061F0EA0EF76EC60EF66E20EEE6F0F5EC96
:107F400061F0350EDF6F13EC62F081B2FEEF3AF0B4
:107F5000A0B1ACEF3FF0F9D7FCEC5DF0230E9D63D0
:107F600064EF40F0E9EC35F0EE0EF76E960EF66E2B
:107F700020EED6F0F5EC61F0EE0EF76EA60EF66E82
:107F800020EEE6F0F5EC61F03998310E39B8320E9A
:107F9000E56F9E6B080E976F00EEEEF011EE40F06D
:107FA00039B811EE48F0E6CFEEFF972FFCD713EC6F
:107FB00062F0640EB06F060EAF6F81B262EF40F0F8
:107FC000A0B10EEF40F0AF67F8D710EEEEF0200E44
:107FD000E66EE66EE66EE66EE66EE66EE66EE66E01
:107FE00013EC62F0640EB06F020EAF6F81B262EFFD
:107FF00040F0A0B10EEF40F0AF67F8D7080E976FD2
:1080000000EEEEF011EE40F039B811EE48F0E6CF98
:10801000EEFF972FFCD713EC62F0CBD7FCEC5DF0B2
:10802000230E9D5D44E02A0E9D630DD0080E976FD0
:1080300011EE40F039B811EE48F0200EE66E972FA1
:10804000FCD79E6BA7D79E670BD0080E976F11EEDB
:1080500040F039B811EE48F0200EE66E972FFCD7AD
:10806000080E9E610AD011EE40F039B811EE48F0CA
:108070009E519DC0E3FF9E2B8DD7EE0EF76EB60E80
:10808000F66E20EEE6F0F5EC61F013EC62F081B2F2
:1080900062EF40F0A0B14EEF40F0F9D7EE0EF76E70
:1080A000A60EF66E20EEE6F0F5EC61F0BFD730A23A
:1080B00002D0FEEF3AF03978310E39B8320EE56F62
:1080C0009E6B68D7FEEF3AF0E90EF76E660EF66E1D
:1080D00020EED6F0F5EC61F0EA0EF76EF60EF66ED5
:1080E00020EEE6F0F5EC61F0360EDF6F13EC62F097
:1080F00081B2FEEF3AF0A0B17FEF40F0F9D7FCEC8F
:108100005DF0230E9D63FCEF40F0E9EC35F0DB0EF3
:10811000F76E760EF66E20EED6F0F5EC61F009EC17
:1081200062F013EC62F02EEC59F09E6B01EED2F08F
:1081300010EEE6F081B2FEEF3AF0A0B1A1EF40F010
:10814000F9D7FCEC5DF0230E9D5D0EE09E2B200E1A
:108150009E659DC0EEFF2A0E9A6F100E9E659AC016
:10816000E6FF13EC62F0E6D701EED2F0330EEE62DA
:1081700035D0380EEE6232D0370EEE622FD0360E8A
:10818000EE622CD0380EEE6229D0330EEE6226D08D
:10819000320EEE6223D0340EEE6220D0DB0EF76E8C
:1081A000960EF66E20EED6F0F5EC61F0DB0EF76E73
:1081B000A60EF66E20EEE6F0F5EC61F013EC62F040
:1081C000FF0ED16FD26F00EED1F0020ECB6F030E17
:1081D000AA6EFE0EA96EC6EC61F0FF00DE0EF76E11
:1081E000360EF66E20EED6F0F5EC61F009EC62F09A
:1081F00013EC62F08FEF14F0E90EF76E660EF66E78
:1082000020EED6F0F5EC61F0EB0EF76E060EF66E92
:1082100020EEE6F0F5EC61F0370EDF6F13EC62F064
:1082200081B2FEEF3AF0A0B117EF41F0F9D7FCECC4
:108230005DF0230E9D632DEF45F0EB0EF76E360ECD
:10824000F66E20EED6F0F5EC61F009EC62F03F96A8
:108250003D903D92D80EF76E740EF66E23EE00F050
:10826000EEEC61F0DE6ADFEC61F0640EAE6F320EB0
:10827000AD6F3DB058EF41F0AD67FBD7EB0EF76E39
:10828000460EF66E20EED6F0F5EC61F0EB0EF76ED2
:10829000560EF66E20EEE6F0F5EC61F013EC62F0AF
:1082A000640EAE6F140EAD6FAD67FED7CCEF36F037
:1082B000100E976F18EE12F000EEE6F0E6CFEEFF2C
:1082C000972FFCD713EC62F081B2FEEF3AF0A0B129
:1082D0006BEF41F0F9D7FCEC5DF02A0E9D6302D004
:1082E00057EF42F0EB0EF76EE60EF66E20EED6F08C
:1082F000F5EC61F0EB0EF76EF60EF66E20EEE6F0A2
:10830000F5EC61F013EC62F09E6B81B2FEEF3AF097
:10831000A0B1AAEF41F0F9D70F0E9A6F100E9E612F
:108320009AC09EF09E5111EED2F09DC0E3FF00EE88
:10833000EEF0070E9A6F9EC097F0080E9E619AC0ED
:1083400097F02A0E9A6F97519AC0EBFF13EC62F0E8
:108350009E2BDBD7FCEC5DF0230E9D63DDD7080E72
:108360009E6389D001EE04F011EED2F0EE50E66289
:1083700082D09E2FFBD7EC0EF76E060EF66E20EE27
:10838000D6F0F5EC61F0EC0EF76E160EF66E20EE00
:10839000E6F0F5EC61F013EC62F02EEC59F013EC22
:1083A00062F09E6B81B2FEEF3AF0A0B1D9EF41F0DE
:1083B000F9D7FCEC5DF0230E9D632CD02F0E11EE4F
:1083C000D2F0E7643CD03A0EE76039D0080E976FE0
:1083D00001EE04F0E6CFEEFF972FFCD7EC0EF76E20
:1083E000260EF66E20EED6F0F5EC61F0EC0EF76E90
:1083F000360EF66E20EEE6F0F5EC61F013EC62F06E
:10840000640EAE6F140EAD6FAD67FED7E9EC35F0BC
:10841000FEEF3AF0070E9A6F080E9E619AC09EF02A
:108420002A0E9A6F9E5111EED2F000EEEEF09DC032
:10843000E3FF9AC0EBFF13EC62F09E2BB3D704EC82
:1084400036F0EC0EF76E660EF66E20EED6F0F5EC1A
:1084500061F0EC0EF76E760EF66E20EEE6F0F5ECBF
:1084600061F013EC62F0640EAE6F140EAD6FAD6789
:10847000FED7FEEF3AF0EC0EF76E460EF66E20EEEB
:10848000D6F0F5EC61F0EC0EF76E560EF66E20EEBF
:10849000E6F0F5EC61F013EC62F004EC36F0640EFB
:1084A000AE6F140EAD6FAD67FED7CCEF36F0EB0EAE
:1084B000F76E660EF66E20EED6F0F5EC61F0EB0E80
:1084C000F76E760EF66E20EEE6F0F5EC61F013EC4A
:1084D00062F02EEC59F09E6B81B2FEEF3AF0A0B143
:1084E00091EF42F0F9D70F0E9A6F100E9E619AC06D
:1084F0009EF09E5111EED2F09DC0E3FF00EEEEF033
:10850000070E9A6F9EC097F0080E9E619AC097F072
:108510002A0E9A6F97519AC0EBFF13EC62F09E2BD4
:10852000DBD7FCEC5DF0230E9D63DDD7080E9E6368
:108530000AD001EE04F011EED2F0EE50E66203D064
:108540009E2FFBD71CD0EC0EF76E460EF66E20EE7B
:10855000D6F0F5EC61F0EC0EF76E560EF66E20EEEE
:10856000E6F0F5EC61F013EC62F004EC36F0640E2A
:10857000AE6F140EAD6FAD67FED7CCEF36F0EB0EDD
:10858000F76E860EF66E20EED6F0F5EC61F009EC93
:1085900062F013EC62F02EEC59F09E6B81B2FEEFAC
:1085A0003AF0A0B1E8EF42F0F9D70F0E9A6F100E33
:1085B0009E619AC09EF09E5111EED2F09DC0E3FFE5
:1085C00000EEE6F09DC0EBFF13EC62F09E2BE6D7C9
:1085D000FCEC5DF02A0E9D6301D0D9D7230E9D637C
:1085E000E4D70F0E9E6301D003D00E0E9E6340D0E1
:1085F0003D903D92D80EF76E6A0EF66E23EE00F0B7
:10860000EEEC61F0DE6ADFEC61F0640EAE6F640EDA
:10861000AD6F3DB04CEF43F03DB214EF43F03FB8C7
:108620004EEF43F0AD67F5D73D92EB0EF76E160EA9
:10863000F66E20EED6F0F5EC61F0EB0EF76E260E3E
:10864000F66E20EEE6F0F5EC61F013EC62F0A66B4E
:10865000A76B53EC5FF0A68753EC5FF0020EC06F80
:10866000C16BBF8F81A232EF43F0AFEC5DF0FF0032
:10867000EB0EF76E960EF66E20EED6F0F5EC61F08E
:10868000EB0EF76EA60EF66E20EEE6F0F5EC61F05E
:1086900013EC62F08FEF14F03D90BBD73F983D9EF6
:1086A000640EAE6F640EAD6F3DBE03D0AD67FCD7F8
:1086B000BCD73D9E150EC963F7D7EB0EF76EB60E0D
:1086C000F66E20EED6F0F5EC61F013EC62F0890E58
:1086D000F76EB40EF66E100E986FD1EC44F0100EDB
:1086E000986FC7EC44F0890EF76EC40EF66E100E4C
:1086F000986FD1EC44F0100E986FC7EC44F0890EDF
:10870000F76ED40EF66E100E986FD1EC44F0100E8A
:10871000986FC7EC44F0890EF76EE40EF66E100EFB
:10872000986FD1EC44F0100E986FC7EC44F0890EAE
:10873000F76EF40EF66E100E986FD1EC44F0100E3A
:10874000986FC7EC44F0030E976F8A0EF76E040E15
:10875000F66E100E986FD1EC44F0100E986FC7ECC7
:1087600044F0972FF2D78A0EF76E140EF66E100EA5
:10877000986FD1EC44F0100E986FC7EC44F08A0E5D
:10878000F76E240EF66E100E986FD1EC44F0100EBA
:10879000986FC7EC44F08A0EF76E340EF66E100E2A
:1087A000986FD1EC44F0100E986FC7EC44F0350E82
:1087B000976F8A0EF76E440EF66E100E986FD1EC1E
:1087C00044F0100E986FC7EC44F0972FF2D78A0E42
:1087D000F76E540EF66E040E986FD1EC44F0040E52
:1087E000986FC7EC44F0640EAE6F050EAD6FAD67C9
:1087F000FED78A0EF76E580EF66E010E986FD1EC0A
:1088000044F0010E986FC7EC44F0640EAE6F0A0E90
:10881000AD6FAD67FED78280576A640EAE6F050EEE
:10882000AD6FAD67FED78290640EAE6F140EAD6F64
:10883000AD67FED73D903D92D80EF76E9A0EF66E5C
:1088400023EE00F0EEEC61F0DE6ADFEC61F0640E26
:10885000AE6F640EAD6F57B637EF44F057B037EFD9
:1088600044F03DB003D0AD67F6D7DFD63D903D90E4
:108870003D92D80EF76E120EF66E23EE00F0EEEC7F
:1088800061F0DE6ADFEC61F0640EAE6F140EAD6F66
:108890003DB051EF44F03DB215EF43F0AD67F8D76E
:1088A000C4D63D903D92D80EF76E2E0EF66E23EE96
:1088B00000F0EEEC61F0DE6ADFEC61F0640EAE6FAA
:1088C000320EAD6F3DB06CEF44F03DB26AEF44F054
:1088D000AD67F8D73D92A9D6640EAE6F140EAD6F9A
:1088E000AD67FED703EE00F0410EEE6E540EEE6E55
:1088F0002B0EEE6E570EEE6E490EEE6E4D0EEE6EB8
:10890000450EEE6E490EEE6E3D0EEE6E100E976F3A
:1089100011EED2F0200EE76404D0E6CFEEFF972FE1
:10892000F9D70D0EEE6EEE6ADFEC61F0640EAE6FFD
:10893000640EAD6F3DB2A2EF44F03DB0A4EF44F041
:10894000AD67F8D73D9271D6EB0EF76EC60EF66E98
:1089500020EED6F0F5EC61F0EB0EF76ED60EF66E6B
:1089600020EEE6F0F5EC61F013EC62F0A66BA76B7D
:1089700053EC5FF0A68753EC5FF0020EC06FC16B43
:10898000BF8F81A2C1EF44F0AFEC5DF0FF0003EEBA
:1089900000F0EECFADFF00009EA8FED7982FF9D7CC
:1089A0001200F86A03EE00F00900F5CFEEFF982FF1
:1089B000FBD712000201FE454550524F4D202020AA
:1089C0002032382F30312F30302031323A303800D9
:1089D0002056657273696F6E2076316130362020C3
:1089E0002020202020433A5C544D505C746D705C14
:1089F0003430305F6D3131622E35345C6F75740008
:108A00002020202020202020202020202020202066
:108A100020202020207E81F7EB1800000090825853
:108A2000AD2A010200CDAB12000100005E01090079
:108A3000BAD34D75FE4A6F92F11A1A1A1A1A1A1AF7
:108A40001A1A1A1A1A1A1A1A1A1A1A1A1A1A1A1A86
:108A50001A1A1A1A1A1A1A910400E90EF76E660EFB
:108A6000F66E20EED6F0F5EC61F0EC0EF76E860EA9
:108A7000F66E20EEE6F0F5EC61F0380EDF6F13ECE9
:108A800062F081B2FEEF3AF0A0B148EF45F0F9D7BD
:108A9000FCEC5DF0230E9D63FEEF3AF0EC0EF76EFA
:108AA000960EF66E20EED6F0F5EC61F030C081F057
:108AB00030B009D0EC0EF76EA60EF66E20EEE6F0A2
:108AC000F5EC61F008D0EC0EF76EB60EF66E20EE07
:108AD000E6F0F5EC61F013EC62F0640EAE6F060E9A
:108AE000AD6F81B2FEEF3AF0A0B190EF45F0AD6707
:108AF000F8D7E20EF76E560EF66E20EEE6F0F5ECC5
:108B000061F013EC62F0640EAE6F020EAD6F81B2D5
:108B1000FEEF3AF0A0B190EF45F0AD67F8D7C8D7B7
:108B2000FCEC5DF02A0E9D6302D03070C1D7230E9D
:108B30009D63BED781A1FEEF3AF030A03488FEEFEE
:108B40003AF0640EAE6F0F0EAD6FAD67FED781B217
:108B5000ECEF57F0E60EF76EB60EF66E20EED6F09E
:108B6000F5EC61F0E60EF76EC60EF66E20EEE6F05E
:108B7000F5EC61F0310EDF6F13EC62F081B2CCEFF7
:108B800036F0A0B1C5EF45F0F9D7FCEC5DF0230E4F
:108B90009D6364EF46F0E60EF76ED60EF66E20EE9D
:108BA000D6F0F5EC61F01EEC4BF013EC62F0640EC5
:108BB000AE6F060EAD6F81B2A1EF45F0A0B1FAEF36
:108BC00045F0AD67F8D7E70EF76E160EF66E20EE9D
:108BD000E6F0F5EC61F013EC62F0640EAE6F020E9D
:108BE000AD6F81B2A1EF45F0A0B1FAEF45F0AD67EE
:108BF000F8D7D9D7FCEC5DF02A0E9D630CD00CC0E1
:108C000081F0FC0E0C16030E8117812B8161816BA4
:108C100081510C12C8D7230E9D63C5D7E70EF76E9E
:108C2000260EF66E20EED6F0F5EC61F00CB409D00D
:108C3000E70EF76E460EF66E20EEE6F0F5EC61F00C
:108C400008D0E70EF76E360EF66E20EEE6F0F5EC85
:108C500061F013EC62F081B2A1EF45F0A0B132EF08
:108C600046F0F9D7FCEC5DF0230E9D5D02E00C743C
:108C7000D5D7E70EF76E560EF66E20EED6F0F5EC71
:108C800061F00CB609D0E70EF76E760EF66E20EEA8
:108C9000E6F0F5EC61F008D0E70EF76E660EF66EC2
:108CA00020EEE6F0F5EC61F013EC62F081B2A1EF9A
:108CB00045F0A0B15DEF46F0F9D7FCEC5DF0230E76
:108CC0009D5D02E00C76D5D7E60EF76EB60EF66E19
:108CD00020EED6F0F5EC61F0E70EF76E860EF66E3C
:108CE00020EEE6F0F5EC61F0320EDF6F13EC62F08F
:108CF00081B2A1EF45F0A0B17FEF46F0F9D7FCECCF
:108D00005DF0230E9D6348EF47F0E70EF76E960E79
:108D1000F66E20EED6F0F5EC61F0E70EF76EA60EDB
:108D2000F66E20EEE6F0F5EC61F013EC62F0640E06
:108D3000B06F060EAF6F81B2A1EF45F0A0B1BAEFF0
:108D400046F0AF67F8D7200EF56F13EC62F0640EB3
:108D5000B06F020EAF6F81B2A1EF45F0A0B1BAEFD4
:108D600046F0AF67F8D70E500F0B300FF56F13ECCE
:108D700062F0DDD7FCEC5DF02A0E9D6304D00E6A34
:108D8000300EF56FD4D7230E9D6301D008D00F0E9F
:108D90009D150E6E9DC0F5F013EC62F0C8D7E70E7E
:108DA000F76EB60EF66E20EED6F0F5EC61F009EC3B
:108DB00062F001EE50F011EED2F0100E8B6FEECF9C
:108DC000E6FF8B2FFCD79E6B01EED2F010EEE6F0A3
:108DD000100E8B6FEECFE6FF8B2FFCD713EC62F0FB
:108DE00081B23CEF47F0A0B1F7EF46F0F9D7FCECC9
:108DF0005DF02A0E9D630AD0100E8B6F01EED2F04B
:108E0000200EEE6E8B2FFCD79E6BDED7230E9D635C
:108E100001D027D09E6708D0100E8B6F01EED2F0E4
:108E2000200EEE6E8B2FFCD7100E9E6115D0010E1A
:108E30009E630BD0300E9D6308D0300E01EED2F051
:108E4000EF6203D09E6B2B0E9D6F9E5111EED2F000
:108E50009DC0E3FF9E2BB8D704EC36F0100E9E6F3A
:108E6000B3D7100E8B6F01EED2F011EE50F0EECFB3
:108E7000E6FF8B2FFCD70CD0100E8B6F01EED2F0DB
:108E800011EE50F0EECFE6FF8B2FFCD7A1EF45F0AF
:108E9000E60EF76EB60EF66E20EED6F0F5EC61F04B
:108EA000E70EF76EC60EF66E20EEE6F0F5EC61F01A
:108EB000330EDF6F13EC62F081B2A1EF45F0A0B189
:108EC00063EF47F0F9D7FCEC5DF0230E9D6307EFED
:108ED0004AF0E70EF76ED60EF66E20EED6F0F5EC01
:108EE00061F0E70EF76EE60EF66E20EEE6F0F5ECBA
:108EF00061F09E6B10C084F059EC5DF080C0F4F01E
:108F000081C0F5F013EC62F0640EB06F060EAF6F27
:108F100081B2A1EF45F0A0B1A8EF47F0AF67F8D755
:108F2000200EF46FF56F13EC62F0640EB06F020E5A
:108F3000AF6F81B2A1EF45F0A0B1A8EF47F0AF67E6
:108F4000F8D780C0F4F081C0F5F013EC62F0DCD704
:108F5000FCEC5DF02A0E9D6304D0010E106E9E6B3A
:108F6000C9D7230E9D5D25E09E6708D0200EF46FC3
:108F7000F56F300E7F6F806F816F9E6B030E9E6169
:108F800012D080C07FF081C080F09DC081F00FECD6
:108F90005DF0000E846507D0210E846104D084C08A
:108FA00010F09E2BA7D704EC36F0010E106E9E6BCE
:108FB000A1D7E70EF76EF60EF66E20EED6F0F5ECC2
:108FC00061F0E80EF76E060EF66E20EEE6F0F5ECB8
:108FD00061F09E6B11C084F059EC5DF080C0F4F03C
:108FE00081C0F5F013EC62F0640EB06F060EAF6F47
:108FF00081B2A1EF45F0A0B118EF48F0AF67F8D704
:10900000200EF46FF56F13EC62F0640EB06F020E79
:10901000AF6F81B2A1EF45F0A0B118EF48F0AF6794
:10902000F8D780C0F4F081C0F5F013EC62F0DCD723
:10903000FCEC5DF02A0E9D6304D0010E116E9E6B58
:10904000C9D7230E9D5D25E09E6708D0200EF46FE2
:10905000F56F300E7F6F806F816F9E6B030E9E6188
:1090600012D080C07FF081C080F09DC081F00FECF5
:109070005DF0000E846507D0210E846104D084C0A9
:1090800011F09E2BA7D704EC36F0010E116E9E6BEB
:10909000A1D7E80EF76E160EF66E20EED6F0F5ECC0
:1090A00061F0E80EF76E260EF66E20EEE6F0F5ECB7
:1090B00061F012C084F059EC5DF080C0E8F02E0E33
:1090C000E96F81C0EAF013EC62F0640EB06F060E37
:1090D000AF6F81B2A1EF45F0A0B18CEF48F0AF6760
:1090E000F8D7200EE86FE96FEA6F13EC62F0640EB8
:1090F000B06F020EAF6F81B2A1EF45F0A0B18CEF5F
:1091000048F0AF67F8D780C0E8F02E0EE96F81C055
:10911000EAF013EC62F0D9D7FCEC5DF0230E9D5D14
:1091200013E02A0E9D6303D0050E126EC2D712C043
:1091300084F0050E8427370E846103D084C012F0BA
:10914000B8D70A0E126EB5D7E80EF76E360EF66E69
:1091500020EED6F0F5EC61F0E80EF76E460EF66EF6
:1091600020EEE6F0F5EC61F013C084F059EC5DF010
:109170007FC0F4F080C0F5F013EC62F0640EB06FC5
:10918000060EAF6F81B2A1EF45F0A0B1E2EF48F05B
:10919000AF67F8D7200EF46FF56F13EC62F0640E32
:1091A000B06F020EAF6F81B2A1EF45F0A0B1E2EF58
:1091B00048F0AF67F8D77FC0F4F080C0F5F013EC4B
:1091C00062F0DCD7FCEC5DF0230E9D5D16E02A0E0C
:1091D0009D6303D00A0E136EC7D713C084F00A0E26
:1091E0008427FB0E846106D0090E846503D084C0F9
:1091F00013F0BAD70A0E136EB7D7E80EF76E560EF5
:10920000F66E20EED6F0F5EC61F00CBE09D0E80E5B
:10921000F76E660EF66E20EEE6F0F5EC61F008D023
:10922000E80EF76E760EF66E20EEE6F0F5EC61F0E5
:1092300013EC62F081B2A1EF45F0A0B121EF49F04B
:10924000F9D7FCEC5DF02A0E9D6302D00C7ED5D7D9
:10925000230E9D63EFD7E80EF76E860EF66E20EEB6
:10926000D6F0F5EC61F0E80EF76E960EF66E20EE95
:10927000E6F0F5EC61F09E6B080E976F11EE70F062
:1092800000EEEEF0E6CFEEFF972FFCD713EC62F086
:1092900081B277EF49F0A0B14FEF49F0F9D7FCEC7C
:1092A0005DF02A0E9D6325D0080E976F01EE70F0D9
:1092B000200EEE6E972FFCD79E6BDED79E6708D0F0
:1092C000080E976F01EE70F0200EEE6E972FFCD710
:1092D0009E2B090E9E6106D09E5111EE6FF09DC02F
:1092E000E3FFCAD704EC36F0080E9E6FC5D7A1EF96
:1092F00045F0230E9D63E2D7E80EF76EA60EF66EDC
:1093000020EED6F0F5EC61F0E80EF76EB60EF66ED4
:1093100020EEE6F0F5EC61F09E6B040E976F11EE17
:1093200078F000EEF2F0E6CFEEFF972FFCD713ECCB
:1093300062F081B2C8EF49F0A0B1A0EF49F0F9D7CF
:10934000FCEC5DF02A0E9D6325D0040E976F01EEB4
:1093500078F0200EEE6E972FFCD79E6BDED79E67BF
:1093600008D0040E976F01EE78F0200EEE6E972F66
:10937000FCD79E2B050E9E6106D09E5111EE77F014
:109380009DC0E3FFCAD704EC36F0040E9E6FC5D72C
:10939000A1EF45F0230E9D63E2D7E80EF76EC60EEF
:1093A000F66E20EED6F0F5EC61F0E80EF76ED60E14
:1093B000F66E20EEE6F0F5EC61F09E6B0F50300F8C
:1093C000F56F13EC62F081B200EF4AF0A0B1EAEF62
:1093D00049F0F9D7FCEC5DF02A0E9D6313D00F6ABB
:1093E0009E6BECD79E2B020E9E6105D09D51F56FB2
:1093F0000F0B0F6EE3D704EC36F09E6B0F6ADED7CF
:10940000A1EF45F0230E9D63EDD7A1EF45F0E60EE9
:10941000F76EB60EF66E20EED6F0F5EC61F0E80EC3
:10942000F76EE60EF66E20EEE6F0F5EC61F0310E2A
:10943000DF6F13EC62F081B2A1EF45F0A0B122EF33
:109440004AF0F9D7FCEC5DF0230E9D63A1EF45F0E7
:109450009E6BE80EF76EF60EF66E20EED6F0F5EC8B
:1094600061F0E90EF76E060EF66E20EEE6F0F5EC12
:1094700061F0000E146207D0320E7F6F350E806FE0
:10948000300E816F20D0010E146207D0330E7F6F33
:10949000370E806F350E816F16D0020E146207D022
:1094A000340E7F6F300E806F300E816F0CD0030E44
:1094B000146207D0350E7F6F300E806F300E816FD3
:1094C00002D0146AD6D77FC0EEF080C0EFF081C022
:1094D000F0F013EC62F0640EB06F060EAF6F81B265
:1094E000A1EF45F0A0B192EF4AF0AF67F8D7200E98
:1094F000EE6FEF6FF06F13EC62F0640EB06F020E60
:10950000AF6F81B2A1EF45F0A0B192EF4AF0AF6723
:10951000F8D77FC0EEF080C0EFF081C0F0F013EC20
:1095200062F0D9D7FCEC5DF02A0E9D6308D0142AB6
:10953000040E1460146A8EEC5FF08E6F9AD7230EBF
:109540009D6397D79E6BE90EF76E160EF66E20EEB2
:10955000D6F0F5EC61F0E90EF76E260EF66E20EE11
:10956000E6F0F5EC61F0000E156207D0320E7F6F69
:10957000350E806F300E816F20D0010E156207D03E
:10958000330E7F6F370E806F350E816F16D0020E4F
:10959000156207D0340E7F6F300E806F300E816FF2
:1095A0000CD0030E156207D0350E7F6F300E806F22
:1095B000300E816F02D0156AD6D77FC0EEF080C022
:1095C000EFF081C0F0F013EC62F0640EB06F060EA5
:1095D000AF6F81B2A1EF45F0A0B10CEF4BF0AF67D8
:1095E000F8D7200EEE6FEF6FF06F13EC62F0640EA1
:1095F000B06F020EAF6F81B2A1EF45F0A0B10CEFDA
:109600004BF0AF67F8D77FC0EEF080C0EFF081C0BD
:10961000F0F013EC62F0D9D7FCEC5DF02A0E9D63FC
:1096200008D0152A040E1560156A9DEC5FF08F6F47
:109630009AD7230E9D6397D7A1EF45F00C50030BEB
:10964000816F000E816309D0E60EF76EE60EF66EAE
:1096500020EEE6F0F5EC61F01200010E816309D016
:10966000E60EF76EF60EF66E20EEE6F0F5EC61F023
:109670001200020E816309D0E70EF76E060EF66E39
:1096800020EEE6F0F5EC61F01200FC0E0C16E60E92
:10969000F76EE60EF66E20EEE6F0F5EC61F01200E5
:1096A000640EAE6F0F0EAD6FAD67FED781B2ECEFFB
:1096B00057F0E10EF76EA60EF66E20EED6F0F5EC42
:1096C00061F0E10EF76EB60EF66E20EEE6F0F5EC08
:1096D00061F0310EDF6F13EC62F081B2CCEF36F047
:1096E000A0B174EF4BF0F9D7FCEC5DF0230E9D6355
:1096F000D9EF4BF0E10EF76EC60EF66E20EED6F007
:10970000F5EC61F016B609D0E10EF76EE60EF66ED6
:1097100020EEE6F0F5EC61F008D0E10EF76ED60E23
:10972000F66E20EEE6F0F5EC61F013EC62F0640EFC
:10973000B06F060EAF6F81B250EF4BF0A0B1CFEF1C
:109740004BF0AF67F8D7E10EF76EF60EF66E20EE2F
:10975000E6F0F5EC61F013EC62F0640EB06F020E0F
:10976000AF6F81B250EF4BF0A0B1CFEF4BF0AF67CE
:10977000F8D716B609D0E10EF76EE60EF66E20EEBB
:10978000E6F0F5EC61F008D0E10EF76ED60EF66E5D
:1097900020EEE6F0F5EC61F013EC62F0C8D7FCECDB
:1097A0005DF02A0E9D6302D01676ACD7230E9D6322
:1097B000BED7E10EF76EA60EF66E20EED6F0F5ECF3
:1097C00061F0E20EF76E060EF66E20EEE6F0F5ECB6
:1097D00061F0320EDF6F13EC62F081B250EF4BF0AC
:1097E000A0B1F4EF4BF0F9D7FCEC5DF0230E9D63D4
:1097F000A7EF4CF0E20EF76E060EF66E20EED6F0F6
:10980000F5EC61F0B0EC52F013EC62F0640EAE6F68
:10981000060EAD6F81B250EF4BF0A0B129EF4CF0C6
:10982000AD67F8D7E20EF76E560EF66E20EEE6F054
:10983000F5EC61F013EC62F0640EAE6F020EAD6FEA
:1098400081B250EF4BF0A0B129EF4CF0AD67F8D7E3
:10985000D9D7FCEC5DF02A0E9D6307D0FC0E1E16D6
:10986000812B030E81151E12CDD7230E9D63CAD7FF
:10987000B0EC52F013EC62F0E20EF76E660EF66E8C
:1098800020EED6F0F5EC61F009EC62F001EE60F04C
:1098900011EED2F0100E8B6FEECFE6FF8B2FFCD7C0
:1098A0009E6B01EED2F010EEE6F0100E8B6FEECF55
:1098B000E6FF8B2FFCD713EC62F081B29BEF4CF0EC
:1098C000A0B164EF4CF0F9D7FCEC5DF02A0E9D637B
:1098D0000AD0100E8B6F01EED2F0200EEE6E8B2FA1
:1098E000FCD79E6BDED7230E9D6301D019D09E67F7
:1098F00008D0100E8B6F01EED2F0200EEE6E8B2F83
:10990000FCD79E2B110E9E6106D09E5111EED1F018
:109910009DC0E3FFC6D704EC36F0100E9E6FC1D792
:10992000100E8B6F01EED2F011EE60F0EECFE6FF7D
:109930008B2FFCD70CD0100E8B6F01EED2F011EEF6
:1099400060F0EECFE6FF8B2FFCD750EF4BF0E10E2F
:10995000F76EA60EF66E20EED6F0F5EC61F0E20E94
:10996000F76E760EF66E20EEE6F0F5EC61F0330E53
:10997000DF6F13EC62F081B250EF4BF0A0B1C2EF99
:109980004CF0F9D7FCEC5DF0230E9D63F6EF4CF044
:10999000E20EF76E860EF66E20EED6F0F5EC61F074
:1099A0001EAC09D0E20EF76E960EF66E20EEE6F0D3
:1099B000F5EC61F008D0E20EF76EA60EF66E20EE22
:1099C000E6F0F5EC61F013EC62F081B250EF4BF091
:1099D000A0B1ECEF4CF0F9D7FCEC5DF02A0E9D63E2
:1099E00002D01E7CD5D7230E9D63DAD7E10EF76E29
:1099F000A60EF66E20EED6F0F5EC61F0E20EF76EF4
:109A0000B60EF66E20EEE6F0F5EC61F0340EDF6F88
:109A100013EC62F081B250EF4BF0A0B111EF4DF0BA
:109A2000F9D7FCEC5DF0230E9D63D5EF4DF0E30E0E
:109A3000F76E060EF66E20EED6F0F5EC61F01EB66F
:109A400009D0E30EF76E160EF66E20EEE6F0F5EC9A
:109A500061F008D0E30EF76E260EF66E20EEE6F00B
:109A6000F5EC61F013EC62F0640EB06F060EAF6FB0
:109A700081B250EF4BF0A0B16CEF4DF0AF67F8D76B
:109A8000E30EF76E360EF66E20EEE6F0F5EC61F0C2
:109A900013EC62F0640EB06F020EAF6F81B250EF44
:109AA0004BF0A0B16CEF4DF0AF67F8D71EB609D000
:109AB000E30EF76E160EF66E20EEE6F0F5EC61F0B2
:109AC00008D0E30EF76E260EF66E20EEE6F0F5EC0B
:109AD00061F013EC62F0C8D7FCEC5DF02A0E9D63D8
:109AE00002D01E76ACD7230E9D63A9D7E30EF76E86
:109AF000460EF66E20EED6F0F5EC61F02EB009D0F1
:109B0000E30EF76E560EF66E20EEE6F0F5EC61F021
:109B100008D0E30EF76E660EF66E20EEE6F0F5EC7A
:109B200061F013EC62F0640EB06F060EAF6F81B29D
:109B300050EF4BF0A0B1CBEF4DF0AF67F8D7E30E8D
:109B4000F76E760EF66E20EEE6F0F5EC61F013ECB3
:109B500062F0640EB06F020EAF6F81B250EF4BF047
:109B6000A0B1CBEF4DF0AF67F8D72EB009D0E30E20
:109B7000F76E560EF66E20EEE6F0F5EC61F008D0CA
:109B8000E30EF76E660EF66E20EEE6F0F5EC61F091
:109B900013EC62F0C8D7FCEC5DF02A0E9D6302D096
:109BA0002E70ACD7230E9D63A9D7E10EF76EA60EDB
:109BB000F66E20EED6F0F5EC61F0E30EF76E860E51
:109BC000F66E20EEE6F0F5EC61F0350EDF6F13EC8B
:109BD00062F081B250EF4BF0A0B1F0EF4DF0F9D749
:109BE000FCEC5DF0230E9D6357EF4EF0E30EF76E35
:109BF000960EF66E20EED6F0F5EC61F01EB409D0AC
:109C0000E30EF76EC60EF66E20EEE6F0F5EC61F0B0
:109C100008D0E30EF76EB60EF66E20EEE6F0F5EC29
:109C200061F013EC62F0640EB06F060EAF6F81B29C
:109C300055EF4EF0A0B14BEF4EF0AF67F8D7E30E03
:109C4000F76EA60EF66E20EEE6F0F5EC61F013EC82
:109C500062F0640EB06F020EAF6F81B255EF4EF03E
:109C6000A0B14BEF4EF0AF67F8D71EB409D0E30EAA
:109C7000F76EC60EF66E20EEE6F0F5EC61F008D059
:109C8000E30EF76EB60EF66E20EEE6F0F5EC61F040
:109C900013EC62F0C8D7FCEC5DF0230E9D5D28E06C
:109CA0002A0E9D63C0D71E74A9D750EF4BF0E10E6A
:109CB000F76EA60EF66E20EED6F0F5EC61F0E30E30
:109CC000F76ED60EF66E20EEE6F0F5EC61F0360E8D
:109CD000DF6F13EC62F081B250EF4BF0A0B172EF86
:109CE0004EF0F9D7FCEC5DF0230E9D6362EF51F06E
:109CF000E30EF76EE60EF66E20EED6F0F5EC61F0B0
:109D0000E30EF76EF60EF66E20EEE6F0F5EC61F07F
:109D100013EC62F081B250EF4BF0A0B191EF4EF036
:109D2000F9D7FCEC5DF0230E9D5D05E02A0E9D63E6
:109D3000F1D734EF51F0A26B2EEC59F0E40EF76E30
:109D4000060EF66E20EEE6F0F5EC61F015EE00F092
:109D500001EED2F00A0EA203F350E126F450E22203
:109D6000FF0EE76205D0780EE8CFD2F13C6A22D030
:109D7000080ECB6F200E806FE7380F0B300F816F0E
:109D80003F0E816180C081F03B0E816302D02B0EBB
:109D9000816F81C0EEFFE6500F0B9A6F300F816F1D
:109DA0003F0E816180C081F081C0EEFFCB2FE4D7F0
:109DB000E6CF3CF0100ECB6F11EED2F000EED6F0F5
:109DC000E6CFEEFFCB2FFCD74E0E3CB0590EF16F15
:109DD0004E0E3CB2590EF26F4E0E3CB4590EF36F5C
:109DE0004E0E3CB6590EF46F4E0E3CB8590EF56F40
:109DF000826BA2C083F0832B75EC5DF080C0E7F02E
:109E000081C0E8F013EC62F081B206EF51F0A0B12E
:109E10000BEF4FF0F9D7FCEC5DF0230E9D5D1EE0DB
:109E20002A0E9D5D20E0370E9D5D18E0380E9D5D89
:109E300015E0390E9D5D12E0310E9D5D07E0320E9A
:109E40009D5D04E0330E9D5D01E0DED7A2073F0E6D
:109E5000CB6F400EA261CBC0A2F06ED7A22B400EFA
:109E6000A261A26B69D79E6B640EB06F060EAF6FD6
:109E700081B206EF51F0A0B163EF4FF0AF67F8D7B2
:109E800010EED6F0100ECB6F200EE66ECB2FFDD766
:109E900013EC62F0640EB06F020EAF6F81B206EF8A
:109EA00051F0A0B163EF4FF0AF67F8D711EED2F0E9
:109EB00000EED6F0100ECB6FE6CFEEFFCB2FFCD727
:109EC00013EC62F0D1D7FCEC5DF0230E9D5DD8B4AD
:109ED00050D02A0E9D6312D02EEC59F0780EE8CFA8
:109EE000D2F1100ECB6F11EED2F000EED6F0E6CF2D
:109EF000EEFFCB2FFCD713EC62F0B5D79E6702D0F4
:109F00002EEC59F00F0E9E6120D0010E9E630AD0F8
:109F1000300E9D6307D011EED2F0E76203D09E6B46
:109F20002B0E9D6F11EED2F09E519DC0E3FF00EE0F
:109F3000D6F011EED2F0100ECB6FE6CFEEFFCB2FA6
:109F4000FCD713EC62F09E2B8FD704EC36F02EEC8E
:109F500059F0780EE8CFD2F100EED6F011EED2F043
:109F6000100ECB6FE6CFEEFFCB2FFCD713EC62F0D9
:109F70007AD711EED2F000EED6F0100ECB6FE6CF0E
:109F8000EEFFCB2FFCD713EC62F0640EB06F060E21
:109F9000AF6F81B206EF51F0A0B1E8EF4FF0AF67BD
:109FA000F8D7200EF16F13EC62F0640EB06F020E62
:109FB000AF6F81B206EF51F0A0B1E8EF4FF0AF679D
:109FC000F8D74E0E3CB0590EF16F13EC62F0DDD7AE
:109FD000FCEC5DF02A0E9D6308D03C704E0E3CB048
:109FE000590EF16F13EC62F0D0D7230E9D63CDD7DD
:109FF0004E0E3CB0590EF16F640EB06F060EAF6F8F
:10A0000081B206EF51F0A0B11FEF50F0AF67F8D763
:10A01000200EF26F13EC62F0640EB06F020EAF6FA1
:10A0200081B206EF51F0A0B11FEF50F0AF67F8D743
:10A030004E0E3CB2590EF26F13EC62F0DDD7FCEC21
:10A040005DF02A0E9D6308D03C724E0E3CB2590E54
:10A05000F26F13EC62F0D0D7230E9D63CDD74E0E76
:10A060003CB2590EF26F640EB06F060EAF6F81B244
:10A0700006EF51F0A0B156EF50F0AF67F8D7200EC1
:10A08000F36F13EC62F0640EB06F020EAF6F81B22B
:10A0900006EF51F0A0B156EF50F0AF67F8D74E0E73
:10A0A0003CB4590EF36F13EC62F0DDD7FCEC5DF0BD
:10A0B0002A0E9D6308D03C744E0E3CB4590EF36FCB
:10A0C00013EC62F0D0D7230E9D63CDD74E0E3CB477
:10A0D000590EF36F640EB06F060EAF6F81B206EFCC
:10A0E00051F0A0B18DEF50F0AF67F8D7200EF46FAC
:10A0F00013EC62F0640EB06F020EAF6F81B206EF28
:10A1000051F0A0B18DEF50F0AF67F8D74E0E3CB6CE
:10A11000590EF46F13EC62F0DDD7FCEC5DF02A0E03
:10A120009D6308D03C764E0E3CB6590EF46F13EC8E
:10A1300062F0D0D7230E9D63CDD74E0E3CB6590E9C
:10A14000F46F640EB06F060EAF6F81B206EF51F080
:10A15000A0B1C4EF50F0AF67F8D7200EF56F13EC45
:10A1600062F0640EB06F020EAF6F81B206EF51F075
:10A17000A0B1C4EF50F0AF67F8D74E0E3CB8590EFF
:10A18000F56F13EC62F0DDD7FCEC5DF02A0E9D63F9
:10A1900008D03C784E0E3CB8590EF56F13EC62F0C7
:10A1A000D0D7230E9D63CDD74E0E3CB8590EF56F18
:10A1B00005EE00F011EED2F00A0EA203F350E926EC
:10A1C000F450EA22780EE7620BD0FF0EEE6EEE6ED0
:10A1D000EE6EEE6EEE6EEE6EEE6EEE6EEE6A3ED6EB
:10A1E000080ECB6F11EED2F0200EE764E768E63878
:10A1F000F00B816F200EE764E7680F0EE614811103
:10A20000EE6ECB2FF1D73CC0EEFF28D605EE00F066
:10A2100011EED2F00A0EA203F350E926F450EA221E
:10A22000780EE7620CD0FF0EEE6EEE6EEE6EEE6E06
:10A23000EE6EEE6EEE6EEE6EEE6A50EF4BF0080EC6
:10A24000CB6F200EE764E768E638F00B816F200ED5
:10A25000E764E7680F0EE6148111EE6ECB2FF1D79D
:10A260003CC0EEFF50EF4BF0A26B15EE00F00A0E73
:10A27000A203F350E126F450E222FF0EE75CD8B4CB
:10A280009CEF4EF0A22B3F0EA265EFD7E40EF76EC7
:10A29000160EF66E20EED6F0F5EC61F0E40EF76ED9
:10A2A000260EF66E20EEE6F0F5EC61F013EC62F0AF
:10A2B00004EC36F0640EAE6F140EAD6FAD67FED7D2
:10A2C0009BEF4EF0E10EF76EA60EF66E20EED6F086
:10A2D000F5EC61F0E40EF76E360EF66E20EEE6F069
:10A2E000F5EC61F0370EDF6F13EC62F081B250EFE6
:10A2F0004BF0A0B17DEF51F0F9D7FCEC5DF0230EEF
:10A300009D63CDEF51F0E40EF76E460EF66E20EE33
:10A31000D6F0F5EC61F024BC09D0E40EF76E560ED1
:10A32000F66E20EEE6F0F5EC61F008D0E40EF76E84
:10A33000660EF66E20EEE6F0F5EC61F013EC62F0DE
:10A34000640EAE6F060EAD6F81B259EF4BF0A0B147
:10A35000C3EF51F0AD67F8D7E40EF76E760EF66EE8
:10A3600020EEE6F0F5EC61F013EC62F0640EAE6FF7
:10A37000020EAD6F81B259EF4BF0A0B1C3EF51F0B7
:10A38000AD67F8D7C8D7FCEC5DF02A0E9D6302D00C
:10A39000247CC1D7230E9D63D3D7E10EF76EA60EA2
:10A3A000F66E20EED6F0F5EC61F0E40EF76E860E58
:10A3B000F66E20EEE6F0F5EC61F0380EDF6F13EC90
:10A3C00062F081B250EF4BF0A0B1E8EF51F0F9D755
:10A3D000FCEC5DF0230E9D6359EF4BF0E40EF76E3D
:10A3E000960EF66E20EED6F0F5EC61F01E389A6F00
:10A3F000030E9A17000E9A630AD09A6BE40EF76E5A
:10A40000A60EF66E20EEE6F0F5EC61F017D0010E28
:10A410009A6309D0E40EF76EB60EF66E20EEE6F003
:10A42000F5EC61F00BD0020E9A63E7D7E40EF76EFD
:10A43000C60EF66E20EEE6F0F5EC61F013EC62F07D
:10A44000640EB06F060EAF6F81B259EF4BF0A0B142
:10A450003DEF52F0AF67F8D709EC62F013EC62F011
:10A46000640EB06F020EAF6F81B259EF4BF0A0B126
:10A470003DEF52F0AF67F8D7B9D7FCEC5DF02A0E8C
:10A480009D630AD09A2B030E9A619A6BCF0E1E160B
:10A490009A391E123886AAD7230E9D63D1D7E40EAF
:10A4A000F76ED60EF66E20EED6F0F5EC61F01EAE2D
:10A4B00009D0E40EF76EE60EF66E20EEE6F0F5EC4F
:10A4C00061F008D0E40EF76EF60EF66E20EEE6F0C0
:10A4D000F5EC61F013EC62F0640EB06F060EAF6F36
:10A4E00081B250EF4BF0A0B1A4EF52F0AF67F8D7B4
:10A4F000E50EF76E060EF66E20EEE6F0F5EC61F076
:10A5000013EC62F0640EB06F020EAF6F81B250EFC9
:10A510004BF0A0B1A4EF52F0AF67F8D71EAE09D050
:10A52000E40EF76EE60EF66E20EEE6F0F5EC61F066
:10A5300008D0E40EF76EF60EF66E20EEE6F0F5ECBF
:10A5400061F013EC62F0C8D7FCEC5DF02A0E9D635D
:10A5500002D01E7EACD7230E9D63BED759EF4BF0C1
:10A560001E50030B816F000E816309D0E20EF76E5F
:10A57000160EF66E20EEE6F0F5EC61F01200010E1C
:10A58000816309D0E20EF76E260EF66E20EEE6F03D
:10A59000F5EC61F01200020E816309D0E20EF76E55
:10A5A000360EF66E20EEE6F0F5EC61F01200030ECA
:10A5B000816309D0E20EF76E460EF66E20EEE6F0ED
:10A5C000F5EC61F01200FC0E1E16E20EF76E160E90
:10A5D000F66E20EEE6F0F5EC61F01200640EAE6F60
:10A5E0000F0EAD6FAD67FED781B2ECEF57F0E00E06
:10A5F000F76E060EF66E20EED6F0F5EC61F0E00E8A
:10A60000F76E160EF66E20EEE6F0F5EC61F0310E08
:10A61000DF6F13EC62F081B2CCEF36F0A0B112EF35
:10A6200053F0F9D7FCEC5DF0230E9D6305EF55F078
:10A63000E00EF76EB60EF66E20EED6F0F5EC61F099
:10A64000E00EF76EC60EF66E20EEE6F0F5EC61F069
:10A650008B6B9E6B826B8BC083F0832B75EC5DF0F4
:10A66000200ED76F80C0D8F081C0D9F004EE40F042
:10A67000040E8B03F350E926E86AEA22EF380F0B49
:10A680007A6FEE500F0B7B6FEF380F0B7C6FEE5035
:10A690000F0B7D6FEF380F0B7E6FEE500F0B7F6F40
:10A6A000EF380F0B806FEE500F0B816FAFEC54F053
:10A6B00013EC62F081B285EF54F0A0B161EF53F07A
:10A6C000F9D7FCEC5DF0230E9D6305D08B2B200E9B
:10A6D0008B618B6BBED72A0E9D5D20E0370E9D5D92
:10A6E00018E0380E9D5D15E0390E9D5D12E0310ECB
:10A6F0009D5D07E0320E9D5D04E0330E9D5D01E03F
:10A70000D9D78B071F0ECB6F200E8B61CBC08BF080
:10A71000A0D78B2B200E8B618B6B9BD79E6B640E0F
:10A72000B06F060EAF6F81B2DAEF53F0A0B1B8EFA1
:10A7300053F0AF67F8D7200EE56F13EC62F0640EAC
:10A74000B06F020EAF6F81B2DAEF53F0A0B1B8EF85
:10A7500053F0AF67F8D7480E9A6F0F0E816381C030
:10A760009AF09AC0E5F0300EE52713EC62F0D7D7E7
:10A77000FCEC5DF02A0E9D6307D00F0E816F780E02
:10A78000E56F13EC62F0CAD7230E9D5D13E0300E27
:10A790009D650DD0330E9D610AD00F0E9D15816F02
:10A7A00081C0E5F0300EE52713EC62F0B7D704EC7A
:10A7B00036F0E3D7480E9A6F0F0E816381C09AF08E
:10A7C0009AC0E5F0300EE52713EC62F09E6B640E44
:10A7D000B06F060EAF6F81B285EF54F0A0B10EEFEF
:10A7E00054F0AF67F8D7200EEF6FF06FF16FF26F94
:10A7F000F36FF46FF56F13EC62F0640EB06F020E3E
:10A80000AF6F81B285EF54F0A0B10EEF54F0AF6797
:10A81000F8D7AFEC54F013EC62F0D9D7FCEC5DF054
:10A82000230E9D5D4AE02A0E9D5D0FE19E530DE0D3
:10A830000F0E7A6F7B6F7C6F7D6F7E6F7F6F806F87
:10A84000AFEC54F013EC62F0C1D79E5308E10F0E49
:10A850007A6F7B6F7C6F7D6F7E6F7F6F806F070E6F
:10A860009E611CD0010E9E6309D0300E9D6306D000
:10A87000000E7A6303D09E6B0B0E9D6F0F0E9D171B
:10A8800010EE7AF09E51E126E86AE2229DC0E3FFD5
:10A89000AFEC54F09E2B13EC62F099D704EC36F039
:10A8A0000F0E7A6F7B6F7C6F7D6F7E6F7F6F806F17
:10A8B000AFEC54F013EC62F089D714EE40F0040EC4
:10A8C0008B03F350E126E86AE222200E7A6307D078
:10A8D000FF0EE66EE66EE66EF00EE66EF7D60F0E33
:10A8E0007A177B177C177D177E177F1780178117C4
:10A8F0007A397B11E66E7C397D11E66E7E397F11E7
:10A90000E66E80398111E66EE1D614EE40F0040E59
:10A910008B03F350E126E86AE222780E7A6308D0CE
:10A92000FF0EE66EE66EE66EF00EE66EEEEF52F0AD
:10A930000F0E7A177B177C177D177E177F178017EE
:10A9400081177A397B11E66E7C397D11E66E7E398E
:10A950007F11E66E80398111E66EEEEF52F0480EFF
:10A960009A6F0F0E816381C09AF09AC0E5F00A0ECB
:10A970007A6303D0FA0E9A6F0CD00B0E7A6303D071
:10A98000FB0E9A6F06D0480E9A6F0F0E7A637AC04C
:10A990009AF09AC0EFF0F00E9A6F0F0E7B637BC0B7
:10A9A0009AF09AC0F0F0F00E9A6F0F0E7C637CC0A4
:10A9B0009AF09AC0F1F0F00E9A6F0F0E7D637DC091
:10A9C0009AF09AC0F2F0F00E9A6F0F0E7E637EC07E
:10A9D0009AF09AC0F3F0F00E9A6F0F0E7F637FC06B
:10A9E0009AF09AC0F4F0F00E9A6F0F0E806380C058
:10A9F0009AF09AC0F5F0300EE527EF27F027F127FF
:10AA0000F227F327F427F5271200E00EF76E060E63
:10AA1000F66E20EED6F0F5EC61F0E00EF76E260E45
:10AA2000F66E20EEE6F0F5EC61F0320EDF6F13EC1F
:10AA300062F081B2EEEF52F0A0B120EF55F0F9D7FD
:10AA4000FCEC5DF0230E9D6390EF55F0640EAE6F4D
:10AA5000FA0EAD6FE00EF76ED60EF66E20EED6F063
:10AA6000F5EC61F0E00EF76EE60EF66E20EEE6F025
:10AA7000F5EC61F017C084F059EC5DF010EEE8F0F1
:10AA800080C0E6FF2E0EE66E81C0E6FF13EC62F09A
:10AA9000640EB06F060EAF6F81B28EEF55F0A0B1AD
:10AAA00073EF55F0AF67F8D710EEE8F0200EE66EC2
:10AAB000E66EE66E13EC62F0640EB06F020EAF6FDE
:10AAC00081B28EEF55F0A0B173EF55F0AF67F8D7B4
:10AAD00010EEE8F080C0E6FF2E0EE66E81C0E6FFC5
:10AAE00013EC62F0D5D7FCEC5DF0230E9D5D16E013
:10AAF0002A0E9D6305D0050E846F84C017F0BAD767
:10AB000017C084F0050E8427370E846103D084C0FB
:10AB100017F0B0D7320EE8CF17F0ACD7EEEF52F007
:10AB2000E00EF76E060EF66E20EED6F0F5EC61F054
:10AB3000E00EF76E360EF66E20EEE6F0F5EC61F004
:10AB4000330EDF6F13EC62F081B2EEEF52F0A0B182
:10AB5000ABEF55F0F9D7FCEC5DF0230E9D6356EF9B
:10AB600056F038EC56F024EC56F013EC62F0640E1C
:10AB7000B06F060EAF6F81B222EF56F0A0B1DAEFE0
:10AB800055F0AF67F8D7200EE36FE46FE56F13EC75
:10AB900062F0640EB06F020EAF6F81B222EF56F01A
:10ABA000A0B1DAEF55F0AF67F8D724EC56F013EC0C
:10ABB00062F0DDD7FCEC5DF02A0E9D6302D01674C6
:10ABC000D2D7230E9D63D3D724EC56F0640EB06F1A
:10ABD000060EAF6F81B222EF56F0A0B10DEF56F026
:10ABE000AF67F8D7E00EF76E960EF66E20EEE6F041
:10ABF000F5EC61F013EC62F0640EB06F020EAF6F13
:10AC000081B222EF56F0A0B10DEF56F0AF67F8D742
:10AC100038EC56F013EC62F0D9D7FCEC5DF02A0E5C
:10AC20009D630CD09A2B030E9A171650FC0B9A11A9
:10AC3000166E38EC56F013EC62F0C8D7230E9D6305
:10AC4000C5D78FD7EEEF52F016B409D0E00EF76EED
:10AC5000560EF66E20EED6F0F5EC61F01200E00E26
:10AC6000F76E460EF66E20EED6F0F5EC61F01200AF
:10AC70001650030B9A6F000E9A6309D0E00EF76E20
:10AC8000660EF66E20EEE6F0F5EC61F00ED0010EE9
:10AC90009A6309D0E00EF76E760EF66E20EEE6F0BF
:10ACA000F5EC61F002D09A6BE9D71200E00EF76E76
:10ACB000060EF66E20EED6F0F5EC61F0E00EF76EC3
:10ACC000A60EF66E20EEE6F0F5EC61F0340EDF6FC6
:10ACD00013EC62F081B2EEEF52F0A0B171EF56F0DA
:10ACE000F9D7FCEC5DF0230E9D637FEF57F0E9ECA4
:10ACF00035F0E00EF76EF60EF66E20EED6F0F5ECBF
:10AD000061F018C0A2F0000EA26309D0E10EF76E48
:10AD1000060EF66E20EEE6F0F5EC61F02ED0010E98
:10AD2000A26309D0E10EF76E160EF66E20EEE6F085
:10AD3000F5EC61F022D0020EA26309D0E10EF76EAD
:10AD4000260EF66E20EEE6F0F5EC61F016D0030E5E
:10AD5000A26309D0E10EF76E360EF66E20EEE6F035
:10AD6000F5EC61F00AD0A26B186AE10EF76E060EE0
:10AD7000F66E20EEE6F0F5EC61F013EC62F0640E96
:10AD8000B06F060EAF6F81B27DEF57F0A0B1E5EF67
:10AD900056F0A2511862F3D7AF67F5D710EEEBF07B
:10ADA0000B0ECB6F200EE66ECB2FFDD713EC62F0AF
:10ADB000640EB06F020EAF6F81B27DEF57F0A0B19D
:10ADC000E5EF56F0AF67F8D79ED7FCEC5DF02A0EA2
:10ADD0009D6305D0A22B040EA261A26B94D7230E13
:10ADE0009D6391D7A2C018F0010EA2658CD7020E08
:10ADF000A26309D0E10EF76E260EF66E20EED6F0B5
:10AE0000F5EC61F00BD0030EA26308D0E10EF76EF3
:10AE1000360EF66E20EED6F0F5EC61F0E10EF76E30
:10AE2000460EF66E20EEE6F0F5EC61F0826B19C08E
:10AE300083F075EC5DF09E6B200EF46F300E806336
:10AE400080C0F4F081C0F5F013EC62F0640EB06FD6
:10AE5000060EAF6F81B27DEF57F0A0B14CEF57F007
:10AE6000AF67F8D7200EF46FF56F13EC62F0640E45
:10AE7000B06F020EAF6F81B27DEF57F0A0B14CEF13
:10AE800057F0AF67F8D7300E806380C0F4F081C010
:10AE9000F5F013EC62F0DAD7FCEC5DF0230E9D6365
:10AEA00015D0300E805F815F0A0E8003F3CF19F05A
:10AEB00081511926000E196403D0320E196419D776
:10AEC000300E806F310E816F9E6BB6D72A0E9D6358
:10AED00006D0300E806F310E816F9E6BADD7000EA5
:10AEE0009E6302D0300E816F81C080F09DC081F0E2
:10AEF0009E2B030E9E63A0D7E3D7EEEF52F0E00E39
:10AF0000F76E060EF66E20EED6F0F5EC61F0E10E6F
:10AF1000F76E560EF66E20EEE6F0F5EC61F0350EAB
:10AF2000DF6F13EC62F081B2EEEF52F0A0B19AEF56
:10AF300057F0F9D7FCEC5DF0230E9D63F7EF52F06C
:10AF4000E10EF76E660EF66E20EED6F0F5EC61F0CF
:10AF50000CB809D0E10EF76E760EF66E20EEE6F034
:10AF6000F5EC61F008D0E10EF76E860EF66E20EE7D
:10AF7000E6F0F5EC61F013EC62F0640EAE6F060ED5
:10AF8000AD6F81B2F7EF52F0A0B1E0EF57F0AD67CF
:10AF9000F8D7E10EF76E960EF66E20EEE6F0F5ECC1
:10AFA00061F013EC62F0640EAE6F020EAD6F81B211
:10AFB000F7EF52F0A0B1E0EF57F0AD67F8D7C0D788
:10AFC000FCEC5DF02A0E9D6302D00C78B9D7230EFD
:10AFD0009D63D3D7F7EF52F0640EAE6F0F0EAD6FD7
:10AFE000EC0EF76EC60EF66E20EED6F0F5EC61F0C4
:10AFF000EC0EF76ED60EF66E20EEE6F0F5EC61F094
:10B0000013EC62F0E2EC60F0AD67FED7716B81A2E9
:10B01000D8EF36F0A0EF0FF0A06B916B926B936BB3
:10B02000956B946B966B906BA083A095A09B120080
:10B0300021EC5EF0A0A312000D5009E0A0A706D0FD
:10B04000A08B640EB06F0DC0AFF001D0A09B32A0FA
:10B0500016D0130E926513D0380E926110D092C0A4
:10B0600084F059EC5DF07F51C4EC58F08051C4EC91
:10B0700058F08151C4EC58F00D0EC4EC58F08E51CC
:10B08000060F926105D08E51FA0F926501D008D05B
:10B090008F51060F926112008F51FA0F92651200C4
:10B0A000A0B90BD0A0B705D092C095F0926BA07953
:10B0B000120092C093F0926B1200A0A704D092C02D
:10B0C00094F0926B120092C096F0926B9351945F41
:10B0D000D8A0946D9551965FD8A0966D0A0E946194
:10B0E0000ED096610CD032B083EC58F0902B050E48
:10B0F00090651200A093A099A085906B1200A09972
:10B10000A095906B120093C084F059EC5DF07F51D4
:10B11000C4EC58F08051C4EC58F08151C4EC58F0A4
:10B12000200EC4EC58F095C084F059EC5DF07F51CE
:10B13000C4EC58F08051C4EC58F08151C4EC58F084
:10B14000200EC4EC58F094C084F059EC5DF07F51AF
:10B15000C4EC58F08051C4EC58F08151C4EC58F064
:10B16000200EC4EC58F096C084F059EC5DF07F518D
:10B17000C4EC58F08051C4EC58F08151C4EC58F044
:10B180000D0EC4EC58F0120000000000A4A8FDD77A
:10B190006D6E1200349034A2120038A007D04150D6
:10B1A000E842E842070B9A6F9AC0E6F0A12B030E23
:10B1B000A117000EA16302D03D0E0BD0010EA163BA
:10B1C00002D07E0E06D0020EA16302D07C0E01D00A
:10B1D0007F0E10EEECF0E76E13EC62F012009F6948
:10B1E0002A0E9D6301D01200230E9D6301D0120030
:10B1F000300E9D6303D00A0E9F6F12003A0E9D61C0
:10B2000012009D510F0B9F6F12009DC09BF0300EDE
:10B210009D6302D00A0E1DD02A0E9D6302D00B0E34
:10B2200018D0230E9D6302D00C0E13D0410E9D63E7
:10B2300002D00D0E0ED0420E9D6302D00E0E09D02C
:10B24000430E9D6302D00F0E04D0440E9D6302D0C6
:10B25000000E9B6F9B510F0B1009120001EED2F0F4
:10B26000200E976F200EEE6E972F32EF59F01200DE
:10B27000976F200EE66E972FFCD7120009EE00F0B4
:10B280009A0E976F200EEE6E972FFCD71200F4C126
:10B290009AF0000E9A6309D0EA0EF76E160EF66E5B
:10B2A00020EEE6F0F5EC61F01200010E9A6309D091
:10B2B000EA0EF76E260EF66E20EEE6F0F5EC61F083
:10B2C0001200020E9A6309D0EA0EF76E360EF66E81
:10B2D00020EEE6F0F5EC61F01200030E9A6309D05F
:10B2E000EA0EF76E460EF66E20EEE6F0F5EC61F033
:10B2F0001200040E9A6309D0EA0EF76E560EF66E2F
:10B3000020EEE6F0F5EC61F01200050E9A6309D02C
:10B31000EA0EF76E660EF66E20EEE6F0F5EC61F0E2
:10B320001200060E9A6309D0EA0EF76E760EF66EDC
:10B3300020EEE6F0F5EC61F01200DE0EF76E160E70
:10B34000F66E20EEE6F0F5EC61F0120022EE00F071
:10B350000D0EDF5CD8B41200410EDE6204D0540E34
:10B36000DE6201D0120038BCE6D20000F86AD60EC8
:10B37000686FE40E696F68C0F7FF69C0F6FF22EEE0
:10B3800000F0060E6E6F0900F55006E0F550DE5C29
:10B3900012E16E2FC3EF59F068C0F7FF69C0F6FFE6
:10B3A000060EF626E86AF7220900F5CF6AF0000ECD
:10B3B0006A630DD01200080E6927E86A6823D70E69
:10B3C000685DD9E1AC0E695DD6E16A6B1200010ED1
:10B3D0006A6302D03D801200FF0E6A6302D03D8294
:10B3E00012000E0E6A6302D03E8012000F0E6A63D6
:10B3F00002D03E82120022EE00F02B0EDF6212001D
:10B40000060E6A5DD8A407EF5AF038841200110EB8
:10B410006A5DD8A414EF5AF0ABEC5CF0BFEC5CF0C2
:10B420006FC040F03D821200030E6A5DD8A43DEF6C
:10B430005AF0ABEC5CF0BFEC5CF03DB81200000ED3
:10B440006F6302D059801200010E6F6302D05982DF
:10B450001200020E6F6302D059841200030E6F6354
:10B4600002D059861200040E6F6302D05988120070
:10B47000050E6F631200598A1200020E6A5DD8A48D
:10B4800091EF5AF0ABEC5CF0BFEC5CF03DB8120011
:10B49000000E6F6302D057801200010E6F6302D05E
:10B4A00057821200020E6F6302D057841200030EFF
:10B4B0006F6302D057861200040E6F6302D0578864
:10B4C0001200050E6F6306D0578ABFEC5CF06FC0A8
:10B4D00070F01200060E6F6306D0578CBFEC5CF064
:10B4E0006FC070F01200070E6F6302D0578E12000B
:10B4F000080E6F6302D058801200090E6F6302D0ED
:10B5000058821200000E6F6302D0588412000B0E96
:10B510006F6302D0588612000C0E6F6312005888B9
:10B520001200160E6A5DD8A4BCEF5AF0ABEC5CF0CA
:10B53000B6EC5CF0BFEC5CF03DB81200000E6F633F
:10B5400002D05A801200010E6F6302D05A8212009C
:10B55000020E6F6302D05A841200030E6F6302D092
:10B560005A861200040E6F6302D05A881200050E2C
:10B570006F6312005A8A1200070E6A5DD8A4DAEFD0
:10B580005AF001EE8CF0120EA86F200EEE6EA82F6E
:10B59000C5EF5AF002EE08F011EE8CF0100EA86F15
:10B5A000220EEF5C05E0EECFE6FFA82FD0EF5AF0B9
:10B5B0003D861200100E6A5DD8A4F8EF5AF001EE35
:10B5C0009EF0120EA86F200EEE6EA82FE3EF5AF039
:10B5D00002EE08F011EE9EF0100EA86F220EEF5C46
:10B5E00005E0EECFE6FFA82FEEEF5AF03D84120003
:10B5F000040E6A5DD8A404EF5BF0ABEC5CF0BFEC2A
:10B600005CF06F51416E1200120E6A5DD8A42EEFED
:10B610005BF03D8C02EE07F0520EEF6202D06F6BD2
:10B620001200530EEF6218D002EE0CF0490EEF62DA
:10B6300008D002EE0EF00D0EEF620ED0010E6F6F0D
:10B640001200550EEF6208D002EE0EF00D0EEF6202
:10B6500003D0020E6F6F12006F691200050E6A5D53
:10B66000D8A472EF5BF0ABEC5CF0BFEC5CF0080EC2
:10B67000A86F11EE7CF0200EE66EA82FFCD7020E0C
:10B680006F6314D001EE7CF0550EEE6E6E0EEE6E12
:10B69000520EEE6E650EEE6E670EEE6E690EEE6E7B
:10B6A000730EEE6E2E0EEE6E3D8A120002EE0BF061
:10B6B000220EEF5C09E0050EA86F11EE7CF0EECFD4
:10B6C000E6FFA82FFCD70CD0EE5011EE7CF0080E50
:10B6D000A86F220EEF5C04E0EECFE6FFA82FF9D7AB
:10B6E0003D8A1200080E6A5DD8A486EF5BF0ABECD1
:10B6F0005CF0B6EC5CF0C0EC5CF000EE43F06FC0C8
:10B7000042F06F516FC0EBFF388A12000B0E6A5D7A
:10B71000D8A49DEF5BF0ABEC5CF0B6EC5CF0DE50D7
:10B72000200EA86F08EE32F0220EDF5C04E0DECFC0
:10B73000EEFFA82FF9D7388C12000C0E6A5DD8A442
:10B74000A4EF5BF03F841200130E6A5DD8A4C1EF32
:10B750005BF0ABEC5CF0DE50100EA86F08EE12F060
:10B76000200EEE6EA82FFCD708EE12F0100EA86F78
:10B77000DF500D0804E0DECFEEFFA82FF9D73F869B
:10B780001200140E6A5DD8A4D0EF5BF0ABEC5CF055
:10B79000BFEC5CF03F98000E6F6312003F88120010
:10B7A000150E6A5DD8A47CEF5CF0ABEC5CF009EEA2
:10B7B00000F019EC5CF0DE50B6EC5CF0B6EC5CF03E
:10B7C000B6EC5CF0B6EC5CF0B6EC5CF0F5EC5CF082
:10B7D0002C0EDF621200DE5009EE16F019EC5CF060
:10B7E0000D0EDE5CD8B4120009EE2CF019EC5CF002
:10B7F0000D0EDE5CD8B4120009EE42F019EC5CF0DC
:10B800000D0EDE5CD8B4120009EE58F019EC5CF0B5
:10B810000D0EDE5CD8B4120009EE6EF019EC5CF08F
:10B820000D0EDE5CD8B4120009EE84F019EC5CF069
:10B830001200F5EC5CF0200E7C6F7D6F7E6F7F6FE9
:10B84000806F816F10EE7CF0200E866386C0E6FF6D
:10B85000876387C0E6FF886388C0E6FF896389C085
:10B86000E6FFDE50F5EC5CF0200E866386C0E6FF56
:10B87000876387C0E6FF886388C0E6FF896389C065
:10B88000E6FF7CC0EEFF7DC0EEFF7EC0EEFF7FC016
:10B89000EEFF80C0EEFF81C0EEFFDE50B6EC5CF044
:10B8A000F5EC5CF086C0EEFF87C0EEFF88C0EEFFCF
:10B8B00089C0EEFFDE50F5EC5CF086C0EEFF87C07D
:10B8C000EEFF88C0EEFF89C0EEFFDE50F5EC5CF0C5
:10B8D00086C0EEFF87C0EEFF88C0EEFF89C0EEFF96
:10B8E000DE50F5EC5CF086C0EEFF87C0EEFF88C04E
:10B8F000EEFF89C0EEFF1200170E6A5DD8A48EEF2E
:10B900005CF0ABEC5CF0BFEC5CF06FC0F2F1B6EC5D
:10B910005CF0C0EC5CF06FC0F3F11200180E6A5DD1
:10B92000D8A49AEF5CF0ABEC5CF0BFEC5CF06FC0BD
:10B93000F4F112001200389C780EA86F08EE52F055
:10B9400012EE00F00D0EE75C04E0E6CFEEFFA82F4C
:10B95000F9D7EF6A120022EE00F0800E6E6F3A0EF9
:10B96000DE5C03E06E2FAFEF5CF01200FF0E6E6F37
:10B970002C0EDE5C03E06E2FB8EF5CF01200DE50A0
:10B980003D98300E876F886F896FDECF89F00D0E7E
:10B99000DF5C13E02C0EDF5C10E089C088F0DECFA6
:10B9A00089F00D0EDF5C09E02C0EDF5C06E088C03C
:10B9B00087F089C088F0DECF89F0320E876503D02A
:10B9C0003D88300E876F6F6B300E875F885F895FB1
:10B9D0000A0E8703F3500A0DF3CF6FF00A0E8803A7
:10B9E000F3506F2789516F271200200E866F876FE3
:10B9F000886F896F040EA86F2C0EDF5CD8B412001C
:10BA00000D0EDF5CD8B4120087C086F088C087F0C6
:10BA100089C088F0DECF89F0A82FEED71200846BA2
:10BA2000300E7F5D640DF3CF84F0300E805D0A0D23
:10BA3000F3508427300E815D84271200836B826B64
:10BA4000300E755F765F775F785F795F060E7561A0
:10BA50002DD0000E756507D0100E8327270E822388
:10BA6000752F2CEF5DF0000E766507D0E80E83276A
:10BA7000030E8223762F36EF5DF0000E776507D038
:10BA8000640E8327000E8223772F40EF5DF0000EB7
:10BA9000786507D00A0E8327000E8223782F4AEF9D
:10BAA0005DF079518327E86A8223120082698369F5
:10BAB00012007F6B806B816B630E846506D0640E11
:10BAC000845F02E37F2BFBD78427090E846506D0B1
:10BAD0000A0E845F02E3802BFBD7842784C081F0A9
:10BAE000300E7F278027812712007D6B7E6B7F6B56
:10BAF000806B816B100E835F270E825B02E37D2BD0
:10BB0000F9D7100E8327270E8223E80E835F030EDA
:10BB1000825B02E37E2BF9D7E80E8327030E822394
:10BB2000640E835F000E825B02E37F2BF9D7640E05
:10BB30008327000E82230A0E835F000E825B02E3DE
:10BB4000802BF9D70A0E8327000E822383C081F051
:10BB5000300E7D277E277F27802781271200F5EC76
:10BB60005DF0C06BC16BBF9F1200D9C9E8FF070B26
:10BB7000E8461009CE6F0C0ECF6FD5EC5EF01200C8
:10BB8000DBC9E8FF070BE8461009CE6F0D0ECF6F3B
:10BB9000D5EC5EF01200DDC9E8FF070BE84610099E
:10BBA000CE6F0D0ECF6FD5EC5EF01200DFC9E8FF4F
:10BBB000070BE8461009CE6F0E0ECF6FD5EC5EF086
:10BBC0001200120ECE6F0C0ECF6FD5EC5EF012008D
:10BBD000120ECE6F0F0ECF6FD5EC5EF01200CF6F4E
:10BBE000160ECE6FD5EC5EF01200000ECE6F000E7A
:10BBF000CF6FD5EC5EF01200E9EC5EF0CF510F0B89
:10BC00009D6F9D6703D00F0E9D6F17D0090E9D6528
:10BC100014D00A0E9D6303D0000E9D6F0ED00B0E44
:10BC20009D6303D0FA0E9D6F08D00C0E9D6303D068
:10BC3000F30E9D6F02D00F0E9D6F300E9D27A091C9
:10BC40001200E9EC5EF0CEB5A087CEA5A097A0913A
:10BC50001200110ECE6F800ECF6FD0EC5EF01E0E74
:10BC6000AB6FAB6731EF5EF0110ECE6F000ECF6F92
:10BC7000D0EC5EF0800ED16F000ED26FBFEC5EF0A4
:10BC8000CAC9D1F0CBC9D2F0BFEC5EF0D6C9D1F0B1
:10BC9000D7C9D2F0BFEC5EF0CCC9D1F0CDC9D2F09B
:10BCA000BFEC5EF0D6C9D1F0D7C9D2F0BFEC5EF0E0
:10BCB000CEC9D1F0CFC9D2F0BFEC5EF0D6C9D1F079
:10BCC000D7C9D2F0BFEC5EF0D0C9D1F0D1C9D2F063
:10BCD000BFEC5EF0D6C9D1F0D7C9D2F0BFEC5EF0B0
:10BCE000D2C9D1F0D3C9D2F0BFEC5EF0D6C9D1F041
:10BCF000D7C9D2F0BFEC5EF0D4C9D1F0D5C9D2F02B
:10BD0000BFEC5EF0D6C9D1F0D7C9D2F0BFEC5EF07F
:10BD10001C0ED16F680ED26FBFEC5EF0240ED16F97
:10BD2000A20ED26FBFEC5EF0240ED16FAD0ED26FBB
:10BD3000BFEC5EF0240ED16FA20ED26FBFEC5EF0AE
:10BD4000110ECE6FF3EC5EF012001E0ECE6F010EE0
:10BD5000CF6FDAEC5EF0110ECE6F410ECF6FD0ECEC
:10BD60005EF012001E0ECE6F030ECF6FDAEC5EF0A7
:10BD7000110ECE6F440ECF6FD0EC5EF01200D1C02A
:10BD8000CEF0D2C0CFF0EEEC5EF0020EAB6FAB6740
:10BD9000C7EF5EF01200010ECD6F32EC5FF01200C3
:10BDA000E00ECD6F10EC5FF01200E10ECD6F10ECE5
:10BDB0005FF01200E20ECD6F10EC5FF01200E30EA8
:10BDC000CD6FF8EC5EF01200E50ECD6F03EC5FF086
:10BDD0001200E60ECD6F1FEC5FF01200E80ECD6F83
:10BDE00010EC5FF01200EC0ECD6FF8EC5EF012007C
:10BDF0008498CDC0CCF032EC5FF0CEC0CCF032EC09
:10BE00005FF0848812008498CDC0CCF032EC5FF0F3
:10BE1000000ECC6F32EC5FF0CCC0CEF08488120004
:10BE20008498CDC0CCF032EC5FF0CEC0CCF032ECD8
:10BE30005FF0CFC0CCF032EC5FF0848812008498C1
:10BE4000CDC0CCF032EC5FF0000ECC6F32EC5FF086
:10BE5000CCC0CEF0000ECC6F32EC5FF0CCC0CFF097
:10BE6000848812000000000000000000080ED06F5F
:10BE7000D890CC37D8A08394D8B083848392000024
:10BE800000000000000000000000000000000000B2
:10BE9000838200008350010BCC1300000000D02FE0
:10BEA00038EF5FF01200849C849A100EA36FA6C036
:10BEB000A4F0A7C0A5F0D890A533A433D8A0849E41
:10BEC000D8B0848E0000000000000000848C0000C8
:10BED0000000000000000000000000000000849C42
:10BEE000A32F5BEF5FF000000000000000000000E7
:10BEF000000000000000848A000000000000000034
:10BF00000000000000000000000000000000000031
:10BF10000000000000000000849A1200000E14646B
:10BF2000190C010E1464250C020E1464280C030E67
:10BF30001464320C030E146E320C000E1564190CCE
:10BF4000010E1564250C020E1564280C030E1564F1
:10BF5000320C156A190C240EE8CFD6F9A20EE8CFE0
:10BF6000D7F9D8C9FDF00F0EFD17000EFD630DD0F7
:10BF7000040EE8CFCAF9AB0EE8CFCBF9050EE8CF37
:10BF8000CCF9DE0EE8CFCDF92FD0010EFD630DD038
:10BF9000040EE8CFCAF9AB0EE8CFCBF9060EE8CF16
:10BFA000CCF9000EE8CFCDF91FD0020EFD630DD005
:10BFB000050EE8CFCAF9550EE8CFCBF9050EE8CF4C
:10BFC000CCF9DE0EE8CFCDF90FD0030EFD63D0D74C
:10BFD000050EE8CFCAF9550EE8CFCBF9000EE8CF31
:10BFE000CCF9000EE8CFCDF9DAC9FDF00F0EFD1740
:10BFF000000EFD630DD0060EE8CFCEF9670EE8CF38
:10C00000CFF9080EE8CFD0F9450EE8CFD1F92FD0FF
:10C01000010EFD630DD0050EE8CFCEF9550EE8CF29
:10C02000CFF9000EE8CFD0F9000EE8CFD1F91FD03C
:10C03000020EFD630DD0050EE8CFCEF9AA0EE8CFB3
:10C04000CFF9000EE8CFD0F9000EE8CFD1F90FD02C
:10C05000030EFD63D0D7050EE8CFCEF9550EE8CF1D
:10C06000CFF9000EE8CFD0F9000EE8CFD1F9DEC944
:10C07000FDF00F0EFD17000EFD630DD0050EE8CF8D
:10C08000D2F9DE0EE8CFD3F9060EE8CFD4F9670E69
:10C09000E8CFD5F91200010EFD630DD0050EE8CFF3
:10C0A000D2F9550EE8CFD3F9060EE8CFD4F9000E39
:10C0B000E8CFD5F91200020EFD630DD0050EE8CFD2
:10C0C000D2F9AA0EE8CFD3F9000EE8CFD4F9000ECA
:10C0D000E8CFD5F91200030EFD63D0D7050EE8CFE7
:10C0E000D2F9550EE8CFD3F9000EE8CFD4F9000EFF
:10C0F000E8CFD5F9120000EE0CF0260ECB6F030E40
:10C10000AA6E000EA96ED6EC60F009EED8F0140EFF
:10C11000CB6F030EAA6ECA0EA96ED6EC60F009EEC4
:10C120009AF0280ECB6F030EAA6E260EA96ED6ECDF
:10C1300060F001EE00F07C0ECB6F030EAA6E4E0E87
:10C14000A96ED6EC60F004EE40F0800ECB6F000ECE
:10C15000AA6E000EA96ED6EC60F005EE00F0A00EFF
:10C16000CB6F000EAA6E800EA96ED6EC60F005EEC5
:10C17000A0F0A00ECB6F010EAA6E200EA96ED6EC19
:10C1800060F006EE40F0A00ECB6F010EAA6EC00E5E
:10C19000A96ED6EC60F006EEE0F0A00ECB6F020EBA
:10C1A000AA6E600EA96ED6EC60F01200A69EA69C48
:10C1B000A6800000A8CFEEFFA92AE86AAA22CB2F0A
:10C1C000F7D7120001EE04F0180ECB6F030EAA6E23
:10C1D000520EA96EC6EC61F0FFEC60F00AEC61F063
:10C1E00029EC61F034EC61F053EC61F068EC61F043
:10C1F0007DEC61F092EC61F09DEC61F0120001EEDB
:10C2000000F0040ECB6F030EAA6E4E0EA96EC6ECA4
:10C2100061F0120000EE0CF00A0ECB6F030EAA6E56
:10C22000000EA96EC6EC61F001EE70F00C0ECB6F43
:10C23000030EAA6EBE0EA96EC6EC61F001EE50F0C0
:10C24000100ECB6F030EAA6E9E0EA96EC6EC61F0A7
:10C25000120000EE16F0080ECB6F030EAA6E0A0E47
:10C26000A96EC6EC61F0120000EE1EF0060ECB6F58
:10C27000030EAA6E120EA96EC6EC61F001EE60F01C
:10C28000100ECB6F030EAA6EAE0EA96EC6EC61F057
:10C2900001EE40F0100ECB6F030EAA6E8E0EA96E4B
:10C2A000C6EC61F0120000EE24F00A0ECB6F030E14
:10C2B000AA6E180EA96EC6EC61F009EE9AF0280E6F
:10C2C000CB6F030EAA6E260EA96EC6EC61F01200AB
:10C2D00000EE2EF0010ECB6F030EAA6E220EA96E99
:10C2E000C6EC61F001EE1CF0240ECB6F030EAA6EBB
:10C2F0006A0EA96EC6EC61F0120000EE30F0010E7D
:10C30000CB6F030EAA6E240EA96EC6EC61F009EE87
:10C31000D8F0140ECB6F030EAA6ECA0EA96EC6EC2F
:10C3200061F0120004EE40F0800ECB6F000EAA6E9A
:10C33000000EA96EC6EC61F0120005EE00F0A00E32
:10C34000CB6F000EAA6E800EA96EC6EC61F005EEF2
:10C35000A0F0A00ECB6F010EAA6E200EA96EC6EC47
:10C3600061F006EE40F0A00ECB6F010EAA6EC00E7B
:10C37000A96EC6EC61F006EEE0F0A00ECB6F020EE7
:10C38000AA6E600EA96EC6EC61F01200A69EA69C75
:10C39000A684F29EF29CEECFA8FF550EA76EAA0EC1
:10C3A000A76EA682F28CF28EA6B2D4EF61F0A92A13
:10C3B000E86AAA22CB2FC9EF61F0A694120003EE1F
:10C3C00000F0EE5005E0AD6E00009EA8FED7F9D754
:10C3D0000D0EAD6E00009EA8FED71200F86A09008F
:10C3E000F5500CE0DE6E04D01200F86A100E986F63
:10C3F0000900F55003E0DE6E982FFAD71200100EF8
:10C40000C76F20EED6F0200EDE6EC72F03EF62F06E
:10C410001200100EC76F20EEE6F0200EDE6EC72F62
:10C420000DEF62F01200080E6EEC62F0000E6EEC82
:10C4300062F0100EC76F20EED6F0DE507DEC62F099
:10C44000C72F1DEF62F00C0E6EEC62F0000E6EEC6A
:10C4500062F0100EC76F20EEE6F0DE507DEC62F069
:10C46000C72F2DEF62F01200030E6EEC62F0280E63
:10C47000AB6FAB6739EF62F0030E6EEC62F00A0E41
:10C48000AB6FAB6741EF62F0030E6EEC62F0020E31
:10C490006EEC62F0020E6EEC62F0080E6EEC62F072
:10C4A000000E6EEC62F0080E6EEC62F0000E6EECA8
:10C4B00062F0010E6EEC62F00A0EAB6FAB675EEFDE
:10C4C00062F0000E6EEC62F0060E6EEC62F0000E92
:10C4D0006EEC62F00C0E6EEC62F01200E83AF00BBB
:10C4E000856E8596859485820000000085923C0EBD
:10C4F0009C6F9C2F79EF62F01200C66FF00B856E77
:10C50000858685948582000000008592C639F00BEF
:10C51000856E8586859485820000000085923C0E9C
:10C520009C6F9C2F91EF62F01200F29E040E6EEC55
:10C5300062F0000E6EEC62F0000E7DEC62F0000E18
:10C540007DEC62F0000E7DEC62F0000E7DEC62F09E
:10C55000000E7DEC62F0000E7DEC62F0000E7DECD2
:10C5600062F0180E7DEC62F0000E7DEC62F0000EC1
:10C570007DEC62F0000E7DEC62F0000E7DEC62F06E
:10C58000000E7DEC62F0000E7DEC62F0180E7DEC8A
:10C5900062F0180E7DEC62F0000E7DEC62F0000E91
:10C5A0007DEC62F0000E7DEC62F0000E7DEC62F03E
:10C5B000000E7DEC62F01C0E7DEC62F0180E7DEC3E
:10C5C00062F0180E7DEC62F0000E7DEC62F0000E61
:10C5D0007DEC62F0000E7DEC62F0000E7DEC62F00E
:10C5E0001C0E7DEC62F01C0E7DEC62F0180E7DECF2
:10C5F00062F0180E7DEC62F0000E7DEC62F0000E31
:10C600007DEC62F0000E7DEC62F01E0E7DEC62F0BF
:10C610001C0E7DEC62F01C0E7DEC62F0180E7DECC1
:10C6200062F0180E7DEC62F0000E7DEC62F0000E00
:10C630007DEC62F01E0E7DEC62F01E0E7DEC62F071
:10C640001C0E7DEC62F01C0E7DEC62F0180E7DEC91
:10C6500062F0180E7DEC62F0000E7DEC62F01F0EB1
:10C660007DEC62F01E0E7DEC62F01E0E7DEC62F041
:10C670001C0E7DEC62F01C0E7DEC62F0180E7DEC61
:10C6800062F0180E7DEC62F01F0E7DEC62F01F0E62
:10C690007DEC62F01E0E7DEC62F01E0E7DEC62F011
:10C6A0001C0E7DEC62F01C0E7DEC62F0180E7DEC31
:10C6B00062F0180E7DEC62F0F28E12000AEE00F0CD
:10C6C0000D0EEF6209D00BEE00F03F0EEE6E0D0E78
:10C6D000EE6E64EC6BF01200440EEE6226D04C0E4F
:10C6E000EE6223D0440EEE6220D0FF0ED16FD26FE7
:10C6F00000EED1F0020ECB6F030EAA6EFE0EA96EF5
:10C70000C6EC61F0DB0EF76E960EF66E20EED6F0FC
:10C71000F5EC61F0DB0EF76EA60EF66E20EEE6F09D
:10C72000F5EC61F013EC62F0FF000AEE00F0440E4D
:10C73000EE622BD0420EEE6228D0470EEE6225D07C
:10C74000A0EC68F0080E846180EF68F084C0FBF014
:10C750002C0EEE6280EF68F0A0EC68F0020E8461AF
:10C7600080EF68F00D0EEE6280EF68F0FB2BD89042
:10C7700081698137FB2FFDD7815184A13216E81ED4
:10C7800084B1321248EC6BF012000AEE00F0430E56
:10C79000EE625AD0500EEE6257D0570EEE6254D071
:10C7A000339E00C1E8FFEE6225D001C1E8FFEE62D2
:10C7B00021D002C1E8FFEE621DD003C1E8FFEE62A6
:10C7C00019D00D0EEE6216D0338E48EC6BF0B7EC3C
:10C7D00068F0CFEC68F013EC69F040EC69F074ECB1
:10C7E00069F0C5EC69F0E0EC69F041EC6AF0ADECA1
:10C7F0006AF012000AEE03F0450EEE6280EF68F078
:10C80000750EEE6280EF68F0720EEE6280EF68F0F7
:10C810006F0EEE6280EF68F0740EEE6280EF68F0EB
:10C82000650EEE6280EF68F0630EEE6280EF68F0F6
:10C83000680EEE6280EF68F00D0EEE6280EF68F039
:10C84000338E48EC6BF012000AEE00F0520EEE62EE
:10C850001ED0420EEE621BD0540EEE6218D0DB0EDC
:10C86000F76EB60EF66E20EED6F0F5EC61F0DB0E4C
:10C87000F76EC60EF66E20EEE6F0F5EC61F013EC06
:10C8800062F0E2EC60F000000000AAEF07F00AEEB0
:10C8900000F0500EEE6224D0530EEE6221D0570EFF
:10C8A000EE621ED033AE80EF68F0EECF7EF0EECFBA
:10C8B0007FF0EECF80F0EECF81F00D0EEE6280EFD4
:10C8C00068F001EE00F07EC0EEFF7FC0EEFF80C09A
:10C8D000EEFF81C0EEFFFFEC60F048EC6BF0120061
:10C8E00033AE80EF68F00AEE00F0460EEE62BBD089
:10C8F000580EEE62B8D04F0EEE62B5D0A0EC68F0E4
:10C9000084C000FC2C0EEE6280EF68F0100E1CEE6E
:10C9100001F038EC59F0100EFB6F1CEE01F02C0EFC
:10C92000EF5C04E0EECFE6FFFB2FF9D72C0EEE62B2
:10C9300080EF68F0A0EC68F084C011FC2C0EEE6271
:10C9400080EF68F0A0EC68F084C012FC2C0EEE6260
:10C9500080EF68F0A0EC68F084C013FC2C0EEE624F
:10C9600080EF68F0A0EC68F084C014FC2C0EEE623E
:10C9700080EF68F0A0EC68F084C015FC2C0EEE622D
:10C9800080EF68F0A0EC68F084C016FC2C0EEE621C
:10C9900080EF68F0A0EC68F084C017FC2C0EEE620B
:10C9A000AFD30C0E1CEE18F038EC59F0080EFB6FEC
:10C9B0001CEE18F02C0EEF5C04E0EECFE6FFFB2F30
:10C9C000F9D72C0EEE629CD3040EFB6F1CEE20F008
:10C9D0002C0EEF5C04E0EECFE6FFFB2FF9D72C0E18
:10C9E000EE628ED3A0EC68F084C024FC2C0EEE62C4
:10C9F00087D3A0EC68F084C025FC0D0EEE6280D3D6
:10CA000000CC0CF025CC0DF011CC0EF024CC0FF0A6
:10CA100012CC10F013CC11F014CC12F015CC13F092
:10CA200016CC14F017CC15F00C0EFB6F1CEE18F0A2
:10CA300001EE70F0E6CFEEFFFB2FFCD7100EFB6F80
:10CA40001CEE01F001EE50F0E6CFEEFFFB2FFCD71D
:10CA50000AEC61F048EC6BF08EEC5FF08E6F9DECB1
:10CA60005FF08F6F12000AEE00F0460EEE6253D0B8
:10CA7000580EEE6250D0530EEE624DD0A0EC68F02E
:10CA800084C000FC2C0EEE623BD3A0EC68F084C0A6
:10CA900001FC2C0EEE6234D3A0EC68F084C002FCE2
:10CAA0002C0EEE622DD3A0EC68F084C003FC2C0E9B
:10CAB000EE6226D3A0EC68F084C004FC2C0EEE627B
:10CAC0001FD3A0EC68F084C005FC2C0EEE6218D3D6
:10CAD000A0EC68F084C006FC2C0EEE6211D3A0EC32
:10CAE00068F084C007FC0D0EEE620AD300CC16F08D
:10CAF00006CC18F007CC19F001CC17F002CC1AF0D4
:10CB000003CC1BF004CC1CF005CC1DF029EC61F02B
:10CB100048EC6BF012000AEE00F0470EEE628AD08D
:10CB2000530EEE6287D04D0EEE6284D0A0EC68F01A
:10CB300084C000FC2C0EEE62E3D2100E1CEE01F05D
:10CB400038EC59F0100EFB6F1CEE01F02C0EEF5C70
:10CB500004E0EECFE6FFFB2FF9D72C0EEE62D0D229
:10CB6000A0EC68F084C011FC2C0EEE62C9D2A0ECDF
:10CB700068F084C012FC2C0EEE62C2D2100E1CEEC5
:10CB800013F038EC59F0080EFB6F1CEE13F02C0E6E
:10CB9000EF5C04E0EECFE6FFFB2FF9D72C0EEE6240
:10CBA000AFD2080EFB6F1CEE1BF02C0EEF5C04E006
:10CBB000EECFE6FFFB2FF9D72C0EEE62A1D2A0EC50
:10CBC00068F084C023FC2C0EEE629AD2A0EC68F0D0
:10CBD00084C024FC2C0EEE6293D2A0EC68F084C0DA
:10CBE00025FC0D0EEE628CD200CC1EF011CC22F092
:10CBF00012CC23F023CC20F024CC21F025CC1FF044
:10CC0000100EFB6F1CEE01F001EE60F0E6CFEEFFC0
:10CC1000FB2FFCD7100EFB6F1CEE13F001EE40F063
:10CC2000E6CFEEFFFB2FFCD734EC61F0388648EC02
:10CC30006BF012000AEE00F04E0EEE62BCD0450E14
:10CC4000EE62B9D0540EEE62B6D0A0EC68F084C0AB
:10CC500000FC2C0EEE6254D2A0EC68F084C001FC03
:10CC60002C0EEE624DD283EC68F083C002FC82C0D1
:10CC700003FC2C0EEE6244D22E0E1CEE04F038ECB7
:10CC800059F0060EFB6F1CEE04F02C0EEF5C04E076
:10CC9000EECFE6FFFB2FF9D72C0EEE62060EFB6FF0
:10CCA0001CEE0AF02C0EEF5C04E0EECFE6FFFB2F4B
:10CCB000F9D72C0EEE6224D2060EFB6F1CEE12F09A
:10CCC0002C0EEF5C04E0EECFE6FFFB2FF9D72C0E25
:10CCD000EE6216D283EC68F083C018FC82C019FCA7
:10CCE0002C0EEE620DD2060EFB6F1CEE1AF02C0E0F
:10CCF000EF5C04E0EECFE6FFFB2FF9D72C0EEE62DF
:10CD0000FFD183EC68F083C020FC82C021FC2C0E94
:10CD1000EE62F6D1060EFB6F1CEE22F02C0EEF5CDD
:10CD200004E0EECFE6FFFB2FF9D72C0EEE62E8D140
:10CD300083EC68F083C028FC82C029FC2C0EEE62D4
:10CD4000DFD1060EFB6F1CEE2AF02C0EEF5C04E028
:10CD5000EECFE6FFFB2FF9D72C0EEE62D1D183EC9C
:10CD600068F083C030FC82C031FC0D0EEE62C8D189
:10CD700000CC24F001CC25F002CC26F003CC27F027
:10CD800004CC28F005CC29F006CC2AF007CC2BF0F7
:10CD900008CC2CF009CC2DF0280EFB6F09EE9AF090
:10CDA0001CEE0AF0E6CFEEFFFB2FFCD753EC61F050
:10CDB00048EC6BF012000AEE00F0530EEE623FD02A
:10CDC0004D0EEE623CD0530EEE6239D0A0EC68F00E
:10CDD00084C000FC2C0EEE6293D1240E1CEE01F0F8
:10CDE00038EC59F0100EFB6F1CEE01F02C0EEF5CCE
:10CDF00004E0EECFE6FFFB2FF9D72C0EEE6280D1D8
:10CE0000100EFB6F1CEE13F00D0EEF5C04E0EECF86
:10CE1000E6FFFB2FF9D70D0EEE6272D100CC2EF09B
:10CE2000240EFB6F1CEE01F001EE1CF0E6CFEEFFCE
:10CE3000FB2FFCD768EC61F048EC6BF012000AEEB7
:10CE400000F0500EEE6251D0520EEE624ED0460E01
:10CE5000EE624BD0A0EC68F02C0EEE6251D1210EA8
:10CE600084614ED1000E84654BD1840784C000FCE0
:10CE7000080EFB6F1CEE01F0E668FB2FFDD7070ED6
:10CE8000FB6F1CEE01F02C0EEF5C05E0EE500F0B7B
:10CE9000E66EFB2FF8D72C0EEE6232D1A0EC68F0D4
:10CEA00084C008FC0D0EEE622BD1040EFB6F1CEE4D
:10CEB00001F004EE40F000CCE8FF040DF350E92649
:10CEC000F450EA22E638F00BEF6EE6500F0BEE124C
:10CED000FB2FF8D71F0E006103D048EC6BF0120057
:10CEE00092EC61F048EC6BF012000AEE00F04C0E90
:10CEF000EE6253D0530EEE6250D0540EEE624DD01F
:10CF0000A0EC68F02C0EEE62FBD0410E8461F8D0EC
:10CF1000000E8465F5D0840784C000FC100EFB6F02
:10CF20001CEE01F0E668FB2FFDD7100EFB6F1CEE28
:10CF300001F02C0EEF5C05E0EE500F0BE66EFB2FC0
:10CF4000F8D72C0EEE62DCD0A0EC68F084C011FCA7
:10CF50000D0EEE62D5D0080EFB6F1CEE01F005EE53
:10CF600000F000CCE8FF0A0DF350E926F450EA2265
:10CF7000E638F00BEF6EE6500F0BEE12FB2FF8D7F2
:10CF800011CCEFFF3F0E006103D048EC6BF01200B4
:10CF90009DEC61F048EC6BF012000AEE00F0470ED9
:10CFA000EE62AED0570EEE62ABD0500EEE62A8D05D
:10CFB000A0EC68F084C000FC2C0EEE62A1D0A0ECC6
:10CFC00068F084C001FC2C0EEE629AD0A0EC68F0F0
:10CFD00084C002FC2C0EEE6293D0A0EC68F084C0FA
:10CFE00003FC2C0EEE628CD0A0EC68F084C004FC34
:10CFF0002C0EEE6285D0A0EC68F084C005FC2C0EEF
:10D00000EE627ED0A0EC68F084C006FC2C0EEE62CE
:10D0100077D0A0EC68F084C007FC2C0EEE6270D0D4
:10D02000A0EC68F084C008FC2C0EEE6269D0A0EC85
:10D0300068F084C009FC2C0EEE6262D0A0EC68F0AF
:10D0400084C00AFC2C0EEE625BD0A0EC68F084C0B9
:10D050000BFC2C0EEE6254D0A0EC68F084C00CFCEB
:10D060002C0EEE624DD0A0EC68F084C00DFC2C0EAE
:10D07000EE6246D0A0EC68F084C00EFC2C0EEE628E
:10D080003FD0A0EC68F084C00FFC2C0EEE6238D0CC
:10D09000A0EC68F084C010FC2C0EEE6231D0A0EC45
:10D0A00068F084C011FC2C0EEE622AD0A0EC68F06F
:10D0B00084C012FC2C0EEE6223D0A0EC68F084C079
:10D0C00013FC2C0EEE621CD0A0EC68F084C014FCA3
:10D0D0000D0EEE6215D000CC30F0140EFB6F1CEE7E
:10D0E00001F009EED8F0E6CFEEFFFB2FFCD77DEC88
:10D0F00061F048EC6BF0ABEC5FF029EC5EF01200F5
:10D1000053EC6BF01200300E756F766F776F786F9F
:10D11000796F050E976F2C0EEF5C0FE00D0EEF5C34
:10D120000CE076C075F077C076F078C077F079C003
:10D1300078F0EECF79F0972FEED71EEC5DF012006D
:10D14000300E7F6F806F816F030E976F2C0EEF5C38
:10D150000BE00D0EEF5C08E080C07FF081C080F036
:10D16000EECF81F0972FF2D70FEC5DF01200F50EA5
:10D17000F76E340EF66E0BEE00F0560EEE6E450EA8
:10D18000EE6E520EEE6E100EFA6F0900F5CFEEFF46
:10D19000FA2FFBD70D0EEE6E64EC6BF012000BEE67
:10D1A00000F0460EEE6E580EEE6E4F0EEE6E0CC098
:10D1B00084F013EC6BF011EE50F0100E3BEC6BF0C2
:10D1C0000EC084F011EC6BF010C084F011EC6BF029
:10D1D00011C084F011EC6BF012C084F011EC6BF014
:10D1E00013C084F011EC6BF014C084F011EC6BF000
:10D1F00015C084F011EC6BF011EE70F0080E3BECF2
:10D200006BF011EE78F0040E3BEC6BF00FC084F085
:10D2100011EC6BF00DC084F011EC6BF00D0EEE6EA6
:10D2200064EC6BF012000BEE00F0460EEE6E580E42
:10D23000EE6E530EEE6E16C084F013EC6BF017C05A
:10D2400084F011EC6BF01AC084F011EC6BF01BC091
:10D2500084F011EC6BF01CC084F011EC6BF01DC07D
:10D2600084F011EC6BF018C084F011EC6BF019C075
:10D2700084F011EC6BF00D0EEE6E64EC6BF01200AE
:10D280000BEE00F0470EEE6E530EEE6E4D0EEE6E90
:10D290001EC084F013EC6BF011EE60F0100E3BEC4E
:10D2A0006BF022C084F011EC6BF023C084F011EC21
:10D2B0006BF011EE40F0080E3BEC6BF011EE48F015
:10D2C000080E3BEC6BF020C084F011EC6BF021C039
:10D2D00084F011EC6BF01FC084F011EC6BF00D0EBC
:10D2E000EE6E64EC6BF012000BEE00F04E0EEE6E84
:10D2F000450EEE6E540EEE6E24C084F013EC6BF00F
:10D3000025C084F011EC6BF026C083F027C082F0BA
:10D3100022EC6BF0060E10EE28F03BEC6BF019EEF1
:10D320009AF0060E3BEC6BF019EEA2F0060E3BEC09
:10D330006BF0A8C983F0A9C982F022EC6BF019EE5A
:10D34000AAF0060E3BEC6BF0B0C983F0B1C982F0D5
:10D3500022EC6BF019EEB2F0060E3BEC6BF0B8C9A4
:10D3600083F0B9C982F022EC6BF019EEBAF0060E28
:10D370003BEC6BF0C0C983F0C1C982F022EC6BF0CA
:10D380000D0EEE6E64EC6BF012000BEE00F0530E1F
:10D39000EE6E4D0EEE6E530EEE6E2EC084F013EC5C
:10D3A0006BF011EE1CF0100E3BEC6BF011EE2EF05A
:10D3B000100E3BEC6BF00D0EEE6E64EC6BF0120099
:10D3C0000BEE00F0470EEE6E570EEE6E500EEE6E48
:10D3D00030C084F013EC6BF0D8C984F011EC6BF022
:10D3E000D9C984F011EC6BF0DAC984F011EC6BF060
:10D3F000DBC984F011EC6BF0DCC984F011EC6BF04C
:10D40000DDC984F011EC6BF0DEC984F011EC6BF037
:10D41000DFC984F011EC6BF0E0C984F011EC6BF023
:10D42000E1C984F011EC6BF0E2C984F011EC6BF00F
:10D43000E3C984F011EC6BF0E4C984F011EC6BF0FB
:10D44000E5C984F011EC6BF0E6C984F011EC6BF0E7
:10D45000E7C984F011EC6BF0E8C984F011EC6BF0D3
:10D46000E9C984F011EC6BF0EAC984F011EC6BF0BF
:10D47000EBC984F011EC6BF00D0EEE6E64EC6BF00A
:10D480001200200EFC6F14EE40F00BEE00F0500E78
:10D49000EE6E520EEE6E460EEE6ED880210EFC55EC
:10D4A000846F59EC5DF080C0EEFF81C0EEFF2C0E62
:10D4B000EE6EE7380F0B7A6F0A0E7A6302D02A0EEF
:10D4C00007D00B0E7A6302D02B0E02D0300E7A25D5
:10D4D0007A6FE6500F0B300F7B6FE7380F0B300F72
:10D4E0007C6FE6500F0B300F7D6FE7380F0B300F5E
:10D4F0007E6FE6500F0B300F7F6FE7380F0B300F4A
:10D50000806FE6500F0B300F816F3A0E7A611AD0A0
:10D510007AC0EEFF7B6116D07BC0EEFF7C6112D03B
:10D520007CC0EEFF7D610ED07DC0EEFF7E610AD033
:10D530007EC0EEFF7F6106D07FC0EEFF806102D02B
:10D5400080C0EEFF2C0EEE6E81C0EEFF0D0EEE6E73
:10D5500064EC6BF0FC2F99D71200400EFC6F15EEB7
:10D5600000F00BEE00F04C0EEE6E530EEE6E540E0D
:10D57000EE6ED880410EFC55846F59EC5DF080C092
:10D58000EEFF81C0EEFF2C0EEE6EE6CF7AF0E6CF16
:10D590007BF0E6CF7CF0E6CF7DF0E6CF7EF0E6CF05
:10D5A0007FF0E6CF80F0E6CF81F0E6CF79F0E6506D
:10D5B0007A390F0B300FFD6F3C0EFD6127D03B0E0B
:10D5C000FD5DD8B4FD99FDC0EEFF7A510F0B300F11
:10D5D0007A6F3A0E7A611AD07AC0EEFF070EFB6FAF
:10D5E00020EE7BF0DF380F0B300FFD6F3A0EFD6140
:10D5F0000DD0FDC0EEFFDE500F0B300FFD6F3A0E69
:10D60000FD6104D0FDC0EEFFFB2FECD779C084F0A4
:10D6100011EC6BF00D0EEE6E64EC6BF0FC2FA1D7ED
:10D6200012002C0EEE6E59EC5DF0300E7F6303D0CD
:10D63000806303D004D07FC0EEFF80C0EEFF81C0C6
:10D64000EEFF12002C0EEE6E75EC5DF0300E7D6379
:10D6500007D07E6307D07F6307D0806307D008D0F0
:10D660007DC0EEFF7EC0EEFF7FC0EEFF80C0EEFF0C
:10D6700081C0EEFF1200FA6F2C0EEE6E01D0FA6F31
:10D68000200EE75C04E0E6CFEEFFFA2FF9D7120098
:10D690000BEE00F04F0EEE6E4B0EEE6E0D0EEE6EBC
:10D6A00064EC6BF012000BEE00F0450EEE6E520EC5
:10D6B000EE6E520EEE6E4F0EEE6E520EEE6E0D0EC2
:10D6C000EE6E64EC6BF01200EF6AF96B0BEE00F09B
:10D6D000A4A8FED7EE5003E06D6EF92FF9D7A4A8E9
:10D6E000FED7120041540000000000004F4B000024
:10D6F000000001002B57494E443A02002B4352458B
:10D70000473A03002B4353513A2004002B434F5018
:10D71000533A05002B4352494E4706002B434C49D0
:10D72000503A07002B434D54493A08002B434D47CC
:10D73000573A09002B434D53533A0A002B434D47A8
:10D74000523A0B002B434D47533A0C004E4F2041A9
:10D750004E530E004255535900000F002B434357C0
:10D76000413A10002B434D45000011002B43504916
:10D770004E3A12004552524F5200FF002B57494D6E
:10D78000454913002B5744574C3A14002B4343454B
:10D79000443A15002B4343454C4C16002B57565228
:10D7A0003A2017002B574D42533A18000000000052
:10D7B0000000000041540000415445310000415434
:10D7C0004800000041544100000041542B434D45A6
:10D7D000453D3100000041542B434C49503D310040
:10D7E000000041542B434C49503D3000000041544F
:10D7F0002B434C49523D3000000041542B434C49CF
:10D80000523D3100000041542B434C49523D3200FF
:10D81000000041542B4950523D3936303000000051
:10D8200041542B4950523D3139323030000041547F
:10D830002B4946433D302C30000041542B57535662
:10D84000473D3100000041542B57494E443D313093
:10D850003233000041542B57494E443D3F000000F5
:10D8600041542B43474D5200000041542B5744571D
:10D870004C00000041542B57494D45493F000000E2
:10D8800041542B434345443D302C33000000415468
:10D890002B4343454C4C3D30000041542B434655EF
:10D8A0004E3D3100000041542B574344503D310060
:10D8B000000041542B435245473D30000000415485
:10D8C0002B435245473D3100000041542B43524504
:10D8D000473D3200000041542B434345443D312C29
:10D8E0003800000041542B4352433D310000415465
:10D8F0002B434943423D320000004154265700006B
:10D9000041542B434F50533D3000000041542B43B2
:10D910004F50533D3200000041542B434F50533D74
:10D92000332C3000000041542B434F50533D332CD7
:10D930003100000041542B434F50533F00004154ED
:10D940002B4343494400000041542B43494D4900B7
:10D95000000041542B434E554D00000041542B43D1
:10D960004C49523D3000000041542B434C49523F3A
:10D97000000041542B434357413D312C312C3100A1
:10D98000000041542B4350494E3F000041542B5757
:10D9900056523F00000041542B574D42533F000068
:10D9A00041542B434D45523D2C30000041542B45F2
:10D9B00043484F3D312C332C33302C383030302C11
:10D9C00032353000000041542B53494445543D3119
:10D9D0002C33000041542B535045414B45523D30B0
:10D9E000000041542B57464D3D312C33330000008D
:10D9F00041542B5647543D30000041542B56475458
:10DA00003D343000000041542B5647523D3634001F
:10DA1000000041542B4543484F3D312C362C3330C8
:10DA20002C35302C36342C3230302C3535302C31EE
:10DA3000352C33323736372C353030302C323734C2
:10DA400038342C33383639372C373331312C3400D5
:10DA5000000041542B53494445543D30000041548B
:10DA60002B535045414B45523D30000041542B57FC
:10DA7000464D3D312C333300000041542B45434883
:10DA80004F3D312C332C33302C383030302C323564
:10DA90003600000041542B53494445543D312C334A
:10DAA000000041542B535045414B45523D3100003D
:10DAB00041542B57464D3D312C3333000000415427
:10DAC0002B43534D533D3000000041542B434D47F1
:10DAD000463D3100000041542B434E4D493D322C10
:10DAE000312C302C302C3000000041542B434D475A
:10DAF000443D000041542B434D47443D312C3400FC
:10DB0000000041542B434D47523D000041542B43EC
:10DB10004D53533D000041542B434D47573D0000AA
:10DB200041542B434D47533D000041542B43484C37
:10DB3000443D3100000041542B43484C443D3200E9
:10DB4000000041542B43484C443D313100004154C6
:10DB50002B43484C443D3132000041542B43484C48
:10DB6000443D330000002A20474154455741592085
:10DB700047534D20202A4C6F6164657220506173B9
:10DB800073776F726420436F64653A2020202020F1
:10DB900020202020202047617465776179206973F7
:10DBA000207265616479746F207468652075706493
:10DBB0006174696E6721536176696E672050617286
:10DBC000616D657465722052657374617274696EFB
:10DBD00067204757202047534D3A202D506F7765D7
:10DBE00072204F4E2D204E6574776F726B3A202055
:10DBF00020202020202053494D783A204175746F11
:10DC00006D617469632053494D783A20204D616EEF
:10DC100075616C2020204552524F523A20204D6FA2
:10DC200064756C6520202020206E6F7420616E73F7
:10DC30007765722020204552524F523A20202020F2
:10DC4000202020202020415420436F6D6D616E64A0
:10DC5000206661696C2E20202053494D202063618D
:10DC6000726420202020206973206E6F74207072EF
:10DC70006573656E742020207761732072656D6F07
:10DC8000766564202020202077617320696E73659B
:10DC900072746564202020202020496E73657274A0
:10DCA000202020202020496E736572742053494D36
:10DCB0002020636172644E6574776F726B207761A8
:10DCC00073206C6F737447534D3A202020202D49E8
:10DCD0006E69742D2020204E6574776F726B2064FE
:10DCE000656E69656420204368616E6765207468AD
:10DCF000652053494D202053494D20756E6B6E6F42
:10DD0000776E202020204E6574776F726B206973C8
:10DD100020666F756E642020204E6574776F726B7D
:10DD200020202020202020776173206E6F742066D1
:10DD30006F756E642020526F616D696E6720697324
:10DD400020666F756E644E6574776F726B3A2075DE
:10DD50006E6B6E6F776E4E6574776F726B3A2020C4
:10DD600020202020202053494D783A205365747498
:10DD7000696E67202020204D616E75616C205365AF
:10DD80006C65637420204E6574776F726B3A202047
:10DD90002020202020204E6574776F726B3A20205F
:10DDA000202020202020202069732073656C65636B
:10DDB00074656420202020206E6F7420616C6C6F6D
:10DDC00077656420202020436F6465206F66204EB5
:10DDD0006574776F726B2020697320616473656E60
:10DDE000742E20202020204E6574776F726B732074
:10DDF000636F6465732020206172652061627365C2
:10DE00006E7420202020566F69636520524154456E
:10DE10003A78782C787820202047534D2042616E44
:10DE200064203F20202020456E746572205061736D
:10DE300073776F726420496E76616C6964205061FB
:10DE40007373776F72645374657020323A20436F36
:10DE50006D6D616E6420202020697320696E76618B
:10DE60006C69642E20204469616C3A204658532026
:10DE7000506F7274202052696E673A2020204753F9
:10DE80004D2E53494D314469616C3A20202047534F
:10DE90004D2E53494D3143616C6C3A20202047533D
:10DEA0004D2E53494D31576169743A202020475314
:10DEB0004D2E53494D3154616C6B3A20202047530D
:10DEC0004D2E53494D31202047534D204469616CFC
:10DED000696E67202020204469726563742044695C
:10DEE000616C696E672E204F6E6C7920546F6E6581
:10DEF000204469616C2E2020202050524956415404
:10DF0000452020202020434944206973206E6F74EF
:10DF100020666F756E644469616C3A2046584F20E4
:10DF2000506F7274202054616C6B3A2046584F2019
:10DF3000506F727420204469616C3A20464F4C4CFB
:10DF40004F57204D452054616C6B3A20464F4C4C46
:10DF50004F57204D45204469616C3A6E6F742073B1
:10DF60007570706F727420205245504C4143494E79
:10DF7000472053494D2053494D313A206C6F61641D
:10DF8000696E6720202053494D323A206C6F6164DE
:10DF9000696E672020204572726F72206F66205272
:10DFA00065616464722E4D656E75202320782E3075
:10DFB00020202020202020202046585320504F523F
:10DFC00054202020202020202047534D204E45540F
:10DFD000574F524B202020202046584F20504F5260
:10DFE0005420202020202020202047415445574104
:10DFF00059202020202020534D5320504152414D84
:10E000004554455253204D656E75202320312E789E
:10E010002020202020205072656669786573206674
:10E020006F722047534D2020204449414C205041DD
:10E030005553452020202047656E65726174696FD5
:10E040006E20434C492047656E65726174696F6E3E
:10E050003A20204F4E2047656E65726174696F6E7D
:10E060003A20204F4646434C493A202042656C6C8A
:10E07000636F72652020434C493A204254204F6E12
:10E080002D686F6F6B20434C493A20562E32332057
:10E09000202020202020434C493A202020202020EE
:10E0A0002020202020205245564552534520504FD5
:10E0B0004C4152495459237878782020666F722059
:10E0C00053494D3A207820507265666978203A7835
:10E0D000787878787878204469616C6C696E67200C
:10E0E0005061757365202020782E78207365636FEA
:10E0F0006E64732020205265766572736520506FC0
:10E100006C6172697479547970653A2044697361FD
:10E11000626C65202020547970653A4261742E52F9
:10E12000657665727365547970653A44626C2E52F7
:10E1300065762E506F6C547970653A427265616BEA
:10E14000204C696E65203130306D73207820546921
:10E150006D653A20202052494E474241434B20549E
:10E160004F4E45202020202052696E674261636B2C
:10E1700020746F6E652020746F6E65203A202064D5
:10E18000697361626C6520746F6E65203A2020208F
:10E19000656E61626C6520746F6E65203A20202088
:10E1A0002020202020204D656E75202320322E78DF
:10E1B00020202020202020554E4C495354454420F7
:10E1C00043414C4C202020556E6C6973746564206B
:10E1D00043616C6C202020416363657074202D20A6
:10E1E000656E61626C6520416363657074202D64A7
:10E1F000697361626C6520416363657074202D20D2
:10E2000020202020202047534D2041434345535395
:10E21000204D4F44453A4469726563746C792074AB
:10E220006F20465853204469726563746C7920747A
:10E230006F2046584F2047534D2F46584F2043617B
:10E240006C6C4261636B2047534D20436F6E666573
:10E2500072656E6365202020202020202020202051
:10E260002020202020204175746F6469616C206E2D
:10E27000756D6265722020205245504541542043FF
:10E28000414C4C2020205265706561742063616CA4
:10E290006C2046584F2066726F6D2047534D3A20D0
:10E2A000656E61626C6566726F6D2047534D3A64AE
:10E2B000697361626C6520202043414C4C424143AC
:10E2C0004B20202020202043414C4C4241434B20F6
:10E2D00053455455502043616C6C6261636B3A65E1
:10E2E0006E61626C652043616C6C6261636B3A6461
:10E2F000697361626C6543616C6C6261636B3A2047
:10E3000020202020202043414C4C4241434B207789
:10E31000696C6C2062657669613A20202047534D14
:10E320002020202020207669613A20202046584F66
:10E330002020202020207669613A202020202020E3
:10E340002020202020202041646465642043414C2B
:10E350004C4241434B2076696120534D53203A642F
:10E36000697361626C6576696120534D53203A2070
:10E37000656E61626C6576696120534D53203A2069
:10E3800020202020202020414343455353207669FC
:10E3900061204C495354204163636573732076694F
:10E3A00061204C697374766961204C4953543A205A
:10E3B000202020202020766961204C4953543A20A7
:10E3C000656E61626C65766961204C4953543A64AC
:10E3D000697361626C6547534D204E554D424552FD
:10E3E00053204C49535447534D204E756D6265720E
:10E3F00073204C6973746B65793A2A2D4164642CDF
:10E40000232D456469742378783A53544154453D2B
:10E410002030303030304D61782E20616D6F756E58
:10E4200074206F662020746865206E756D62657259
:10E4300073203D2036342052494E474241434B2001
:10E44000544F4E4520202052696E674261636B2015
:10E45000546F6E65202066726F6D2047534D3A648D
:10E46000697361626C6566726F6D2047534D3A65E2
:10E470006E61626C652066726F6D2047534D3A2065
:10E48000202020202020434C495220616E642050DF
:10E4900052495641544520204D79204E756D626594
:10E4A000723A2020202020736574206279204E6506
:10E4B00074776F726B202064697361626C6564208D
:10E4C0006E756D6265722020656E61626C65642098
:10E4D0006E756D62657250726976617465206361F4
:10E4E0006C6C20746F204C6F63616C204C6E3A65CD
:10E4F0006E61626C65204C6F63616C204C6E3A6497
:10E50000697361626C654C6F63616C204C6E3A207C
:10E51000202020202020204E45542F43454C4C20C5
:10E5200053454C454354204E4554574F524B20536E
:10E53000454C454354202020204175746F2053657D
:10E540006C656374202020506572696F6469632074
:10E5500053656C65637478204E6574776F726B3A9F
:10E56000202020202020506572696F642F7365631E
:10E570003A2020202020204D616E75616C2053656B
:10E580006C6563742020204D616E75616C2053654D
:10E590006C65637420204E6574776F726B3A20202F
:10E5A000202020202020202043454C4C2053454C47
:10E5B00045435420202043656C6C2053656C656393
:10E5C000742066726F6D4E6574776F726B3A20209F
:10E5D0002020202020202020204175746F205365AA
:10E5E0006C656374202020506572696F64696320D4
:10E5F00053656C6563745072643D78787878782CD4
:10E6000052783D787878204D616E75616C20536545
:10E610006C65637420204552524F523A20202020CE
:10E62000202020202020202043656C6C2053656C26
:10E630006563742020207820434C3A787878782CD1
:10E6400052783A7878784E3A7878787878782C4397
:10E65000483A787878782053656C656374656420EF
:10E6600043656C6C20206973206E6F742061766145
:10E67000696C61626C6557616974696E673A2020E4
:10E68000202020202020202043656C6C2053656CC6
:10E690006563742020202053656C65637465642075
:10E6A00043656C6C202020202020776173207365E7
:10E6B000742E202020204D656E75202320332E7867
:10E6C0002020202020202046584F204143434553FE
:10E6D00053204D4F444546584F2041636365737343
:10E6E000204D6F64653A4469726563746C79207477
:10E6F0006F20465853204469726563746C792074A6
:10E700006F2047534D202027464F4C4C4F57204DEC
:10E7100045272020202020202020202020202020CD
:10E720002020202020202047534D2053656C656316
:10E7300074696F6E20206279205072656669786511
:10E74000733A20594553627920507265666978653D
:10E75000733A20204E4F20202020546F20546573A0
:10E760007420202020204E756D626572204C6973E4
:10E77000743A205945534E756D626572204C697329
:10E78000743A20204E4F202027464F4C4C4F5720A4
:10E790004D4527202020202027466F6C6C6F772066
:10E7A0004D65272020202752696E677327204E75FC
:10E7B0006D6265723A20466F6C6C6F77204D6527ED
:10E7C0004E756D62657220204449414C494E472088
:10E7D0004D4F44452020204D696E2E204469616CC8
:10E7E0006C696E672020204469676974733A202041
:10E7F000202020207878204D61782E204469616C9B
:10E800006C696E672020204469676974733A202020
:10E81000202020207878204469616C6C696E672024
:10E820005061757365202020782E78207365636FA2
:10E830006E64732020202054696D652057616974CF
:10E84000696E67206F666469616C6C696E672873B6
:10E850006563293A7878205053544E2F4578742EAA
:10E86000204C696E65204469616C696E6720203AAE
:10E8700020546F6E65204469616C696E6720203A90
:10E880002050756C7365202020436F756E7472790B
:10E8900020202020202020436F646520203A202063
:10E8A0002020202020204E6174696F6E616C20440E
:10E8B0006972656374204469616C696E672F4E44A8
:10E8C000443A20202020506175736520616674658C
:10E8D00072206469616C204E4444202831207365A5
:10E8E00063202A293A205053544E2F4578742E4CD9
:10E8F00020546F6E657320204275737920546F6EBB
:10E90000653A202020204F4E2F4F46463A20353082
:10E9100030206D7365632052656F72646572205498
:10E920006F6E653A20204F4E2F4F46463A203235C3
:10E9300030206D7365632052494E4720504152414B
:10E940004D45544552532052696E67204672657199
:10E9500075656E63792020202020202020203A2019
:10E9600078787820487A4D656E75202320342E788B
:10E9700020202020202020204761696E20436F6ED8
:10E9800074726F6C2020537065616B65722020205B
:10E99000203A202D78204D6963726F70686F6E6524
:10E9A000203A202B7820566F696365205261746588
:10E9B0002054797065204F757420436F64696E67C9
:10E9C00020203A202020496E20436F64696E672022
:10E9D00020203A202020205468697320566F6963F4
:10E9E0006520526174652020206E6F7420737570ED
:10E9F000706F72742E2020202047534D2042616E8C
:10EA00006420202020204672657175656E63792030
:10EA100042616E643A204D6F6E6F3A20202020389C
:10EA20003530204D487A4D6F6E6F3A2020203930B6
:10EA30003045204D487A4D6F6E6F3A202020313896
:10EA40003030204D487A4D6F6E6F3A20202031399A
:10EA50003030204D487A4475616C3A3835302F316A
:10EA60003930304D487A4475616C3A3930302F3145
:10EA70003830304D487A4475616C3A3930302F3136
:10EA80003930304D487A47534D206E6F742073757E
:10EA900070706F7274206120737065636966696558
:10EAA000642062616E6453455454494E472050417E
:10EAB0005353574F524420456E746572206E6577EC
:10EAC00020505357202053455454494E4720504915
:10EAD0004E20434F44452020202053657474696EB6
:10EAE00067202020202050494E20434F4445206677
:10EAF0006F722053494D20202020555044415449E5
:10EB00004E47202020204D6F64756C6520494420BD
:10EB1000284D494429204368616E67696E67204D1E
:10EB20004944202020202020202077617320666126
:10EB3000696C65642021202043757272656E7420B3
:10EB40004D49442020204552524F523A2020202047
:10EB500020202020202052656164696E67206F6646
:10EB6000204D494421204368616E67696E67206FBC
:10EB700066204D494420636F6E6669726D3A2020AD
:10EB8000202020202020456E746572206E6577203D
:10EB90004D49443A20204D49442073686F756C6498
:10EBA0002068617665206F662031342F313520640E
:10EBB00069676974732E2053657474696E67206F7A
:10EBC00066204D4944204368616E67696E67206F17
:10EBD00066204D4944202077617320636F6D706C0F
:10EBE000657465642021436F6E6669726D20746878
:10EBF00065206F6C64204D4944205053573A2020C3
:10EC000020202020202020456E74657220746865C5
:10EC1000206E657720204D4944205053573A2020DC
:10EC200020202020202020204E6577204D494420A0
:10EC30005053572020202020207761732073657463
:10EC4000212020202020456E7465726564204D4986
:10EC500044205053572020697320494E56414C4957
:10EC6000442021212120456E7465726564206E6503
:10EC70007720505357202077617320756E636F7231
:10EC8000726563742E20524F5554455220574F528F
:10EC90004B204D4F444520576F726B204D6F64657C
:10ECA0003A20202020202020566F696365204D6F78
:10ECB00064652020202020202044617461204D6F55
:10ECC0006465202020202020536176696E67202013
:10ECD000202020202020202020504152414D45540A
:10ECE000455253202020202047534D207C2054653E
:10ECF0006C2E4C696E6520206E6F74207072657387
:10ED0000656E7420202020496E636F6D696E6720E8
:10ED100043616C6C20202020746F2046584F205097
:10ED20006F72742E202046584F3A2020496E636F30
:10ED30006D696E67202052696E673A4E6574776F11
:10ED4000726B2047534D205053544E2F465853203A
:10ED50006973206E6F74636F6E6E65637465642093
:10ED6000746F2046584F205053544E2F465853200E
:10ED7000206973202020636F6E6E65637465642064
:10ED8000746F2046584F466F6C6C6F77204D652727
:10ED90004E756D626572206973206E6F742070729B
:10EDA0006573656E74212066726F6D20465853201E
:10EDB000506F727420202066726F6D2046584F206D
:10EDC000506F7274202020446973636F6E6E6563A8
:10EDD00074696F6E20202066726F6D2043454C4C25
:10EDE000554C4152202046584F2043616C6C207492
:10EDF0006F2047534D204175746F6469616C2074B6
:10EE00006F2046584F202046584F2F204578742EAB
:10EE1000204C696E652077617320646973636F6E3F
:10EE20006E656374656443616C6C4261636B2076EC
:10EE300069612046584F2047534D206E6F74206102
:10EE40006E7377657220202047534D20496E636FA3
:10EE50006D696E6720202063616C6C207761732080
:10EE600064656E696564436C6261636B3A20475305
:10EE70004D2E53494D782053494D20697320626CC3
:10EE80006F636B65642E53494D2050494E20726567
:10EE900071756972656453657474696E6720504951
:10EEA0004E2053494D7850494E2053494D3A202029
:10EEB0002020202020204572726F723A3E20382098
:10EEC00064696769747320496E636F7272656374F5
:10EED0002050494E202053494D2050554B207265FB
:10EEE000717569726564205245504C414345205309
:10EEF000494D2021212120202052656365697665D6
:10EF00006420202020204552524F523A20202020B9
:10EF100020202020202053494D3120697320707219
:10EF20006573656E742E456D70747920736F636BB5
:10EF3000657420312E2053494D3220697320707240
:10EF40006573656E742E456D70747920736F636B95
:10EF5000657420322E204C6F6164696E672074687E
:10EF6000652053494D314C6F6164696E6720746848
:10EF7000652053494D3246584F206E6F7420666F9E
:10EF8000756E642E202044656E6965642046584F76
:10EF90002043616C6C2044656E6965642047534D65
:10EFA0002043616C6C2E202053494D206661696CB2
:10EFB0007572652E2020205245504C414345205308
:10EFC000494D20212121202020204661696C757245
:10EFD0006520202020206F6620737769746368693C
:10EFE0006E672053494D2053494D207265717569F4
:10EFF0007265206F66206F7468657220706172613F
:10F000006D65746572212050756C7365206469614B
:10F010006C6C696E673A206D75737420626520644C
:10F0200069676974732020496E6974696C697A61D3
:10F0300074696F6E202020206F6620534D53204D41
:10F040004F444520202052656164696E6720534D0E
:10F0500053206661696C6973206E6F7420636F6EF4
:10F060006669726D656420636F6D6D616E642065A5
:10F0700072726F72202020204C6973742069732093
:10F0800066756C6C2020534D53206E6F7420707227
:10F0900069766174652020776173206E6F742066D5
:10F0A0006F756E642020436C6F7365642043616CE0
:10F0B0006C6261636B204D656E75202320352E31A7
:10F0C000202020202020434F4E54524F4C20766960
:10F0D0006120534D53204D656E75202320352E320F
:10F0E00020202020202050726976617465205061B4
:10F0F0007373776F726453657474696E6720666F9B
:10F10000722020534D53436F6E6669726D3A202012
:10F110002020202020202020456E74657265642008
:10F1200050535720202020697320494E56414C49A6
:10F13000442021212120436F6E6669726D206F6C1F
:10F1400064205053573A20456E746572206E65777F
:10F1500020505357203A4E6577205052495641541B
:10F160004520505357202020207761732073657409
:10F170002E2020202020436F6E74726F6C206279E5
:10F18000204C4953542076696120534D53203A64F2
:10F19000697361626C6576696120534D53203A65ED
:10F1A0006E61626C652076696120534D53203A2070
:10F1B00020202020202020436F6E6669726D202061
:10F1C000616374696F6E76696120534D53203A64B0
:10F1D000697361626C6576696120534D53203A65AD
:10F1E0006E61626C65202050726976617465206E74
:10F1F000756D62657220666F7220534D53203A64BC
:10F20000697361626C65666F7220534D53203A6575
:10F210006E61626C6520456E7465726564206E6512
:10F220007720505357202077617320756E636F727B
:10F23000726563742E2020534D5320436F6E6669B0
:10F24000726D696E67202020776173206661696C3A
:10F2500065642E2020202050726976617465204EEE
:10F26000756D6265722020436F6E74726F6C2044FE
:10F2700069676974732053657276696365205365A5
:10F280007474696E672E5365727669636520536581
:10F290007474696E672E436F6E6669726D3A2020D2
:10F2A0002020202020202020456E74657265642077
:10F2B00050535720202020697320494E56414C4915
:10F2C0004420212121202053657276696365204EF8
:10F2D000756D626572202020534D5320434F4E546C
:10F2E000524F4C202020202020697320636C6F73C4
:10F2F00065642E202020464D453A204E4F54204133
:10F300004E5357455220464D453A202042555359B9
:10F3100020202020202052413A20204E4F542041CE
:10F320004E535745522052413A20202042555359BE
:10F330002020202020205254523A204E4F54204169
:10F340004E53574552205254523A20204255535959
:10F35000202020202020434C423A204E4F54204170
:10F360004E5357455220434C423A20204255535960
:10F3700020202000434F4E464552454E43453A20FB
:10F3800043616C6C436F6E666572656E6365206D7C
:10F390006F64652020207761732066696E697368E9
:10F3A00065642E20434F4E464552454E43453A2014
:10F3B00057616974434F4E464552454E43453A2086
:10F3C00042757379434F4E462E3A4E6F7420416E0C
:10F3D00073776572434F4E464552454E43453A203A
:10F3E00054616C6B20436F6E666572656E63652059
:10F3F0004D6F6465202020204552524F522021211C
:10F40000212020202020202047534D2043616C6C78
:10F410002020202020206E6F7420616C6C6F776537
:10F42000642E2020205072656669782077617320F1
:10F430006E6F742020666F756E6420696E20746133
:10F44000626C652E4552524F523A202053657475B6
:10F4500070206F667370656564203D3139323030DD
:10F460002062707352342E31202D44415441204D7E
:10F470004F44452D20202020313932303020627019
:10F48000732020204552524F523A202027454348AE
:10F490004F27202020202052455354415254494E9A
:10F4A000472020202743616C6C4261636B27206DED
:10F4B0006F64652020776173206E6F7420736574AC
:10F4C000212121202053494D206E6F7420737570C7
:10F4D000706F72742743616C6C6261636B27204D9F
:10F4E0006F6465204572726F723A20534D53204D00
:10F4F0006F64652020696E697469616C697A6174F2
:10F50000696F6E204669726D77617265205665720B
:10F5100073696F6E50726F6772616D6D20566572A0
:10F5200073696F6E5254522D342E39302D52342E51
:10F53000312D422D475734393052342E312D32354A
:04F540003035313001
:06FFFA007BFFBBE95A0485
:020000040030CA
:0600010022001E83838033
:0600080000800F800F4094
:0200000400F00A
:10000000052FFFF1050FFFF2FFFFFFF1FFFFFFF1EB
:10001000FFFFFFF1FFFFFFF1FFFFFFF1FFFFFFF128
:10002000FFFFFFF1FFFFFFF1FFFFFFF1FFFFFFF118
:10003000FFFFFFF1FFFFFFF1FFFFFFF1FFFFFFF108
:10004000FFFFFFF2FFFFFFF2FFFFFFF2FFFFFFF2F4
:10005000FFFFFFF2FFFFFFF2FFFFFFF2FFFFFFF2E4
:10006000FFFFFFF2FFFFFFF2FFFFFFF2FFFFFFF2D4
:10007000FFFFFFF2FFFFFFF2FFFFFFF2FFFFFFF2C4
:10008000FFFFFFFFFFFFFFFF00FFFFFFFFFFFFFF7F
:10009000FFFF00FFFFFFFFFFFFFFFFFF00FFFFFF6E
:1000A000FFFFFFFFFFFF00FFFFFFFFFFFFFFFFFF5F
:1000B00000FFFFFFFFFFFFFFFFFF00FFFFFFFFFF4E
:1000C000FFFFFFFF00FFFFFFFFFFFFFFFFFF00FF3E
:1000D000FFFFFFFFFFFFFFFF00FFFFFFFFFFFFFF2F
:1000E000FFFF00FFFFFFFFFFFFFFFFFF00FFFFFF1E
:1000F000FFFFFFFFFFFF00FFFFFFFFFFFFFFFFFF0F
:1001000000FFFFFFFFFFFFFFFFFF00FFFFFFFFFFFD
:10011000FFFFFFFF00FFFFFFFFFFFFFFFFFF00FFED
:10012000FFFFFFFFFFFFFFFF00FFFFFFFFFFFFFFDE
:10013000FFFF00FFFFFFFFFFFFFFFFFF00FFFFFFCD
:10014000FFFFFFFFFFFF00FFFFFFFFFFFFFFFFFFBE
:1001500000FFFFFFFFFFFFFFFFFF00FFFFFFFFFFAD
:10016000FFFFFFFF00FFFFFFFFFFFFFFFFFF00FF9D
:10017000FFFFFFFFFFFFFFFF00FFFFFFFFFFFFFF8E
:10018000FFFF00FFFFFFFFFFFFFFFFFF00FFFFFF7D
:10019000FFFFFFFFFFFF00FFFFFFFFFFFFFFFFFF6E
:1001A00000FFFFFFFFFFFFFFFFFF00FFFFFFFFFF5D
:1001B000FFFFFFFF00FFFFFFFFFFFFFFFFFF00FF4D
:1001C000FFFFFFFFFFFFFFFF00FFFFFFFFFFFFFF3E
:1001D000FFFF00FFFFFFFFFFFFFFFFFF00FFFFFF2D
:1001E000FFFFFFFFFFFF00FFFFFFFFFFFFFFFFFF1E
:1001F00000FFFFFFFFFFFFFFFFFF00FFFFFFFFFF0D
:10020000FFFFFFFF00FFFFFFFFFFFFFFFFFF00FFFC
:10021000FFFFFFFFFFFFFFFF00FFFFFFFFFFFFFFED
:10022000FFFF00FFFFFFFFFFFFFFFFFF00FFFFFFDC
:10023000FFFFFFFFFFFF00FFFFFFFFFFFFFFFFFFCD
:1002400000FFFFFFFFFFFFFFFFFF00FFFFFFFFFFBC
:10025000FFFFFFFF00FFFFFFFFFFFFFFFFFF00FFAC
:10026000FFFFFFFFFFFFFFFF00FFFFFFFFFFFFFF9D
:10027000FFFF00FFFFFFFFFFFFFFFFFF00FFFFFF8C
:10028000FFFFFFFFFFFF00FFFFFFFFFFFFFFFFFF7D
:1002900000FFFFFFFFFFFFFFFFFF00FFFFFFFFFF6C
:1002A000FFFFFFFF00FFFFFFFFFFFFFFFFFF00FF5C
:1002B000FFFFFFFFFFFFFFFF00FFFFFFFFFFFFFF4D
:1002C000FFFF00FFFFFFFFFFFFFFFFFF00FFFFFF3C
:1002D000FFFFFFFFFFFF00FFFFFFFFFFFFFFFFFF2D
:1002E00000FFFFFFFFFFFFFFFFFF00FFFFFFFFFF1C
:1002F000FFFFFFFF00FFFFFFFFFFFFFFFFFF00FF0C
:1003000010320000030A323203000032000F32962E
:100310000000000501013000400C100E30202020AC
:10032000202000000000202020202020000020208D
:1003300020202020100E202020202020100E202001
:1003400020202020100E202020202020100E3030D1
:10035000303034323338363738333132333435365F
:1003600037383132333435363738202020202020BA
:10037000202020202020202020202020202020207D
:10038000202020202020202020202020202020206D
:10039000202020202020202020202020202020205D
:1003A000202020202020202020202020202020204D
:1003B000202020202020202020202020202020203D
:1003C00020202020202020202020000100010001EA
:0E03D000000132323232191919196496009662
:0403FC00FAFF000004
:00000001FF
